:020000040000FA
:100000000848040001000000F8270000F82700005D
:10001000F8270000F8270000F8270000F827000064
:10002000F8270000F8270000F8270000F827000054
:10003000F8270000A6090000F8270000F8270000B4
:10004000F8270000CC090000F2090000F8270000A2
:10005000F8270000F8270000F82700002C9F000078
:10006000F8270000F8270000F82700008E10000095
:10007000F8270000C20700002E090000F827000042
:10008000F8270000E8070000F8270000F827000024
:10009000F8270000260A00004C0A00006E09000044
:1000A000F8270000F8270000F8270000F8270000D4
:1000B000F8270000F8270000F8270000F8270000C4
:1000C000F8270000F8270000F8270000F8270000B4
:1000D000F8270000F8270000F8270000F8270000A4
:1000E000F8270000F8270000F8270000F827000094
:1000F00028110000F8270000F82700009C070000E6
:10010000F8270000F8270000F8270000F827000073
:10011000F8270000F8270000F8270000F827000063
:10012000F8270000F8270000F8270000F827000053
:10013000F8270000F8270000F8270000F827000043
:10014000F8270000F827000088070000F8270000C3
:10015000F8270000F8270000F8270000F827000023
:10016000F8270000F8270000F8270000F827000013
:10017000F8270000F8270000F8270000C21100004F
:10018000800A0000F8270000F8270000F827000088
:10019000F8270000F8270000F8270000600800009A
:1001A000F8270000F8270000F8270000F8270000D3
:1001B000F8270000F8270000F8270000F8270000C3
:1001C000F8270000F8270000F8270000F8270000B3
:1001D000F8270000F8270000F8270000F8270000A3
:1001E000F8270000F8270000F8270000F827000093
:1001F000F8270000F8270000F8270000F827000083
:100200000000000000000000F8270000F8270000B0
:10021000F8270000F8270000F8270000F827000062
:10022000F8270000F8270000F8270000F827000052
:10023000F8270000A6090000F8270000F8270000B2
:10024000F8270000CC090000F2090000F8270000A0
:10025000F8270000F8270000F82700002C9F000076
:10026000F8270000F8270000F82700008E10000093
:10027000F8270000C20700002E090000F827000040
:10028000F8270000E8070000F8270000F827000022
:10029000F8270000260A00004C0A00006E09000042
:1002A000F8270000F8270000F8270000F8270000D2
:1002B000F8270000F8270000F8270000F8270000C2
:1002C000F8270000F8270000F8270000F8270000B2
:1002D000F8270000F8270000F8270000F8270000A2
:1002E000F8270000F8270000F8270000F827000092
:1002F00028110000F8270000F82700009C070000E4
:10030000F8270000F8270000F8270000F827000071
:10031000F8270000F8270000F8270000F827000061
:10032000F8270000F8270000F8270000F827000051
:10033000F8270000F8270000F8270000F827000041
:10034000F8270000F827000088070000F8270000C1
:10035000F8270000F8270000F8270000F827000021
:10036000F8270000F8270000F8270000F827000011
:10037000F8270000F8270000F8270000C21100004D
:100380009E480100F8270000F8270000F827000029
:10039000F8270000F8270000F82700006008000098
:1003A000F8270000F8270000F8270000F8270000D1
:1003B000F8270000F8270000F8270000F8270000C1
:1003C000F8270000F8270000F8270000F8270000B1
:1003D000F8270000F8270000F8270000F8270000A1
:1003E000F8270000F8270000F8270000F827000091
:1003F000F8270000F8270000F8270000F827000081
:1004000000480400010000006F0B2300807D2400E1
:1004100000018800000000000B000700A057290021
:100420000100200010000700000020000000E00094
:100430000200320000000200000000007AB5020055
:10044000000000000000FE004440A90040502100D0
:100450000000E0000300320000002000A00188003E
:100460004440A80000000600F8FF2000591C2100AD
:1004700091018800800078000000EB001A0037002E
:100480008180E80032A0B4009101BA00E28040000F
:1004900032A0B4009102BA00E280400032A0B40061
:1004A0000002EB00472BDE00F507B200602CE100F4
:1004B00009003A00330007000700E00002003200A4
:1004C0000059EB00010037000201E8008301E90058
:1004D000F8FF3E00040037006128E100010032000F
:1004E0000082EB00040007001101BA000200E000E6
:1004F000E3FF3A0000000600220007000700E000CA
:10050000020032003159BA00020037008100E800D1
:100510000201E8008301E90017003200190007001A
:100520000700E000020032002159BA000200370043
:100530008100E9000201E8008301E9000D003200BA
:100540000400E00003003A00E280400032A0B40062
:10055000E9FF37000B0007000700E000020032004F
:1005600011D9BA00010037000201E8008301E90057
:10057000F5FF3A008100E800E180400032A0B400BD
:10058000000006000810E600020037000910E6002F
:10059000020037008083EB00000006008003EB00C0
:1005A0000000060091018800800078000000EB0048
:1005B00015003700E280400032A0B4009101BA007B
:1005C000E280400032A0B4009102BA00E280400014
:1005D00032A0B4000002EB00472BDE00F507B200AA
:1005E000602CE10004003A000059EB008301E900AF
:1005F000FDFF3E00040037006128E10001003200E9
:100600000082EB00040007001101BA000200E000C4
:10061000E8FF3A00000006003159BA008301E90002
:100620000C0032002159BA008301E90008003200B1
:100630000400E00003003A00E280400032A0B40071
:10064000F5FF370011D9BA008301E900FAFF3A003B
:100650008100E800E180400032A0B4000000060004
:100660005C9B0400000000004C99040000000000A6
:100670005099040000000000809904000000000070
:10068000A89A040000000000C66C040000000000EE
:10069000F86C040000000000286D04000000000059
:1006A0006A6D040000000000AC6D04000000000052
:1006B000EE6D040000000000346E04000000000035
:1006C000986E040000000000DC6E040000000000D2
:1006D000206F0400000000008E6F04000000000086
:1006E00006700400000000005870040000000000C4
:1006F0007270040000000000FC70040000000000A4
:100700004671040000000000807104000000000039
:10071000BA710400000000004E72040000000000E6
:1007200088720400000000008273040000000000D2
:100730005891040000000000029204000000000034
:10074000D09104000000000034920400000000007A
:1007500066920400000000009A920400000000006D
:100760001A930400000000007693040000000000CB
:1007700048930400000000002095040000000000E1
:10078000A493040000000000F693040000000000A1
:100790009494040000000000C294040000000000D3
:1007A000DA94040000000000F2940400000000004D
:1007B0004A950400000000005CB504000000000041
:1007C000329F040000000000D6B4040000000000C6
:1007D000BCB4040000000000F0B4040000000000FD
:1007E000E4B40400000000008EB404000000000027
:1007F00002C0040000000000BAB9040000000000BC
:1008000090C5040000000000E6A9040000000000FC
:1008100000740400000000001876040000000000CE
:100820002ECB040000000000E2AC04000000000039
:10083000FC80040000000000020AB900001BB9009F
:100840000200B80081004200810043000000060061
:1008500080017800110009008280D8008001FD002D
:10086000110009004288D8008300780000000600CB
:100870006022B800060220000000D0008180D20073
:100880000482D2008582D2000000A0000202520041
:1008900083825A00030031000202420083824A0030
:1008A0000000A1000603E900F3FF3A000000060083
:1008B000839F68000100E00002003D00600010001E
:1008C000E08018000300E00002003D00600111001C
:1008D000E0811900E6FF07004F00E00002003B0046
:1008E00060001000E080180000000600889FBE0035
:1008F0008A9FBE008C1F78000205BE000004BE0067
:100900000006EB00E00F5000E08F5800E00F5900A8
:10091000E08F590007003D006000B8006011B8008A
:1009200008045000898458000A0559008B85590035
:100930001C002000E00F5200E08F5A00E00F5B0027
:10094000E08F5B0002003D000F0007000C00A200DA
:100950000800BE000A01BE001D0107000203BE0020
:100960000002BE000C00E00001003200060007009B
:100970000400BE000601BE004F0678004F05BE0011
:100980004F04BE00000006006000B8006011B8000F
:1009900004025000858258000603590087835900DD
:1009A00000000600881F7800000478005001BE0097
:1009B0004000BE0004004000858048000601490058
:1009C00087814900009CBE000294BE000400E10043
:1009D0000588E1000690E1000798E100020031007F
:1009E000680044001008E8004F047800000006008A
:1009F000F4874700889FBE008A9FBE008C9FBE0080
:100A00008E1F78000205BE000004BE00D4B79F0010
:100A1000E5B79F00F6B79F0087BF9F000000EB007F
:100A2000C0B79F00B0B79F00A0B79F0090B79F00CE
:100A300080B79F000D042000BFB097004FB0970013
:100A4000000140000000E0000F003D004F08DE0004
:100A500000007100C0B79F009E00070001003D002C
:100A600012002000A100070001003D00120020003C
:100A7000A6000700B1000700B60007000F00400005
:100A8000C8FF0700220037004F08DE000006710093
:100A9000CCB79F008F00070001003D00120020002E
:100AA0009200070001003D0012002000970007009F
:100AB000A20007000FB297009FB297002FB39700D4
:100AC000BFB39700A90007000000520081805A00C0
:100AD00002015B0083815B0080B79F0091B79F009C
:100AE000A2B79F00B3B79F000007EB009F0007006D
:100AF0000020E10001A8E10002B0E10003B8E1003C
:100B0000010031001E0020000E005600C0B79F00FB
:100B10004FB297000400E0000700350010002000ED
:100B2000010020006011B800080470008984700082
:100B30000A0571008B8571008D06E900BEFF3A0041
:100B40000400E00003003D00820007000F004000A9
:100B500094FF07004FA897000000E00004003A004F
:100B60000FB497009FB497002FB59700BFB59700BB
:100B7000940007004F0778004F06BE004F05BE00E7
:100B80004F04BE004F01B10000000600881F78002E
:100B900018002000881F780095FF07008F87E90064
:100BA0004F04780000000600801FEB0090FF070054
:100BB0008F87E90000000600889FBE008A9FBE0064
:100BC0008C1F78006E00070007003D0073000700CF
:100BD000E00F5B00E08F5B0007003D003200070084
:100BE0000006EB00040037003400070002003D005F
:100BF0002A0007001C00200072000700E3FF070026
:100C00000203BE000002BE000C00E0000100320042
:100C1000220007000400BE000601BE004F06780057
:100C20004F05BE004F04BE0000000600889FBE00B6
:100C30008A9FBE008C1F78005100070005003D0010
:100C400056000700E00F5B00E08F5B0006003D00F0
:100C5000040037001900070003003D006000B800E1
:100C60006011B8001000070056000700CEFF070013
:100C70000203BE000002BE000C00E00001003200D2
:100C8000060007000400BE000601BE004F06780003
:100C90004F05BE004F04BE00000006006000B80013
:100CA0006011B8000000370004025000858258002F
:100CB0000603590087835900000006000006EB0078
:100CC000E00F5200E08F5A00E00F5B00E08F5B0006
:100CD000000006000180400090B79F000001EB007B
:100CE0008FB097000100E0000000060002007000D5
:100CF00090B79F000180400080B79F000001EB008B
:100D0000FFA897000100E00000000600020070004C
:100D100080B79F00018040006FAA9700CF20DE00BF
:100D200001007000F0AF9F000402420025000700A0
:100D30004F18DE000002720000000600E4AF9F00C2
:100D40000804440089844C000A054D008B854D0041
:100D5000000006003FB29700CFB297005FB3970044
:100D6000EFB3970000FE2F00000006003FB0970091
:100D7000CFB097005FB19700EFB197000000060079
:100D80000205BE000004BE00E00F5000E08F5800D6
:100D9000E00F5900E08F5900000006006000B80025
:100DA0006011B80008045000898458000A055900F1
:100DB0008B8559001C002000E00F5200E08F5A0084
:100DC000000006000800BE000A01BE000000060088
:100DD000889FBE008A9FBE008C9FBE000404B8009E
:100DE0000506B8008904460060854E000606B80076
:100DF0000A054600E0854E000706B8008B05460050
:100E0000040EB800890446000A854E00E0854D00B6
:100E1000050EB8000A0546008B854E00060EB80088
:100E20008B0546000416B8000A0546008B854E0067
:100E30000516B8008B054600041EB8008B05460059
:100E40000800BE000A01BE004F06BE004F05BE00EE
:100E50004F04BE00000006000400FA00E0BF9F003F
:100E6000E4815700812978000002EB000F00370071
:100E70006FB89700904078007FB8970010407800D6
:100E80000402E80080CF5000040032008180FB00A3
:100E90000080FB0000805000070037006FB897000B
:100EA0000000E800E0BF9F009309E800820F5200B5
:100EB000EFFF3A000000EB000080FA00000006009F
:100EC0008001EB0002003700817178008301E800A7
:100ED000828F5100FCFF3A0000000600800078007D
:100EE0003004E000FEFF3A00010050000000E9007D
:100EF000000006008001EB000200370061F079007D
:100F00008301E800828F5100FCFF3A0000000600D8
:100F10003400F800881F780008002000A80188002D
:100F20004F0478008D00A9009D00A9008AA0A800A8
:100F30003400F900004006003600F800809FBE0033
:100F4000829FBE00849FBE00869FBE003400F800D2
:100F500000002000A00188008AA0A9009AA0A90092
:100F60000000EB00D45607003400F9004F03BE0028
:100F70004F02BE004F01BE004F00BE003600F90018
:100F8000004006003600F800809FBE00829FBE0031
:100F9000849FBE00869FBE003400F8000000200041
:100FA000A00188008660A900DA42E20001003D004D
:100FB000065C07003400F9004F03BE004F02BE007C
:100FC0004F01BE004F00BE003600F9000040060091
:100FD0003600F800809FBE00829FBE00849FBE0046
:100FE000869FBE003400F80000002000A0018800A9
:100FF00086E0A900E30B800078C1BF0081CFB30079
:101000000140600078E1B700F0E2A80035C6A90011
:10101000D2F98000C9C2BF000058A3000B003A00FB
:10102000007122000018B80009FE070022C5210047
:101030000001510093002000110009000301D800B5
:1010400080017800CDA2A9000E0037000200E00068
:101050000B0032006F10B80003004000E080480031
:1010600068004000E08048004C09DD004400DE00DC
:1010700000007100C408DE00D0F9880001003700CC
:10108000D3F98800EC62A900E1F980000100E000DA
:10109000020032000300780001000100F0C2A90044
:1010A000C9A2A9003400F9004F03BE004F02BE00E0
:1010B0004F01BE004F00BE003600F90000400600A0
:1010C0003600F800809FBE00829FBE00849FBE0055
:1010D000869FBE003400F80000002000A0018800B8
:1010E0008FA0A900F1F58000BC1EE2000E003A00BE
:1010F00010002000E0F58800200C8000D0F588006A
:1011000000002800C0F58800E0002000B0F588004D
:101110006011B800010078009E2D0700F0F58000F6
:1011200071300700460037006011B80001007800F8
:10113000982D070080C1BF000048A3003D00320089
:1011400037003700210C8000D0F58000008150006E
:10115000D1F58800F0232A000000410021D22200AE
:10116000810F50000C003E00C1F58000B2F58000F8
:101170008201E800100020000300DD000080600014
:101180000000D10080807000C1F588000201E900F4
:10119000B2F5880024003700B0512700000041005C
:1011A000C1782300810F50000C003E00C2F5800082
:1011B000B1F580000100E800130020000018DD00F8
:1011C0000000610013003A000118DD00000071000A
:1011D000C0F588000100E9000F00370020272C002F
:1011E000800F51000E003600C2F58000B1F580007E
:1011F0000100E800130020000018DD00000061007D
:10120000070032000100E9000018DD000000710055
:10121000C0F588000180E900B0F5880002003700C1
:10122000125E070006003700B61EE20001003C0017
:101230000E5E070080C1BF000038A300C1FF3A0066
:101240003400F9004F03BE004F02BE004F01BE0044
:101250004F00BE003600F900004006003600F800DE
:10126000809FBE00829FBE00849FBE00869FBE00FE
:101270003400F80000002000A00188008680A9004A
:1012800042B4800061B48000F0072000808F5000DD
:1012900004003600E06821000200E00004003A008B
:1012A000060037000200E00004003200E070210078
:1012B000020001000000E00001003A00285C070085
:1012C0003400F9004F03BE004F02BE004F01BE00C4
:1012D0004F00BE003600F900004006003600F8005E
:1012E000809FBE00829FBE00849FBE00869FBE007E
:1012F0003400F80000002000A001880087A0A900A9
:1013000051B48000F0072000808F500004003600A8
:10131000E0782100235C0700E0782100030037001B
:10132000E08021001F5C0700E08021008B50070057
:101330003400F9004F03BE004F02BE004F01BE0053
:101340004F00BE003600F900004006003600F800ED
:10135000809FBE00829FBE00849FBE00869FBE000D
:101360003400F80000002000A00188000000EB001D
:1013700021F18000010001008460A9003400F9001F
:101380004F03BE004F02BE004F01BE004F00BE0023
:101390003600F900004006003600F800809FBE00CD
:1013A000829FBE00849FBE00869FBE003400F8006E
:1013B00000002000A001880084E0A90010002000A7
:1013C00041F18000010001003400F9004F03BE002C
:1013D0004F02BE004F01BE004F00BE003600F900B4
:1013E000004006003600F800809FBE00829FBE00CD
:1013F000849FBE00869FBE003400F80000002000DD
:10140000A00188008500A90050F1800066006000FE
:10141000E60F500003003A009000200041F18000E8
:10142000020037002000200061F18000010001006F
:101430003400F9004F03BE004F02BE004F01BE0052
:101440004F00BE003600F900004006003600F800EC
:10145000809FBE00829FBE00849FBE00869FBE000C
:101460003400F80000002000A00188008760A90077
:101470003000200081F18000010001003400F900FB
:101480004F03BE004F02BE004F01BE004F00BE0022
:101490003600F900004006003600F800809FBE00CC
:1014A000829FBE00849FBE00869FBE003400F8006D
:1014B00000002000A00188008780A90090F1800032
:1014C00066006000E60F500003003A00A000200014
:1014D00081F180000200370040002000A1F180006F
:1014E000010001003400F9004F03BE004F02BE00AE
:1014F0004F01BE004F00BE003600F900004006005C
:101500003600F800809FBE00829FBE00849FBE0010
:10151000869FBE00889FBE008A1F78003400F800B6
:1015200000002000A00188000200FA000082800074
:10153000E10F500008003A0094C4BF000068A30007
:1015400005003A008AA4EF008C04A8008C84A8004F
:1015500020002000008288008AC4BF000028A30069
:101560000C00320082C4BF000048A3000900320012
:1015700008012000082488008430EF000001EB00FF
:101580008000EB00400720007D5E07008284A900F8
:101590000824880088C4BF000018A300D4023A00C1
:1015A0008AC4BF000008A300090032008CC4BF0039
:1015B0000008A30006003200C04807009EC0A80033
:1015C0004000200000828800100020005024880085
:1015D0008AC4BF000048A3000D0032008CC4BF00C5
:1015E0000048A3000A0032008284A80008012000FD
:1015F0005824880010002000208488000001EB009F
:101600008000EB00500720005D5E07005824880032
:101610008AC4BF000028A3000F0032008CC4BF00A2
:101620000028A30004003200120020008000EB001C
:1016300030072000525E0700400020005024880040
:101640008650E200010032008670ED008650E20014
:1016500001003A00E04807008A44E20014003D001F
:101660008C44E20012003D00AAC4BF000018A30091
:101670000D003200328280009240900000C8B3001A
:1016800080CF500007003A00808280009040900098
:1016900040C8B30080CF500002003A0068404000CC
:1016A00010419800AA24A9000008200050248800B6
:1016B0008AC4BF000018A3000A0032008CC4BF0017
:1016C0000018A30007003200120020008000EB0089
:1016D000F0FF27002A5E07008EA4EF002000200004
:1016E0005024880000828000E30F50008002360002
:1016F0008CC4BF000038A3007D0232000045EB001F
:101700008AC4BF000038A300790232009024800010
:101710006CF0B7006CD0BF000080FB004400DE001E
:101720006AF0B70080002000502488006CD0BF0011
:101730000038A30004003A006AD0BF000080FB001C
:1017400021072100030037006AD0BF000080FB00A2
:10175000E10621000100400010417800E1406100F5
:101760000104A2001004A10010C870006A50E20039
:1017700058023A00D0C2B30086F0B7006CD0BF0068
:1017800080017800B30FB20015023A006CD0BF00A0
:10179000C00FB20001002100010140003282880028
:1017A000428288004850AA0012409000C043B20014
:1017B00041C3B300814F50009A013A008200780083
:1017C000020321001100900010F179001100900037
:1017D0000000E800900098008301E800E88F5100C5
:1017E000F8FF3A00920098005670EF007630EF0054
:1017F0007C30EF007E30EF008030EF005870EF005B
:1018000081828000114090000074A10090409800F7
:101810005050AA0081828000114090000074A10005
:10182000904098005050AA004182800011409000E2
:101830000074A100904098005C70EF005E30EF00F3
:101840006270EF0063D0BF006370EF0064D0BF0030
:101850006470EF0030D0BF000046B20040013A0093
:1018600031D0BF000080FB0001002000EB0F5000D2
:10187000E08F58003A013E00006001005D00370033
:101880008900370036013700870037003401370000
:1018900006003700080037002D01370053003700DD
:1018A0003300370018013700210137005CF0A80031
:1018B000800020004500370001032100914078009E
:1018C00000C8B30080CF500025013A0000CCB3001F
:1018D0005CF0B70033D0BF00E24F50000800320088
:1018E000E34F500013003200E14F50001E003A0059
:1018F00000122100D082880020012000180037004B
:1019000032D0BF000080FB0000004000E11B21003E
:1019100060807800D0828800D082800020409000D3
:101920005EF0B700D0828000304090005FF0B700DA
:101930000B01370032D0BF00E24F50000A003E00DA
:1019400032D0BF000080FB0000004000011C2100DD
:1019500060807800D0828800D08280001080FB00F8
:10196000F0828800FE0037005C70EF00FC0037005A
:101970005CF0A800AC24EF00AE24EF000000EB0008
:1019800001002100010178000019EB000019EB00B3
:101990000000E800EC0F5000FBFF3A009424A80080
:1019A0004470EF009424A900800021008082880008
:1019B000318288004182880032D0BF0042F0B700F7
:1019C0004250E20003003A0000012000008288003B
:1019D000E300370012002000210421001000200045
:1019E000675D070000022000F8FF37002004210097
:1019F000C90037003870EF003970EF0030D0BF00F9
:101A00007F006000E10F50000B003200E20F500039
:101A10000B0032000000E0001B003A005CF0A80060
:101A20003810A80010848000E10F500016003A0022
:101A30003830A800140037005CF0A800120037000E
:101A40005CF0A8003450E2000500350034D0BF003F
:101A50006F00600000004000A10421000400370076
:101A600034D0BF006F00600000004000010521007D
:101A700060807800104090000028A300020032002F
:101A800010C0B30038F0B7005C50E200B4003D0075
:101A900080032100D08288005C10A80020C0B30021
:101AA0005EF0B700AE00370032D0BF00E14F50000B
:101AB0000B003A0030D0BF007F40600008003A00C1
:101AC0005CF0A80031D0BF00E34F500003003A00A3
:101AD0001000200010848800010037008230EF00E1
:101AE0003250E2009E003A0030D0BF007F406000DC
:101AF000E24F50009A003A0034D0BF006F406000BF
:101B00009700320034D0BF006F006000E20F500039
:101B100093003C000182800000022000808F500072
:101B20008F003A005CF0A8003450E2000A00350053
:101B300034D0BF006F00600000004000A10421000D
:101B400060807800F0BF9F0034D0BF006F0060005D
:101B5000210721000900370034D0BF006F0060006A
:101B6000000040000105210060807800F0BF9F0068
:101B700034D0BF006F006000E106210060C478002F
:101B80000808A30004003A006FF997000224A1009E
:101B9000E2FF9F00030037006FF897000024A000C9
:101BA000E0FF9F003450E2000500350034D0BF0054
:101BB0006F00600000004000A10421000400370015
:101BC00034D0BF006F00600000004000010521001C
:101BD0007FB9970002B0780031D0BF00E34F5000CA
:101BE00014003A007FB897001000E0000B003D00A1
:101BF0003450E2000400350034D0BF006F006000B4
:101C0000210721000300370034D0BF006F006000BF
:101C1000E1062100010040001014A0007FB89700E9
:101C20009040900042C8B30082C0700011409800FC
:101C30004B0037008F84E9006FF897000024A20062
:101C4000E0FF9F00FFB89700114090001100E000F6
:101C50000B003D000074A10090409800FFB8970071
:101C6000114090000064A0009040980022002000E5
:101C7000FFB8970050002000C15C07000200370049
:101C80000064A000904098001924A2000818A30046
:101C900006003A007FB9970000402800120060005B
:101CA00001002800810F500013003A003450E20078
:101CB0000400350034D0BF006F0060002107210010
:101CC0000300370034D0BF006F006000E106210040
:101CD000010040001014A100FFB8970011409000CF
:101CE000B043B2009040980022002000FFB8970057
:101CF000500020001900370012409000B043B2009D
:101D0000104198001600370034D0BF000080FB005F
:101D10004104210001004000D08288005C10A8002E
:101D200010C0B3005EF0B7005CF0A8000C003700F4
:101D30005CF0A80034D0BF000080FB00410421000B
:101D4000220321001241780002F0780004003700DD
:101D50000001EB008000EB0020002000885C070001
:101D60000001EB008000EB0030002000845C0700E5
:101D700094A4A9005C50E200130035006250E20018
:101D800008003D0020C0B30058F0B7007E10E2000C
:101D900001003A00634707007A30EF007830EF0027
:101DA000D000370081C0B300408280000148780035
:101DB000418280000003210090009800C0C8B30059
:101DC00090409800A40037003050E20006003D002B
:101DD00010C0B30058F0B7007C10E2000C003A00CD
:101DE000504707000A00370020C0B30058F0B70082
:101DF00081C0B300408280000148780041828000A9
:101E0000000321009000980040C8B3009040980063
:101E10007A30EF007830EF007610E200B1003A003F
:101E20005E00370058D0BF00E24F50005D003A001E
:101E30001242780063D0BF000080FB004106210001
:101E400091407800C808DD00808070000480FB00AD
:101E5000810F50000400360063D0BF00410621000E
:101E600091407800004278003106210091407800CE
:101E70008180FB0064D0BF004800DD0001007000DD
:101E80008480FB0001005000310621009140780061
:101E900063F0B7004800DE00410621009140780061
:101EA00064F0B7008503210010003700010621000F
:101EB000914078008180FB0061D0BF004800DD00C8
:101EC000010070008280FB0061D87A0001062100C9
:101ED0009140780060F0B7004800DE001106210054
:101EE0009140780061F0B7008301E8000341780079
:101EF00084CF5100EDFF390042828000310621007D
:101F0000914078008180FB0064D0BF004800DD0074
:101F1000010070000A00320080C0B3000049780060
:101F20004182800080032100900098003082800070
:101F3000104090000068A3004E0032004F003700B0
:101F400080C0B30000497800418280000003210076
:101F50009000980040C8B3009040980051062100BE
:101F6000914078008180FB0066D0BF004800DD0012
:101F700001007000070032005106210091407800F6
:101F80008180FB0066D0BF004800DD0001007000CA
:101F90000000010062F0A9009FFF37008E46070095
:101FA000500037008001FD0058F0B7008001FD00AF
:101FB0008010E20008003A0081C0B3004082800037
:101FC00001487800418280000003210090009800C1
:101FD000C0C8B3002A0037000384880041003700DE
:101FE0006CD0BF00B00FB200E80F50003D003A00C7
:101FF00080828000104090004600DE006104600096
:102000005050AA0000828000E80F500008003A00FB
:1020100032D0BF000080FB00B02488000001200007
:102020009604E20001003A0040002000008288008F
:1020300058D0BF00E14F500013003A008003210048
:1020400081828000900098008846070056D0BF002B
:10205000E24F500004003A0041C8B3008082800083
:10206000114098001F003700818280000804E000C2
:1020700002003A0080CCB3000100370080C8B300F2
:1020800090409800170037006250E2000F003D00BA
:1020900051062100914078008180FB0066D0BF008E
:1020A0004800DD00010070000700320051062100E9
:1020B000914078008180FB0066D0BF004800DD00C1
:1020C000010070000000010062F0A9005870EF00EC
:1020D000040037000001EB00C106210020072000AA
:1020E000A75B07000A45E800E44F550084FD3A006D
:1020F0008EC0A9000080FA003400F9004F05780076
:102100004F04BE004F03BE004F02BE004F01BE0091
:102110004F00BE003600F900004006003600F8000F
:10212000809FBE00829FBE00849FBE00869FBE002F
:102130003400F80000002000A00188000400FA002C
:102140008620A90020F38000E10F500003003A0030
:102150000110800030F380000148780093202000B7
:10216000934178008381FB0012F38000C719DE00E1
:102170008F80E9000000EB0004F380000400010000
:1021800080007800E0BF9F00E40F5000190032008B
:1021900006003C00E20F50001000320013003C002B
:1021A000E10F50001C003A0008003700E60F500015
:1021B0001500320011003500E70F50001400320006
:1021C000E80F500014003A00190037007FB897005C
:1021D00030F388000662A800140037007FB897002B
:1021E0001080FB0010108800100037000622A800A5
:1021F0000E00370006A2A9000100370006A2A800C1
:102200000682A800090037000642A8000700370030
:10221000603EEF0005003700E481570042A0200037
:10222000F10F200060672A000E5D070021F388008F
:102230000080FA003400F9004F03BE004F02BE00D8
:102240004F01BE004F00BE003600F90000400600FE
:102250003600F800809FBE00829FBE00849FBE00B3
:10226000869FBE003400F80000002000A001880016
:102270000400FA008A40A90060F38000E10F5000DA
:1022800003003A008110800070F38000014878005C
:1022900093212000934178008381FB0052F380005A
:1022A000C719DE008F80E9001000200044F3800091
:1022B0000400010080007800E0BF9F00E40F5000A0
:1022C0001900320006003C00E20F500010003200FE
:1022D00013003C00E10F50001C003A0008003700DA
:1022E000E60F50001500320011003500E70F5000D6
:1022F00014003200E80F500014003A0019003700B3
:102300007FB8970070F388001662A80014003700A9
:102310007FB897001080FB009010880010003700F5
:102320001622A8000E00370016A2A90001003700EF
:1023300016A2A8001682A800090037001642A800BD
:1023400007003700683EEF0005003700E4815700C2
:1023500042A02000E113200060672A00C15C070052
:1023600061F388000080FA003400F9004F03BE00DA
:102370004F02BE004F01BE004F00BE003600F90004
:10238000004006003600F800809FBE00829FBE001D
:10239000849FBE00869FBE003400F800000020002D
:1023A000A00188000400FA008EA0A900A0F380001C
:1023B000E10F500003003A0081138000B0F3800069
:1023C0000148780093272000934178008381FB0027
:1023D00092F38000C719DE008F80E9002000200002
:1023E00084F380000400010080007800E0BF9F00BB
:1023F000E40F50001900320006003C00E20F5000CC
:102400001000320013003C00E10F50001C003A00A5
:1024100008003700E60F50001500320011003500AB
:10242000E70F500014003200E80F500014003A008B
:10243000190037007FB89700B0F388007662A800D3
:10244000140037007FB897001080FB0090138800BD
:10245000100037007622A8000E00370076A2A900EF
:102460000100370076A2A8007682A8000900370094
:102470007642A80007003700703EEF0005003700E5
:10248000E481570042A02000D117200060672A0095
:10249000745C0700A1F388000080FA003400F900A2
:1024A0004F03BE004F02BE004F01BE004F00BE00F2
:1024B0003600F900004006006D61000074680000FD
:1024C0002E720000616E000064000000666900006A
:1024D0006C6C0000206100007272000061790000E5
:1024E000207700006974000068200000726100001D
:1024F0006E6400006F6D000020760000616C0000CB
:1025000075650000730000006465000073740000CE
:10251000000000005C92000066920000FFFF0000D7
:102520008492000000000000000000006D610000C7
:10253000746800002E6E00007A7300006571000060
:1025400000770000726900007465000020740000CC
:102550006F200000646500007374000020740000A8
:1025600068650000206D000069640000646C000074
:1025700065200000696E000064650000782000009E
:102580006F6600002074000068650000206C000089
:102590006172000067650000737400002073000022
:1025A00065710000756500006E6300006520000025
:1025B0006F660000206E00006F6E00002D7A000034
:1025C000657200006F200000656C0000656D000002
:1025D000656E00007473000020660000726F0000DA
:1025E0006D20000073720000632C0000202D00009D
:1025F0003120000069660000206E00006F7400004A
:10260000206600006F7500006E640000206F0000FF
:102610007220000069660000207300006D610000F8
:102620006C6C00006572000020740000686100009E
:102630006E2000006D6900006E4C0000656E0000A9
:1026400067740000680000007372000063000000FF
:102650006D6900006E4C0000656E0000677400003C
:102660006800000096920000A192000001000000A6
:1026700084920000FFFF000024930000010000008E
:102680002893000000000000000000006D610000C1
:10269000746800002E730000717200007400000066
:1026A00070650000726600006F7200006D730000BC
:1026B0002064000065730000742000003D200000CD
:1026C0007371000072740000287800002920000057
:1026D000656C0000656D0000656E000074200000F0
:1026E00062790000206500006C6500006D650000E7
:1026F0006E740000007800000000000046930000A7
:1027000050930000FFFF000084920000FFFF0000D4
:102710007B93000000000000000000006D610000DD
:10272000746800002E7200006F7400003200000018
:10273000726F000074610000746500007320000077
:10274000762000006F660000206100006E670000C8
:102750006C65000020610000207400006F20000004
:1027600064650000737400000076000000610000E2
:10277000000000008E93000098930000020000000B
:102780008492000002000000B593000001000000E8
:10279000B793000000000000000000006D61000021
:1027A000746800002E6300006F730000007000006A
:1027B00065720000666F0000726D000073200000FB
:1027C0006465000073740000203D00002063000079
:1027D0006F7300002878000029200000656C00005D
:1027E000656D0000656E00007420000062790000D5
:1027F000206500006C6500006D6500006E740000CF
:1028000000000000CE930000D7930000FFFF0000FF
:1028100084920000FFFF00007B9300000000000096
:10282000000000006D610000746800002E7300005D
:10283000696E00000070000065720000666F0000A5
:10284000726D000073200000646500007374000066
:10285000203D000020730000696E00002878000011
:1028600029200000656C0000656D0000656E0000A9
:102870007420000062790000206500006C65000093
:102880006D6500006E7400000000000012940000EE
:102890001B940000FFFF000084920000FFFF000077
:1028A0007B93000000000000000000006D6100004C
:1028B000746800002E610000746100006E32000038
:1028C0000070000065720000666F0000726D00000D
:1028D000732000006465000073740000203D000058
:1028E00020610000746100006E3200002879000051
:1028F0002C78000029200000656C0000656D000048
:10290000656E000074200000627900002065000000
:102910006C6500006D6500006E74000000790000B9
:10292000000000005694000061940000FFFF0000CA
:1029300084920000FFFF00008F940000FFFF000062
:102940007B93000000000000000000006D610000AB
:10295000746800002E6D0000756C00006469000052
:102960007600000070650000726600006F72000063
:102970006D73000020640000657300007420000087
:102980003D200000286100002A620000292F00007D
:1029900063200000696E0000203300003220000038
:1029A0006269000074730000206500006C6500001F
:1029B0006D6500006E740000206200007920000048
:1029C000656C0000656D0000656E0000740000001D
:1029D0006200000063000000A6940000B2940000B2
:1029E000FFFF000084920000FFFF0000B79300008B
:1029F000FFFF0000E8940000FFFF0000EA940000E1
:102A000000000000000000006D610000746800001C
:102A10002E7300006F72000074000000736F0000DE
:102A20007274000020610000727200006179000081
:102A3000206900006E200000706C000061630000DF
:102A40006500000061720000726100007900000002
:102A5000049500000E950000FFFF00002295000085
:102A600000000000000000006D61000074680000BC
:102A70002E61000072670000626F0000756E00003A
:102A8000647300000067000065740000207400009B
:102A900068650000206900006E6400006963000042
:102AA000657300002028000061720000676D00005F
:102AB000696E00002C20000061720000676D00004C
:102AC00061780000292000006F660000207400007B
:102AD00068650000202800006D6900006E69000034
:102AE0006D7500006D2C0000206D00006178000005
:102AF000696D0000756D00002920000076610000FE
:102B00006C75000065730000206F000066200000F7
:102B1000737200006300000061720000676D0000C6
:102B2000696E000000610000726700006D610000C6
:102B3000780000003495000043950000FFFF00007E
:102B400024930000010000008C95000001000000AB
:102B50009395000000000000000000006D6100007F
:102B6000746800002E73000074610000740000009F
:102B700070650000726600006F7200006D730000E7
:102B80002073000074610000746900007374000019
:102B900069630000732000006F6E00002073000066
:102BA00072630000006D0000696E0000006D00009F
:102BB00061780000006D0000656100006E0000009B
:102BC000AE950000B8950000FFFF000024930000C0
:102BD00001000000D395000001000000D79500001F
:102BE00001000000DB950000000000000000000074
:102BF0006D610000746800002E6400006F740000B6
:102C00000077000072690000746500007320000006
:102C10007468000065200000646F000074200000EC
:102C2000707200006F640000756300007420000083
:102C30006F66000020730000726300003120000006
:102C4000616E0000642000007372000063320000B7
:102C5000207400006F2000006465000073740000A1
:102C60002C200000616600007465000072200000E6
:102C700061200000736800006966000074000000B5
:102C80007372000063310000007300007263000083
:102C900032000000736800006966000074000000E4
:102CA000F8950000019600000100000084920000E9
:102CB000FFFF000040960000FFFF00004596000067
:102CC000010000004A960000000000000000000023
:102CD0006D610000746800002E6D000061780000D6
:102CE0000077000072690000746500007320000026
:102CF00074680000652000006D61000078690000C4
:102D00006D7500006D2000006F66000020730000EC
:102D10007263000031200000616E0000642000003A
:102D20007372000063320000207400006F20000006
:102D300064650000737400002C200000656C0000C6
:102D4000656D0000656E000074200000627900006F
:102D5000206500006C6500006D6500006E74000069
:102D6000000000006896000071960000FFFF000060
:102D700084920000FFFF000040960000FFFF00006B
:102D80004596000000000000000000006D6100009A
:102D9000746800002E6D0000696E0000007700006E
:102DA0007269000074650000732000007468000000
:102DB000652000006D6900006E6900006D750000FF
:102DC0006D2000006F660000207300007263000039
:102DD00031200000616E000064200000737200006A
:102DE00063320000207400006F2000006465000062
:102DF000737400002C200000656C0000656D0000FD
:102E0000656E0000742000006279000020650000FB
:102E10006C6500006D6500006E740000000000002D
:102E2000C6960000CF960000FFFF000084920000CD
:102E3000FFFF000040960000FFFF000045960000E5
:102E400000000000000000006D61000074680000D8
:102E50002E640000697600000064000069760000BE
:102E60006964000065730000207300007263000055
:102E700031200000627900002073000072630000BE
:102E800032200000746F00002064000065730000B1
:102E9000742C0000206500006C6500006D6500006A
:102EA0006E7400002062000079200000656C000054
:102EB000656D0000656E000074000000249700003E
:102EC0002D970000FFFF000084920000FFFF00002C
:102ED00040960000FFFF0000459600000000000043
:102EE000000000006D610000746800002E6D00009D
:102EF000756C0000006D0000756C000074690000C6
:102F0000706C00006965000073200000737200009F
:102F100063310000206100006E6400002073000037
:102F20007263000032200000746F00002064000013
:102F300065730000742C0000206500006C650000C3
:102F40006D6500006E7400002062000079200000B2
:102F5000656C0000656D0000656E00007400000087
:102F6000729700007B970000FFFF00008492000032
:102F7000FFFF000040960000FFFF000045960000A4
:102F800000000000000000006D6100007468000097
:102F90002E7300007562000000730000756200006F
:102FA00073740000726100006374000073200000FD
:102FB000737200006332000020660000726F000030
:102FC0006D20000073720000633100002074000067
:102FD0006F20000064650000737400002C20000066
:102FE000656C0000656D0000656E000074200000D7
:102FF00062790000206500006C6500006D650000CE
:103000006E74000000000000C4970000CD9700001F
:10301000FFFF000084920000FFFF000040960000C8
:10302000FFFF0000459600000000000000000000C7
:103030006D610000746800002E610000646400008F
:1030400000610000646400007320000073720000DF
:1030500063310000206100006E64000020730000F6
:103060007263000032200000746F000020640000D2
:1030700065730000742C0000206500006C65000082
:103080006D6500006E740000206200007920000071
:10309000656C0000656D0000656E00007400000046
:1030A0001898000021980000FFFF000084920000A3
:1030B000FFFF000040960000FFFF00004596000063
:1030C00000000000000000006D6100007468000056
:1030D0002E6100006464000073630000616C0000F6
:1030E0006172000000610000646400002073000051
:1030F000636100006C61000072200000746F0000CA
:10310000206500006163000068200000656C00001D
:10311000656D0000656E0000742000006F660000A1
:103120002073000072630000206100006E640000E4
:1031300020730000746F00007265000020720000B0
:1031400065730000756C000074200000746F00004F
:1031500020640000657300007400000073630000C9
:10316000616C0000617200000000000064980000C3
:1031700073980000FFFF000084920000FFFF000032
:103180002493000001000000AE9800000000000041
:10319000000000006D610000746800002E660000F1
:1031A000696C00006C000000666900006C6C000037
:1031B0007320000064650000737400002077000035
:1031C0006974000068200000636F00006E730000E7
:1031D000746100006E74000020760000616C0000D5
:1031E0007565000000760000616C000075650000E8
:1031F00000000000CA980000D4980000FFFF000003
:103200008492000001000000F3980000000000001C
:10321000000000006D610000746800002E63000073
:103220006F70000079000000636F0000706900009B
:1032300065730000207300007263000020740000BA
:103240006F200000646500007374000020650000BA
:103250006C6500006D6500006E7400002062000067
:1032600079200000656C0000656D0000656E00004F
:10327000740000000A99000014990000FFFF00008C
:1032800084920000FFFF0000249300000000000073
:103290000000000000000000930100002403000073
:1032A000B704000048060000DA0700006B090000C0
:1032B000FC0A00008C0C00001C0E0000AB0F00008C
:1032C0003B110000C812000056140000E315000076
:1032D0006E170000F9180000831A00000C1C000093
:1032E000941D00001A1F0000A020000024220000EE
:1032F000A723000029250000A82600002728000099
:10330000A4290000202B0000992C0000122E0000A0
:10331000872F0000FC3000006F320000DF33000018
:103320004E350000BA360000253800008D39000007
:10333000F33A0000573C0000B93D0000173F000081
:1033400074400000CE410000264300007B44000092
:10335000CD4500001D4700006A480000B449000048
:10336000FC4A0000404C0000824D0000C04E0000AE
:10337000FC4F000034510000695200009B530000D4
:10338000CA540000F65500001E57000043580000C4
:1033900064590000835A00009D5B0000B45C00008B
:1033A000C85D0000D75E0000E45F0000EC60000034
:1033B000F1610000F2620000EF630000E9640000C8
:1033C000DE650000D0660000BD670000A768000051
:1033D0008C6900006E6A00004B6B0000246C0000DA
:1033E000F96C0000CA6D0000976E00005F6F00006E
:1033F00023700000E37000009E7100005572000011
:1034000008730000B67300006074000005750000CA
:10341000A575000042760000D97600006C770000A8
:10342000FB77000084780000097900008A790000A9
:10343000067A00007D7A0000EF7A00005D7B0000D4
:10344000C67B00002A7C0000897C0000E47C000030
:10345000397D00008A7D0000D77D00001D7E0000C0
:10346000607E00009D7E0000D67E0000097F000087
:10347000397F0000627F0000877F0000A77F000087
:10348000C27F0000D87F0000EA7F0000F67F0000C6
:10349000FE7F0000FF7F00008C020000DF020000C2
:1034A0003003000080030000D1030000220400006C
:1034B00073040000C204000014050000B3050000FE
:1034C00054060000F10600008F0700002D080000E0
:1034D000CA08000063090000FC090000340B00006A
:1034E0005C0C0000820D0000A40E0000BD0F000067
:1034F000D3100000E2110000E7120000EF140000FA
:10350000CC16000092180000401A0000D61B0000E4
:10351000531D0000B51E00000B20000079220000A2
:103520008D2400006F260000142800009029000060
:10353000E02A0000112C0000252D0000052F0000BE
:1035400089300000D3310000EC320000DD33000090
:10355000AE340000673500000D3600002037000053
:10356000FB370000B23800004A390000CC390000B7
:103570003B3A00009B3A0000F33A0000833B000016
:10358000F43B0000513C00009F3C0000E13C000087
:103590001A3D00004B3D0000783D0000C03D00009A
:1035A000F93D0000283E00004F3E0000703E000044
:1035B0008D3E0000A53E0000BC3E0000E03E000045
:1035C000FD3E0000143F0000283F0000383F00008F
:1035D000473F0000533F00005E3F0000703F000087
:1035E0007F3F00008A3F0000943F00009C3F0000A6
:1035F000A43F0000AA3F0000AF3F0000B83F00001A
:10360000C03F0000C53F0000CB3F0000CE3F0000A0
:10361000D23F0000D53F0000D83F0000DC3F000053
:10362000E03F0000E33F0000E53F0000E83F00000E
:10363000E93F0000EB3F0000EC3F0000EE3F0000E0
:10364000F13F0000F13F0000F33F0000F43F0000B5
:10365000F53F0000F53F0000F73F0000F73F000096
:10366000F93F0000F83F0000FA3F0000FA3F000079
:10367000FA3F0000FB3F0000FB3F0000FC3F000062
:10368000FC3F0000FC3F0000FE3F0000FD3F00004B
:10369000FD3F0000FD3F0000FE3F0000FE3F000038
:1036A000FE3F0000FE3F0000FE3F0000FE3F000026
:1036B00000400000FF3F0000FF3F0000FF3F000010
:1036C000FF3F0000FF3F0000FF3F0000FF3F000002
:1036D000FF3F0000FF3F0000FF3F0000FF3F0000F2
:1036E00000400000004000000040000000400000DA
:1036F00000400000004000000040000000400000CA
:1037000000400000004000000040000000400000B9
:10371000004000000040000000400000746800000D
:10372000796D0000696F00002D490000490000001C
:103730005F6900006400000065760000656E0000AF
:10374000742E0000736F0000757200006365000046
:1037500000650000766500006E7400002E610000B8
:1037600072670000730000005F660000777600005B
:1037700065720000736900006F6E0000005F00005A
:10378000707200006F6400007563000074490000EF
:103790006400000062750000747400006F6E000029
:1037A000732E00005F72000061770000006200006D
:1037B00075740000746F00006E2E000062610000DE
:1037C000636B00007761000072640000006200001B
:1037D00075740000746F00006E2E00006C650000B0
:1037E000667400000062000075740000746F0000D1
:1037F0006E2E0000636500006E74000065720000AC
:103800000062000075740000746F00006E2E0000EE
:10381000666F0000727700006172000064000000B3
:1038200062750000747400006F6E00002E7200005C
:103830006967000068740000006200007574000091
:10384000746F00006E7300002E5F00006D65000055
:10385000616E00000062000075740000746F00006B
:103860006E7300002E5F00006E6F00006973000031
:1038700065000000707200006F7800002E68000084
:103880006F720000697A00006F6E000074610000C2
:103890006C000000707200006F7800002E6700005E
:1038A000726F0000756E0000642E0000616D0000F4
:1038B00062690000616E0000740000007072000018
:1038C0006F7800002E670000726F0000756E0000B8
:1038D000642E000072650000666C000065630000E5
:1038E0007465000064000000707200006F780000D2
:1038F0002E670000726F0000756E0000642E0000DD
:10390000646500006C740000610000006D6F0000D1
:10391000746F0000722E00006C6500006674000079
:103920002E740000617200006765000074000000E2
:103930006D6F0000746F0000722E0000726900004D
:1039400067680000742E0000746100007267000058
:1039500065740000005F0000766200006174000082
:10396000006D00006F7400006F7200002E6C00008C
:1039700065660000742E000073700000656500002D
:10398000640000006D6F0000746F0000722E000074
:103990007269000067680000742E000073700000F8
:1039A00065650000640000006D6F0000746F00002A
:1039B000722E00006C650000667400002E7000001E
:1039C000776D0000006D00006F7400006F720000E2
:1039D0002E72000069670000687400002E700000FD
:1039E000776D000000610000636300000074000058
:1039F000656D000070650000726100007475000064
:103A00007265000000720000633500002E61000046
:103A100064640000726500007373000000720000AF
:103A2000633500002E6300006F6D00006D610000C3
:103A30006E640000006D0000696300002E690000E4
:103A40006E740000656E00007369000074790000F8
:103A5000006D0000696300002E74000068720000B1
:103A600065730000686F00006C640000006D00006A
:103A7000696300002E5F00006D650000616E00004C
:103A800000740000696D0000657200002E70000077
:103A900065720000696F000064000000616300004F
:103AA000632E00005F7400006170000000000000E1
:103AB0008E9B000001000000989B000001000000A8
:103AC0009C9B000020000000A99B00000200000059
:103AD000B49B000001000000BF9B00000500000037
:103AE000CA9B000001000000D79B000001000000FD
:103AF000E79B000001000000F39B000001000000B4
:103B0000019C000001000000109C00000500000066
:103B10001D9C0000050000002B9C00000700000019
:103B20003A9C0000020000004A9C000002000000D5
:103B30005E9C000002000000749C00000100000078
:103B4000869C000001000000989C0000020000001C
:103B5000AB9C000001000000B19C000001000000CF
:103B6000C29C000001000000D49C00000100000085
:103B7000E39C000003000000F39C00000100000033
:103B8000F79C000001000000039D00000100000000
:103B90000F9D0000010000001B9D000001000000BF
:103BA000299D000001000000379D00000200000078
:103BB000419D0000010000004E9D0000000000003B
:103BC00000000000DE000000AD000000CA000000A0
:103BD000FE000000BE000000EF0000000400000036
:103BE000020000005F73000079730000746500003C
:103BF0006D2E00007365000074740000696E000093
:103C0000677300002E6600006C610000736800009E
:103C10000057000072690000746500002074000005
:103C2000686500002073000065740000746900007E
:103C30006E67000073200000696E0000746F000062
:103C4000206600006C61000073680000005F0000E7
:103C50007379000073740000656D00002E7300001E
:103C600065740000746900006E670000732E000028
:103C70007772000069740000650000005772000050
:103C80006974000065200000612000007365000079
:103C900074740000696E0000670000006164000039
:103CA000647200006573000073000000766100001C
:103CB0006C750000650000005F7300007973000000
:103CC000746500006D2E00007365000074740000C0
:103CD000696E0000677300002E72000065610000CD
:103CE0006400000052650000616400002061000073
:103CF0002073000065740000746900006E670000A6
:103D0000005F00007379000073740000656D0000AF
:103D10002E720000656200006F6F000074000000EA
:103D200052650000626F00006F7400002074000094
:103D300068650000206D000069630000726F00007C
:103D4000636F00006E740000726F00006C6C000006
:103D50006572000000420000616300006B770000A4
:103D6000617200006420000062750000747400003D
:103D70006F6E000020730000746100007475000015
:103D80007320000063680000616E0000676500003A
:103D9000640000004C6500006674000020620000B2
:103DA00075740000746F00006E20000073740000D2
:103DB00061740000757300002063000068610000FA
:103DC0006E6700006564000000430000656E00003F
:103DD00074650000722000006275000074740000B9
:103DE0006F6E0000207300007461000074750000A5
:103DF0007320000063680000616E000067650000CA
:103E000064000000466F00007277000061720000DD
:103E10006420000062750000747400006F6E000082
:103E200020730000746100007475000073200000AE
:103E300063680000616E00006765000064000000B8
:103E4000526900006768000074200000627500007D
:103E5000747400006F6E0000207300007461000035
:103E6000747500007320000063680000616E00003C
:103E70006765000064000000627500007474000053
:103E80006F6E000073000000427500007474000043
:103E90006F6E000073200000766100006C750000FA
:103EA00065730000207500007064000061740000FC
:103EB0006564000000700000726F00007800000070
:103EC000507200006F780000696D00006974000096
:103ED00079200000766100006C75000065730000B9
:103EE00020750000706400006174000065640000CB
:103EF00000740000617000000041000020740000A8
:103F000061700000206900007320000064650000FB
:103F100074650000637400006564000000410000E7
:103F200063630000656C0000657200006F6D000047
:103F3000657400006572000020760000616C00006E
:103F4000756500007320000075700000646100005A
:103F500074650000640000006D69000063000000EB
:103F60004669000072650000642000007768000068
:103F7000656E0000206D000069630000726F000034
:103F8000706800006F6E000065200000696E000020
:103F9000746500006E7300006974000079200000F1
:103FA0006973000020610000626F00007665000008
:103FB000207400006872000065730000686F0000E4
:103FC0006C640000007300006F7500006E640000F8
:103FD0002E660000696E00006973000068650000CD
:103FE0006400000046690000726500006420000063
:103FF00077680000656E00002074000068650000AE
:10400000207000006C6100007962000061630000B4
:104010006B2000006F66000020610000207500002A
:104020007365000072200000696E00006974000072
:10403000696100007465000064200000736F000077
:10404000756E0000642000006973000020660000A7
:10405000696E00006973000068650000640000007C
:10406000546500006D70000065720000617400000E
:104070007572000065200000766100006C7500001C
:104080006520000075700000646100007465000028
:10409000640000007263000035000000524300001D
:1040A000352000006D65000073730000616700003B
:1040B00065200000726500006365000069760000FD
:1040C00065640000006D00006F7400006F720000F6
:1040D000004D00006F7400006F720000207400003B
:1040E000696D00006572000000740000696D0000D9
:1040F0006572000030000000546900006D6500002A
:104100007220000030000000746900006D6500003E
:104110007231000000540000696D000065720000FB
:104120002031000000000000D79B0000AB9E000083
:10413000E79B0000CA9E0000F39B0000E59E000084
:10414000019C0000029F0000109C0000209F0000C6
:104150003C9F0000449F00005B9F0000609F0000A8
:10416000799F00007D9F0000F39C00008F9F00005E
:10417000AC9F0000B09F0000E39F0000F29F000092
:10418000F79C000030A000004AA000004EA00000F4
:1041900063A0000069A0000075A000007CA00000E2
:1041A00084A000008BA000000000000000000000C0
:1041B0004164000064720000657300007320000019
:1041C0006F750000742000006F660000207300000F
:1041D00065740000746900006E67000073000000E1
:1041E000536C000065650000702000006D6F0000DA
:1041F00064650000206E00006F74000020730000F2
:1042000075700000706F000072740000656400003B
:1042100000450000727200006F7200003A2000003A
:104220006D6900006E2000003D3D00002030000060
:10423000784600004646000046460000464600001C
:10424000462000002100000045720000726F00004F
:10425000723A0000205500006E610000626C0000A0
:1042600065200000746F0000206600006C61000093
:10427000736800002062000079740000656300002C
:104280006F64000065200000283100002920000034
:104290002100000045720000726F0000723A0000B9
:1042A000205500006E610000626C00006520000077
:1042B000746F0000206600006C61000073680000ED
:1042C0002062000079740000656300006F640000E4
:1042D0006520000028320000292000002100000095
:1042E00045720000726F0000723A00002055000015
:1042F0006E610000626C000065200000746F0000B9
:10430000206600006C6100007368000020620000FD
:1043100079740000656300006F6400006520000090
:10432000283300002920000021000000466C000016
:1043300061730000686900006E670000204F000094
:104340004B000000736F0000756E0000642E0000CB
:10435000776100007665000000530000657400007E
:104360002074000068650000207000007269000081
:104370006D61000072790000207700006176000016
:10438000652000006F660000207400006865000072
:10439000207400006F6E000065200000676500005B
:1043A0006E65000072610000746F00007200000012
:1043B0007761000076650000007300006F750000F3
:1043C0006E6400002E66000072650000710000003F
:1043D000506C0000617900002066000072650000EA
:1043E00071750000656E00006379000000480000F0
:1043F0007A00000064730000006C00006564000037
:10440000732E0000746500006D700000657200007E
:1044100061740000757200006500000053650000C3
:10442000742000006E740000632000006C650000C2
:10443000640000007265000064000000626C00000F
:1044400075650000006C000065640000732E0000BC
:10445000736F0000756E000064000000536500007B
:1044600074200000736F0000756E0000642000006F
:104470006C650000640000006C65000064000000D2
:104480006C650000647300002E7200006300000081
:10449000536500007420000072630000206C00006F
:1044A00065640000006C000065640000732E00006D
:1044B000707200006F7800002E760000005300003C
:1044C00065740000207600006572000074690000C9
:1044D000636100006C200000707200006F780000C3
:1044E000696D000069740000792000006C650000AF
:1044F00064730000006C0000656400002030000060
:10450000006C00006564000020310000006C0000B9
:1045100065640000732E0000707200006F78000068
:104520002E68000000530000657400002068000041
:104530006F720000697A00006F6E00007461000005
:104540006C200000707200006F780000696D000040
:1045500069740000792000006C650000647300003D
:10456000006C00006564000020320000006C000058
:104570006564000020330000006C000065640000EA
:1045800020340000006C000065640000203500004D
:10459000006C00006564000020360000006C000024
:1045A0006564000020370000006C000065640000B6
:1045B000732E000062750000747400006F6E0000BE
:1045C0007300000053650000742000006275000055
:1045D000747400006F6E0000732000006C650000B2
:1045E00064730000006C000065640000732E00001E
:1045F000626F0000747400006F6D00002E6C00008C
:10460000656600007400000053650000742000001F
:104610005247000042200000626F0000746F0000EB
:104620006D2000006C65000066740000206C0000C6
:10463000656400000067000072650000656E0000A0
:10464000006C000065640000732E0000626F0000C3
:10465000747400006F6D00002E7200006967000026
:1046600068740000005300006574000020520000D0
:1046700047420000206200006F7400006F6D000070
:10468000207200006967000068740000206C000060
:1046900065640000006C000065640000732E00007B
:1046A000746F00007000000053650000742000006B
:1046B0005247000042200000746F0000702000008C
:1046C0006C650000640000006C650000647300000D
:1046D0002E63000069720000636C0000650000003A
:1046E00053650000742000006369000072630000DD
:1046F000756C00006172000020720000696E00009D
:10470000672000006C650000647300000073000007
:104710006F7500006E6400002E7300007973000056
:10472000746500006D0000005374000061720000A9
:1047300074200000706C000061790000626100006C
:10474000636B0000206F000066200000737900009A
:1047500073740000656D0000207300006F75000029
:104760006E640000204E0000004E00000073000048
:104770006F7500006E6400002E720000657000000E
:104780006C61000079000000537400006172000049
:1047900074200000706C000061790000626100000C
:1047A000636B0000206F000066200000724E000066
:1047B0002E77000061760000007300006F75000026
:1047C0006E6400002E7000006C6100007900000033
:1047D000537400006172000074200000706C0000CF
:1047E0006179000062610000636B0000206F0000CF
:1047F00066200000704E00002E77000061760000F9
:10480000007300006F7500006E6400002E720000DF
:10481000656300006F7200006400000053740000C4
:10482000617200007420000072650000636F000078
:1048300072640000696E0000672000006F6600006F
:10484000207200004E2E000077610000760000000C
:104850005F6C000065640000732E0000736500004B
:1048600074000000536500007420000074680000AC
:10487000652000006C6500006400000062720000AA
:1048800069670000687400006E65000073730000C3
:1048900000700000000000000000000000000000A8
:1048A0000000000000000000000000007200000096
:1048B00000000000000000000000000000000000F8
:1048C0000000000000720000000000000000000076
:1048D00000000000000000000000000000000000D8
:1048E0007300000000000000000000000000000055
:1048F000000000000000000000450000727200008F
:104900006F7200003A200000736100006D700000BB
:104910006C650000732000006D750000737400006A
:104920002062000065200000696E0000205B00002E
:104930002D310000323800002C31000032370000E9
:104940005D200000726100006E67000065000000DD
:1049500030110000070000007C1500000700000077
:10496000C81900000700000000000000000000005F
:1049700030110000070000007C1500000700000057
:104980000000000000000000C81900000500000041
:10499000BE0A00000400000000000000000000004B
:1049A0009C27000002000000AB2200000100000074
:1049B0009D1C000002000000FB1800000200000027
:1049C0002D32000001000000322D00000100000027
:1049D0004628000002000000E82600000100000058
:1049E000BF22000002000000FB18000002000000CF
:1049F000FF32000001000000C6200000010000009E
:104A0000762F0000020000002C2E000001000000A4
:104A1000CE2C000001000000FD3900000200000063
:104A20000000000000000000E40C0000070000008F
:104A3000301100000D000000C81900000700000040
:104A400000000000000000004C040000070000000F
:104A500098080000070000000000000000000000AF
:104A6000781E00000D000000001900000700000083
:104A7000EC130000070000003011000007000000E8
:104A8000480D0000070000000000000000000000CA
:104A9000480D00000D00000030110000070000006C
:104AA000EC130000070000000019000007000000E0
:104AB000781E000007000000000000000000000059
:104AC000733000002E770000617600000073000054
:104AD000322E000077610000760000007333000082
:104AE0002E7700006176000000730000342E000075
:104AF0007761000076000000733500002E7700001B
:104B00006176000000730000362E0000776100001F
:104B100076000000733700002E77000061760000F9
:104B200000000000809A0000904100008E410000CB
:104B30008F800000454500004549000049490000BC
:104B40008E8F000090920000924F0000994F00005D
:104B500055550000599900009A9B00009C9D00004B
:104B60009E9F0000414900004F550000A5A5000090
:104B7000A6A70000A8A90000AAAB0000AC21000075
:104B8000AEAF0000B0B10000B2B30000B4B5000099
:104B9000B6B70000B8B90000BABB0000BCBD000049
:104BA000BEBF0000C0C10000C2C30000C4C50000F9
:104BB000C6C70000C8C90000CACB0000CCCD0000A9
:104BC000CECF0000D0D10000D2D30000D4D5000059
:104BD000D6D70000D8D90000DADB0000DCDD000009
:104BE000DEDF0000E0E10000E2E30000E4E50000B9
:104BF000E6E70000E8E90000EAEB0000ECED000069
:104C0000EEEF0000F0F10000F2F30000F4F5000018
:104C1000F6F70000F8F90000FAFB0000FCFD0000C8
:104C2000FEFF0000222A00002B2C00003A3B00006F
:104C30003C3D00003E3F00005B5D00007C7F0000CB
:104C4000000000005A3A00005C6D00006F6C00002C
:104C50006F6C0000655C000069320000635C00005E
:104C60002F690000326300005F700000726900006D
:104C7000762E0000680000005A3A00005C6D0000CB
:104C80006F6C00006F6C0000655C00006932000012
:104C9000635C00006D6100007374000065720000C9
:104CA0005F700000726F0000746F0000636F00009F
:104CB0006C2E0000630000005A3A00005C6D00009A
:104CC0006F6C00006F6C0000655C000069320000D2
:104CD000635C00002F690000326300005F70000019
:104CE00072690000762E0000680000005A3A000049
:104CF0005C6D00006F6C00006F6C0000655C000074
:104D000069320000635C00006D6100007374000094
:104D1000657200002E630000000000005249000090
:104D2000464600000000000000000000574100005F
:104D300056450000666D0000742000001000000061
:104D4000000000000100000001000000841E0000BF
:104D500000000000841E00000000000001000000B0
:104D600008000000646100007461000000000000A1
:104D7000000000005A3A00005C6D00006F6C0000FB
:104D80006F6C0000655C0000746900006D650000D8
:104D9000725C0000746900006D650000722E0000F6
:104DA0006300000001000000000000000800000097
:104DB00000000000400000000000000000010000B2
:104DC000000000005F4C00004F4700004455000009
:104DD0004D5000002E23000040210000005F000025
:104DE00054450000535400004D4F0000442E000075
:104DF0002340000021000000564D0000434F0000FA
:104E0000444500002E410000424F00000000000019
:104E10005A3A00005C6D00006F6C00006F6C00007F
:104E2000655C000069320000635C00002F690000CF
:104E3000326300005F70000072690000762E00008F
:104E4000680000005A3A00005C6D00006F6C0000C2
:104E50006F6C0000655C0000666C00006173000010
:104E6000685C0000666C000061730000682E000042
:104E7000630000005F7000006F7700006572000043
:104E80006F66000066000000506F0000776500004C
:104E9000726F000066660000000000006D6D00008B
:104EA0006137000036360000302E0000630000003D
:104EB00000000000000000000000000000000000F2
:104EC0000400FA00889FBE008A9FBE008C9FBE002F
:104ED000800578000005EB00A925210043EF2100A3
:104EE000C8EE210006EF21006D2C21008C0220006D
:104EF000F0835700990078006B007D00010150009D
:104F000013004100800978008D0F5000010034002B
:104F10008D097800A0D32E00930F100001003D00F2
:104F2000800978000100E00007003A009600E800E0
:104F3000010B780070022000808F500003003400C5
:104F40000C0B780001003700000BEB00960F1600E9
:104F500004003A00800BEB008009EB00000CEB0032
:104F6000060037006512B9001300780032002000F7
:104F7000110009000200D800840B4000980078005E
:104F80003780400022002000110009000200D800F4
:104F9000001C7800E00498000A85E8008984E80095
:104FA0008381E8000683E800E40F5500D1FF3A0052
:104FB00060F780005D40070070F780007B400700CD
:104FC0004F06BE004F05BE004F04BE000080FA0031
:104FD000000006000000EB00A0F78800B0F7880092
:104FE0008002200080F7880090F78800000006000B
:104FF0000000FE000040060000000000000000006D
:1050000000000000000000000000000000000000A0
:105010000000000000000000000000000000000090
:105020000000000000000000000000000000000080
:105030000000000000000000000000000000000070
:108000008001EB000200370061F079008301E80095
:10801000828F5100FCFF3A00000006008001EB0057
:108020000200370001F079008301E800828F5100DF
:10803000FCFF3A0000000600889FBE008A9FBE0039
:108040008C9FBE008E1F7800000478000206BE00E0
:1080500050159000E0159000820F5500838F5D0051
:1080600034003200404090000004E0002100320063
:10807000EE022000080747001840900014C0B3002B
:108080000A01BE008E007800CF2407000000E00047
:1080900026003A004044980078089000881090002C
:1080A00058099000E80990000000410081804900D3
:1080B000800F5500818F5D000E003100B8449000A4
:1080C0000A00370058089000E80890000A054000B0
:1080D0008B8548001840900014C0B3000A01BE0010
:1080E0008E007800B82407008944E900E1CF5400ED
:1080F000F4FF3E00E00F5600E08F5E000D003200FE
:10810000E1022000888040001840900014C0B300B5
:108110000C01BE00702407000000E00003003A00DC
:108120005C1498006D1498000300370010002000C4
:10813000010037000000EB004F0778004F06BE003B
:108140004F05BE004F04BE0000000600881F7800E7
:108150000004780062025100E0825900C0089000DB
:108160003008900062005000E08058006011B800B4
:10817000800F5200818F5A00090031002841900081
:108180000281FB00030020000400BE00AAE10700FA
:1081900038119000C8119000000141008181490010
:1081A0000200BE004F04780000000600889FBE0059
:1081B0008A9FBE00000578000204BE00E10F510056
:1081C000E08F590079003600C00890003008900018
:1081D000800F5100818F5900740031001A407800DF
:1081E000E24F50002E003200E34F500043003200B7
:1081F000E14F500070003A00820478000200D10084
:10820000000441004941DE007A0890008A10900085
:1082100002014000E08148000A00780086FF070064
:108220000000E00064003A0008007800F01FB2008F
:10823000E002B0000A0040009085FB000804E8005E
:108240004941DE007A0890008A1090000201400047
:10825000E08148000A00780077FF07000000E00096
:1082600055003A00F81FB200E0022000080040006C
:108270000A0040001080FB004800DD00808075008F
:108280000908A300020032004408DE0002003700A3
:10829000F0FF20000080600001002000480037004F
:1082A0004818DD004811DE0002017000C819DE0028
:1082B0007A0890008A1090000201400083814800F3
:1082C0000A0078005CFF07000000E0003A003A0076
:1082D000E20220000A0141000800440089804C00AD
:1082E000F01FB20000014100124090004800DD0084
:1082F0009280FB0001007000E7FF37004918DD00A5
:108300004711DE0002017000C719DE007A089000F4
:108310008A10900002014000838148000A00780022
:1083200045FF07000000E00023003A00E4022000BF
:108330000A0242004248DD00CE40DE0081007000AB
:108340004240DD00F01FB2000002420034419000C4
:10835000C811DD0002002000244090008080FB0056
:108360000000200000017100818171001440900024
:108370004800DD00010020000001710081817100D2
:10838000144078000080FB00010020000001710013
:1083900081817100F0FF20000300600080037800FD
:1083A000020378000600BE00050037001000200020
:1083B00001002000020037000080EB008080EB000D
:1083C0004F05BE004F04BE0000000600E4874700D2
:1083D000889FBE008A9FBE008C9FBE008E1F7800C3
:1083E000000578000204BE000406BE00E10F510043
:1083F000E08F59009F003600C008900030089000C0
:10840000800F5100818F59009A0031001A40780086
:10841000E24F500044003200E34F50005900320058
:108420002B002000E14F50008F003A000200D100E5
:10843000800441004949DE007A0890008A109000CB
:1084400002014000E08148000A007800FAFE0700BF
:10845000800578000000E00083003A00EE02200072
:108460000A07470009007800F01FB200000147002A
:10847000610064000100200080BF9F000000E00058
:108480000500320012427800EF4062004460DD00D7
:1084900001407000010037000C407800004978006E
:1084A0000904E80010C0B300404598004941DE00CF
:1084B0007A0890008A10900002014000E081480094
:1084C0000A007800DCFE0700800578000000E0006C
:1084D00065003A00F81FB200880147000FB8970006
:1084E0000000E000050032004C69DD004460DE0061
:1084F00000007100C468DE000800370002CFB3003E
:1085000013416100486ADD004860DE00000072002F
:10851000C868DE006F40600000407100804978004C
:108520008005EB00500037004818DD004811DE00E0
:1085300002017000C819DE007A0890008A109000CD
:1085400002014000838148000A007800BAFE07005B
:10855000800578000000E00043003A00E0022000BF
:108560000A0040000801440089814C00F21FB2005B
:10857000020040000C487800C860DE0011409800FE
:1085800039003700491ADD004711DE000201720090
:10859000C719DE007A0890008A109000020140009E
:1085A000838148000A007800A3FE07008005780058
:1085B0000000E0002C003A00E40220000A02420021
:1085C0004248DD00CE40DE00810070004240DD0008
:1085D000F01FB20000024200E30342000483E800FF
:1085E0008402E80017417800C811DD000200200075
:1085F000164078008080FB00000020000001710020
:10860000818171001580FB004800DD000100200021
:108610000001710081817100144078000080FB002E
:1086200001002000000171008181710000002F0015
:108630000300600001002000C000DD0000002000F9
:108640000000760081807600004A78004801DE0054
:10865000824A78004009DE0003002000024B7800C7
:108660004808DE00804B780010C0B30040459800F9
:10867000010037002B0020000B0078004F07780026
:108680004F06BE004F05BE004F04BE004F00B100B4
:10869000000006000400FA00889FBE008A9FBE000A
:1086A0008C1F78000006780092BF9F00A3BF9F0038
:1086B000E00F5100E08F59000B003A005005900088
:1086C000E0059000E00F5500E08F5D0015003200DE
:1086D000C008900030089000800F5500818F5D0029
:1086E00010003100110037001FB99700AFB9970093
:1086F000AEFE07000001BE00E10F5000E08F580001
:108700004D0036003C089000CC089000800F5100CE
:10871000818F59004C0039001FBD9700AFBD9700F5
:10872000020037001A0020000B0020000A04BE00DF
:1087300061044400E0844C003C089000CC089000A8
:10874000800F5400818F5C0005003900E10F550057
:10875000E08F5D003B00360028002000090020006B
:108760000801BE000C00780090FE07000001BE006A
:10877000E00F5000E08F58000A003200E10F400087
:10878000E08F480030003200E10F5000E08F5800C9
:108790002D0032008A0F54008B8F5C0029003200BC
:1087A000E3FF3700F4FF2F00F5FF20000801BE00B3
:1087B0000C00780005FF07000000E0001A003A00F6
:1087C0001FB89700AFB89700E00F5000E08F580037
:1087D000060032000802BE000001BE000C00780056
:1087E000FAFE07000000E0000F003A00580698006B
:1087F000690698007C0090008C089000E10F400012
:10880000E08F48000600320061005000E080580010
:1088100070069800010E980010C0B30050469800F2
:108820000801BE00080037000081EB008081EB00EA
:10883000E10F50000400320012002000030020006D
:10884000010037006011B8000200BE004F0678003A
:108850004F05BE004F04BE000080FA000000060075
:10886000889FBE008A1F78000004BE002104980083
:1088700030019000C0019000E10F5100E08F5900DD
:10888000480032001002780034089000C4089000BC
:10889000800F5100818F590042003100E00F5100DC
:1088A000E08F590016003A0030C0B300944F10001A
:1088B00005003A0014119000A4119000E00F51003F
:1088C000E08F59000E003A006000B8005004980094
:1088D0006104980044009000808F54003100310002
:1088E0004448DE0014119000A411900000004100E3
:1088F000E080490070049800010C98001F003700C8
:10890000244090000080FB004405DD00100037008B
:108910001800780025FE07000001BE00E10F4000AE
:10892000E08F48001D003200E10F5000E08F58003A
:108930001C00360018007800C00890003008900035
:10894000800F5100818F5900160031008A84540035
:108950008A8F5400EEFF310052049800630498009F
:1089600018007800F9FD07004449DE0002014000CC
:10897000E081480072049800030C9800E002200097
:10898000980040006F8064004500DD00808040005A
:10899000110C98000000EB000300370010002000CD
:1089A00001003700200020004F0578004F04BE0072
:1089B00000000600889FBE008A9FBE008C9FBE00FC
:1089C0008004780001047800200090000006E80090
:1089D000770032007900900089089000E00F500085
:1089E000E08F580072003200EF06660068003A001F
:1089F00061004000E0804800F0049800810C98007D
:108A00001902780059019000E9019000E00F51002F
:108A1000E08F590004003A0044009000800F560097
:108A20005B00390062003700C460DE002440900023
:108A30000080FB000000E9008080600054003A00E4
:108A400004007800D9FD07000005BE00E10F5000CA
:108A5000E08F580058003600E10F4000E08F4800DA
:108A6000570032001902780034089000C4089000C2
:108A7000800F5500818F5D003E0039000800E00046
:108A80004B00320059019000E90190000400780089
:108A900000FF07000005BE0070002000E00F550039
:108AA000E08F5D0047003200E10F5500E08F5D0070
:108AB00041003200E10F4500E08F4D0040003200E0
:108AC0006011B800190078005BFD07000000E000AD
:108AD0003B003A00E1022000198040000220200003
:108AE0008D0078004DFD0700190478000A01BE00D2
:108AF0000800780095FD0700501498006114980054
:108B00000D0478000F00370010C0B30040429800F9
:108B10006011B8001900780047FD07000804E8005C
:108B20000000E00026003A00190178005210900081
:108B3000E210900061004000E08048005011980071
:108B4000611198001902780024409000804F540071
:108B5000EDFF39000881FB00030020005410900055
:108B6000E4109000020050008380580050129800DA
:108B700061129800DA049800EB0498000A01BE0024
:108B80001900780071FD0700F0049800810C98002E
:108B9000AC049800E102200019804000C568DD00A7
:108BA00001004000900C98000000EB000500370029
:108BB00040002000030037002000200001003700A3
:108BC000100020004F06BE004F05BE004F04BE003F
:108BD00000000600881F7800E8022000000444001E
:108BE0001040900014C0B30088007800BA2107003C
:108BF000320020000000E0003F003A0078F89300C7
:108C00004800DD00E8F893008180FB00010070005F
:108C10002200200051A52A00810F500036003A00A2
:108C200018799000C811DD0002002000087890003B
:108C30008080FB0000002000000171008181710034
:108C4000787090004800DD000100200000017100F4
:108C500081817100687090000080FB00010020009D
:108C600000017100818171000380FB0080027800A7
:108C7000020278000400BE006614240047052000AC
:108C8000860F5000878F58001A00320058D190008C
:108C9000C811DD000200200048D090008080FB0059
:108CA00000002000000171008181710038D0900027
:108CB0004800DD0001002000000171008181710089
:108CC00028D090000080FB0001002000000171000E
:108CD000818171000380FB0080027800020278002D
:108CE0000400BE0012002000860F5000878F58003D
:108CF00001003A000001EB00020078004F04780008
:108D000000000600000178000000E0000C003200C6
:108D10001004E0000A00320030009000810F500083
:108D200007003A00124090006421070061006000D3
:108D30003100200003003A00800078000100370075
:108D4000910020000100780000000600B200200021
:108D50000004E00009003A0002FA80000200E0008E
:108D600001003200004978000100E00001003200FB
:108D70008048780001FA88000001EB0002007800CA
:108D800000000600EF03B000889FBE008A9FBE006F
:108D90008C9FBE008E1F7800E0B79F00010778000F
:108DA0000008EB007F406100C0DF9F007E4461004F
:108DB0009100FB0000FD2F0000814000E90F5100F1
:108DC00008003E009E409000A0C3B30080CF50003A
:108DD00004003A000E87E800B90020000200E0001D
:108DE000A2013A000AFA80009AA79F00C900200059
:108DF0000A00E0009D0132001A04E0000A0032007F
:108E00001A4090002D2107000080FB000008A300FD
:108E100005003A000804E000910132000028A30098
:108E20008D013A008E0137000040EB00004D7800C4
:108E300010459800942007000080FB0039002000B6
:108E40000008A30089013A000804E0000200320093
:108E50000028A30080013A006011B8000A007800E1
:108E60005CFF07006011B80092B79F00A3B79F0096
:108E7000E14F50001B003A00E40220000A024200C9
:108E800024C093000004E0007701320014C993006D
:108E9000C811DD000200200004C893008080FB00A0
:108EA00000002000000171008181710074C09300F6
:108EB0004800DD0001002000000171008181710087
:108EC00064C093000080FB000100200000017100DD
:108ED0008181710092B79F00A3B79F000A007800BC
:108EE0003CFF070019002000E34F50005F013200F3
:108EF0000004E0005C013A00EB0220008A85450096
:108F00002A7890004800DD009A7890008180FB006C
:108F10000100700001202000810F500052013A0032
:108F2000DAC09000C808DD004AC090000080FB0055
:108F300080807000610AB80012003A007B619000E6
:108F4000C811DD00020020006B6090008080FB00F3
:108F50000000200000017100818171005B609000C1
:108F60004800DD00010020000001710081817100D6
:108F70004B6090000080FB000100200000027100A7
:108F800081827100540D9800650D9800EA78900078
:108F9000314598000140E900E14F500032013E00A8
:108FA0000181FB00030020000400BE0022DE070058
:108FB000F0B79F0081BF9F00BA7B900027459800C3
:108FC0000704E000280132000780FB008000E90070
:108FD0000100600024013A000AC090004800DD0052
:108FE000FA7890008180FB0001037000460598002C
:108FF0006F0063001C013A00AAC09000C808DD00A1
:109000001AC090000080FB0080807000610AB800E8
:1090100012003A003B619000C811DD000200200000
:109020002B6090008080FB00000020000001710098
:10903000818171001B6090004800DD00010020006C
:1090400000017100818171000B6090000080FB00C5
:10905000010020000002710081827100DA78900026
:10906000C808DD004A7890000080FB000080700096
:10907000FD0032006104B800C8B79F00D9B79F0057
:109080007FB197008FB9970008004100898049009F
:109090004431DE0002044000E0844800880F5200A2
:1090A000898F5A00F00039000800520089805A0068
:1090B0000781FB0003002000EDDD0700E00F5000FA
:1090C000E08F5800E800320013C0B300E3E79F00D0
:1090D00054FF2000840F5000E08F58000700360036
:1090E00035C0B300E5E79F00EB0F4000E08F58006C
:1090F00002003E0022C0B300E2E79F00620640008B
:10910000E08648003C0D98004D0D98001FB2970076
:10911000AFB297000400440085804C0030159800E1
:10912000411598004FB49700DFB497000400440045
:1091300085804C00700D9800011598004A01900040
:10914000EFE49700E3CF54001B003A000200E00078
:10915000C5003A007B699000C811DD0002002000C4
:109160006B6890008080FB0000002000000171000F
:10917000818171005B6890004800DD0001002000E3
:1091800000017100818171004B6890000080FB003C
:10919000010020000001710081817100121598000A
:1091A000231598004268DD00CE60DE00810070006B
:1091B0004260DD00170037000200E000AA00320024
:1091C0007FB197008FB9970000004100818049006E
:1091D0001015980021159800EFE19700E2CF51009B
:1091E00003003A000C0046008D804E000900370055
:1091F00032002000030020000C00BE008EDD0700BE
:109200008100D1000080D3006101660002004000AF
:10921000E0804800F01FB0000180B000C909DE0006
:10922000470ADD004901DE00020172005A08900081
:10923000EA089000820F5000838F58008A0039009E
:109240000080EB008080EB0070059800010D980015
:109250006000B8005005980061059800EFE29700A3
:10926000E3CF520071003A000040EB0050459800F7
:109270001B7190004811DD000B7090000080FB0016
:10928000000171001FB49700AFB4970002014400C1
:10929000E0814C00120D9800230D98001A409000B8
:1092A00014C0B3008B0078000B2007000000E00022
:1092B0005E003A007BF893004800DD00EBF8930075
:1092C0008180FB000100700051A52A00810F500031
:1092D00056003A003B419000C811DD00020020001A
:1092E0002B4090008080FB000000200000017100F6
:1092F000818171001B4090004800DD0001002000CA
:1093000000017100818171006A6890000080FB009B
:1093100001002000000171008181710020252500DD
:1093200011162400800F5100818F59003F003A0030
:109330007BE19300C811DD00020020006BE0930088
:109340008080FB000000200000017100818171001D
:109350005BE093004800DD00010020000001710087
:10936000818171004BE093000080FB000100200030
:10937000000171008181710020272700111426004F
:10938000800F5100818F590028003A007BE993003B
:10939000C811DD00020020006BE893008080FB0014
:1093A0000000200000017100818171005BE89300E2
:1093B0004800DD0001002000000171008181710082
:1093C0004BE893000080FB000100200000017100C9
:1093D0008181710052059800630598003BE9930074
:1093E000C811DD00020020002BE893008080FB0004
:1093F0000000200000017100818171001BE89300D2
:109400004800DD0001002000000171008181710031
:109410000BE893000080FB000100200000017100B8
:109420008181710072059800030D9800EFE49700A8
:10943000094D78003E1FEC00F0F9880030059800D7
:109440006000B80050159800611598000040EB00CE
:109450004045980002003700A900200003003700B3
:109460008004EB0001003700D900200060FB2F00D2
:109470000F004000B0AF9F000900E000CF003A00AD
:109480009E407800F0C2B30080CF5000050032004B
:10949000C0C5B30080CF5000020032000E04780037
:1094A000010037000E04E8006000B800C0A79F006C
:1094B000D1A79F00F1C1B30098CF100009003E0072
:1094C0008000EB0022FC2F000F004100E4FC0700AD
:1094D000800478000000EB00A0AF9F00B7003700C9
:1094E0000804E80098407800F0C2B30080CF500034
:1094F000FBFF3200C0C5B30080CF5000F8FF320040
:10950000BFAC9700B20020000102200009007800E3
:10951000C2FA07008041EB008002EB00850378006F
:1095200086002000E8C07B00014178008703E80046
:1095300000C2B30080CF5000350036006F404000BD
:1095400080CF500032003200C0C5B30080CF500041
:109550002F003200E0C2B30080CF50000200320082
:10956000868F520008003900E80F530090003A003F
:1095700080CF50008E003A00C219DD0086027800CC
:10958000B6002000E7FF37000104E00005003D00C1
:109590003340B3000180FB000008B10021592A00CC
:1095A00060C178000282FB0021612A0001003700BF
:1095B0008100E800114078000004E000040032005F
:1095C0000000FB00840F5000F9FF3A0078003700DC
:1095D000F0CBB30000404100F94F500002003E00C4
:1095E0000314A00007003700F0C9B3000040410099
:1095F000F94F500003003E000304A00000CEB3006A
:109600000041410082F27C008502E800C5FF37007E
:109610000704440042C0B30000C2B30080CF500032
:109620000600360004003700490020003E003700E5
:10963000800478003C0037000041EB000500E000AA
:109640005B00320054CEB300994F120002003A0082
:1096500050C0B300804C7800E80F530001003A007E
:10966000C219DD008380FB0063806000E10F5000C1
:1096700001003A000244A0006C806000E40F50003A
:1096800001003A000234A000B24C98008000EB00C8
:1096900025FC2F000F80420071FC07008004780039
:1096A0000000E00020003A000FA997009FA9970052
:1096B0001FA0970060FA0700800478000000E00017
:1096C00019003A00AFA897001104E000D6FF32005D
:1096D000314890000038A3000E003A0001027800E3
:1096E000BFA99700B2002000090078000201E9003C
:1096F000E10F410005003200B480FB003380FB0025
:109700000080500003003A00F8FF37000000E0003E
:10971000C7FF32008000EB0029FC2F000F804400BF
:10972000A4FC0700DDFF37003FA8970030489000F9
:109730000900E00005003200E48F54001F003A00E9
:109740000028A3001C0032001C0037000028A300E2
:109750001A003A00AFA89700314890000048A300D3
:1097600015003200515190004811DD004150900029
:109770000080FB000001710003002000C011DD002B
:1097800002002000315890004800DD00215A90006E
:109790000482FB0004007000010020000001710041
:1097A00081817100C2A79F00D3A79F004DFF3700A2
:1097B000690020000100370059002000AFAE97007B
:1097C0000900E00003003A000D00E00001003A004B
:1097D000690020004FD897008080FB007C806000EB
:1097E000A30032000900E0002E003200E48F540094
:1097F00025003A008000EB0022FC2F000F00410002
:1098000017FC0700800478000000E0001E003A000A
:1098100023FC2F000F8441000FA997009FA99700F8
:109820001800780004FA0700800478000000E000C7
:1098300015003A002FA8970010407800FB4F400019
:10984000D80032000004E000D600320011002000F1
:109850000800780057FC0700EAFF37002FAC97009C
:10986000020220000800BE00ECF90700BFA8970024
:10987000B200200008007800E1F907009A007800A3
:1098800010C0B300C04098004FDA97000434A00025
:10989000C4DF9F00AFAE97000900E000080032006F
:1098A000D90037003D489000710060007900200029
:1098B000D5003A00890020000128A300D2003A0018
:1098C000CFDA97000538A3007C0032009D2E0700F8
:1098D000E04E98004801DE00F24E98004009DE009C
:1098E00003002000825698004808DE009056980039
:1098F0008042EB00B54E9800C55E9800D55E98009A
:10990000E55E9800F55E9800F58446007484460094
:10991000FB8346007A8346001981FB004811DD0075
:109920001880FB000001710003002000C011DD0061
:10993000020020001780FB004800DD001682FB00BB
:10994000040070000100200000017100818171009D
:10995000F2AF9F0083B79F00054B7800854B7800DE
:10996000054C7800854C780028FC2F000F0144003E
:109970009200780010C0B300C04098007FA8970004
:109980008FB09700E00F5000E08F58004600320083
:10999000120678005C119000EC119000C2AF9F009D
:1099A000D3AF9F00E10F5000E08F58002E0036002B
:1099B0003C089000CC0890007FAA97008FB29700D7
:1099C000800F5200818F5A00270031000404BE002E
:1099D0000801BE000C007800F4F907000005BE0085
:1099E000E00F5000E08F580078003200E10F500087
:1099F000E08F58001C003200E10F4000E08F48006B
:109A0000800032006022B8000801BE000C0078001F
:109A10006EFA0700800478000000E0007A003A0047
:109A20007C0090008C089000E10F4000E08F48001F
:109A30000600320061004000E08048007006980097
:109A4000010E980010C0B300504698003C089000EA
:109A5000CC089000800F5500818F5D005B003100C5
:109A60000A04BE00DAFF3700290020006600370034
:109A70000900E00064003A003D4890000080FB00CF
:109A8000490020000048A3005F003A000118A3002D
:109A900003003200790020000008A3005A003A00B9
:109AA0000138A300050032008004EB00CFDA9700F4
:109AB0000554A000C5DF9F00010037008004EB00C3
:109AC0009FA2970055109000E51090006FB197008D
:109AD00050099800610998007D099800CFD9970036
:109AE000434198005D5190004811DD004D509000B9
:109AF0000080FB000001710003002000C011DD00A8
:109B0000020020003D5890004800DD002D5A9000D2
:109B10000482FB00040070000100200000017100BD
:109B2000818171006FB2970072029800030A980059
:109B30007D599000C811DD00020020006D58900092
:109B40008080FB0000002000000171008181710015
:109B50005D5890004800DD00010020000001710008
:109B6000818171004D5890000080FB0001002000B1
:109B70000001710081817100520298006302980017
:109B80006000B8003002980041029800300A980046
:109B9000410A9800050A7800B50290001502980065
:109BA0001900370025FC2F000F8542000FA99700F0
:109BB0009FA997001A0078001FF907008004780019
:109BC0000000E00030FF3A0024FF37001FA097009C
:109BD0007FAC97008FB4970061015400E0815C0076
:109BE00052009800630098004FA99700DFA99700E2
:109BF00011F90700800478000000E000ABFF32009C
:109C00000100370019002000090078004F07780094
:109C10004F06BE004F05BE004F04BE00EF03B1006B
:109C200000000600E6874700889FBE008A9FBE00AE
:109C30008C9FBE008E1F7800800478000207780099
:109C400083BF9F00F1B79F008009EB009000900058
:109C5000100078002BFC07000000E000AE003A0086
:109C6000C9409000200020000104E000AA00350057
:109C7000700020000108A300A70032000D0037008B
:109C8000494090000074A000C044980020002000CB
:109C9000A10037000174A000C14498000300370000
:109CA000494090000074A000C044980010002000BB
:109CB0009900370059009000E900900039019000A8
:109CC000C901900002015000838158006170B80002
:109CD000820F5000838F58008C00360002077800F6
:109CE0008A00370039029000C90290000400780011
:109CF000F01FB2006C003A00990078004728DD00A0
:109D00004921DE0002017000C929DE0021409000D7
:109D10000040E9008246600012003A00E00F520065
:109D2000E08F5A0003003A00790090008908900003
:109D30000400370019099000A9099000010078007B
:109D40001AF90700E10F5000E08F5800CCFF3600F1
:109D5000E10F4000E08F4800D1FF3200900C9800E6
:109D6000A10C98001906780019099000A909900023
:109D70000C007800F5F807000001BE00E00F50006D
:109D8000E08F5800BEFF32000D80FB000100200074
:109D900002054000838548004974DE00250032003A
:109DA000AC4090000D81FB00080041008180FB0069
:109DB000810F500001003600028450001C409000CA
:109DC000084278000A01BE00FFB09700421D07005C
:109DD000C94090000000E000AEFF3A000168A30017
:109DE0001200320039089000C90890000A015000A2
:109DF0008B8158006140B800800F5100818F59005D
:109E00000A0031000102200089804000491ADD006B
:109E1000C711DE00830172004911DD007FB2970097
:109E2000020042000220200075F807004944DD00CE
:109E30002A00370039099000C90990008A0F5100A3
:109E40008B8F590016003200494090000068A30033
:109E50000A00320001022000898040001C4090006E
:109E600014C0B300581D0700C94090000000E00076
:109E700088FF3A000164A100C1449800010220005B
:109E800089804000190078001040900014C0B30091
:109E90000A01BE00101D07000000E00080FF3A002C
:109EA000BA0C9800CB0C9800B9019000F31FB200D7
:109EB00000202000030450008E0F540001003600E3
:109EC0000E04780001022000898040008380400059
:109ED000080178007FB0970049F807007FB097002D
:109EE00008004000F0B79F0039009000C9009000C2
:109EF00008004000E0804800B0049800C1049800C9
:109F00000FBA9700140A4400080757000E00E0003B
:109F100074FF3A000E0078004F0778004F06BE002D
:109F20004F05BE004F04BE006F00B10000000600E8
:109F3000E6874700889FBE008A9FBE008C9FBE00B8
:109F40008E1F7800000478008206780083BF9F008F
:109F5000F1B79F008009EB0090009000100078009E
:109F600068FB07000000E000CE003A00C840900007
:109F7000200020000104E000CA003500700020002D
:109F80000118A300C70032000D0037000174A000C3
:109F90004144980008003700484090000074A00039
:109FA0004044980020002000BE0037004840900048
:109FB0000074A0004044980010002000B900370051
:109FC00058019000E80190000D004100E080490038
:109FD000820F5000838F5800A5003900A20037007F
:109FE00038029000C802900004007800F01FB20010
:109FF00081003A00980078004728DD004921DE0002
:10A0000002017000C929DE00214090000040E900F3
:10A01000024760001E003A00E00F5200E08F5A0035
:10A020000B003A007801900088099000E00F510081
:10A03000E08F59000E003A000100780095F9070002
:10A040000001BE0070049800010C98000500370064
:10A0500018099000A8099000010078008DF9070008
:10A060000001BE00E00F5100E08F59008000320077
:10A07000E10F5100E08F5900C7FF3200E10F4100AE
:10A08000E08F4900C9FF3200120C9800230C9800A1
:10A09000484090000068A3000D003200380990008D
:10A0A000C8099000180078001040900014C0B30058
:10A0B0000102200088804000C31C0700C8409000B7
:10A0C0000000E000B1FF3A000164A10041449800A3
:10A0D0001806780018099000A80990000C00780074
:10A0E0001AF807000001BE00E00F5000E08F580092
:10A0F000A9FF32000E80FB00010020000205400095
:10A1000083854800C96CDE0025003200AC40900019
:10A110000E81FB00090041008180FB00810F50008F
:10A1200001003600828450001C40900009427800F3
:10A130000A01BE00FFB09700A31C07000000E0006A
:10A140009AFF3A0038089000C80890000A015000B1
:10A150008B8158006148B800800F5100818F5900F1
:10A160000D0031004918DD00C710DE0081007000CD
:10A170004910DD007FB197008000410002202000DF
:10A1800000022000080040009DF7070048409000B2
:10A190000064A10040449800C94CDD00260037004F
:10A1A00038089000C80890008A0F50008B8F580024
:10A1B0000F00320038019000C80190005800900054
:10A1C000E8009000800F5100818F59000800310095
:10A1D0001C40900014C0B3000A01BE000102200020
:10A1E000888040003C1C07000000E0006FFF3A0040
:10A1F0003A0C98004B0C9800B8019000F31FB20085
:10A2000000202000830450008D8F54000100360090
:10A210008D04780000022000080040000300400088
:10A2200009017800FFB0970075F7070048409000DB
:10A230000064A000404498007FB0970009004000EF
:10A24000F0B79F0038009000C8009000090040005F
:10A25000E080480030049800410498000FB997004E
:10A2600012894400898656000D00E0005CFF3A0028
:10A2700038019000C801900058009000E80090005C
:10A28000800F5100818F590002003600520498005F
:10A2900063049800484090000054A0004044980097
:10A2A0000000EB004F0778004F06BE004F05BE00D0
:10A2B0004F04BE006F00B10000000600889FBE0082
:10A2C0008A9FBE0080047800900090001000780003
:10A2D0008CFA0700000578000000E00082003A00D8
:10A2E000494090000080FB000058A3007D00320030
:10A2F0000068A3000D00320039099000C9099000E0
:10A300000102200089804000190078001040900070
:10A3100014C0B3002C1C07000000E0006F003A00DE
:10A32000494090000064A100C04498005909900081
:10A33000E9099000190078003FF707000005780050
:10A340000000E00068003A00790C90006B004400C7
:10A350001054A00029489000405C980039489000B3
:10A36000505C980049489000605C98005948900003
:10A37000705C980069489000205C980079489000D3
:10A38000305C98000950900040549800195090009B
:10A3900050549800EB2B0700605498004801DE00F1
:10A3A000725498004009DE0003002000025C98000F
:10A3B0004808DE00105C9800494090000054A1005D
:10A3C000C0449800190078001BC0B3004B409800AF
:10A3D000990478006011B8000900780016F70700AA
:10A3E000000578000000E0003F003A0030C0B300F4
:10A3F000994F100033003A00594090000004E000EB
:10A40000300032006000B800D0149800E1149800C9
:10A41000E802200009044400022020008A0078009D
:10A4200008007800FDF6070050C5B30060FC9B00F3
:10A43000A0CAB30070FC9B0020C5B300004C78009C
:10A44000F06C980012C6B3008274980011C4B30077
:10A450009174980020C7B30040E49B0050E49B0037
:10A4600061E49B0072E49B006948900000EC9B0053
:10A470007948900010EC9B000950900020EC9B0064
:10A480001950900030EC9B002948900040EC9B0054
:10A490003948900050EC9B004948900060EC9B00CC
:10A4A0005948900070EC9B0019099000A909900090
:10A4B000194090000B42780088007800C21B07000A
:10A4C000DA449800194090000001EB008040EB0056
:10A4D0000B1C07000000E000020032001A00200000
:10A4E000010037000005EB000A0078004F05BE00B0
:10A4F0004F04BE0000000600881F780000047800AA
:10A500006EFF07000000E00001003A00000C780038
:10A510004F047800000006000800FA00889FBE0083
:10A520008A9FBE008C9FBE000005780082BF9F00FE
:10A5300093BF9F009000900010007800F1F9070091
:10A54000000178000000E000EC003A004A40900072
:10A55000220020000004E000E80035005A019000CD
:10A56000EA0190000FBA97009FBA9700820F52003D
:10A57000838F5A00040036000018A30002003A003E
:10A5800082BF9F0093BF9F003A019000CA019000D4
:10A590006000B80030059800410598000FB897009A
:10A5A0009FB89700E00F5000E08F58009A003200EB
:10A5B0009A0578002B4090000080FB0001002000ED
:10A5C000490ADD00C702DE00850272004902DD0093
:10A5D000E4B79F00F5B79F00E00F5100E08F5900EE
:10A5E0002400320061065100E08659000FB997003F
:10A5F0009FB9970061005100E08059000401BE003E
:10A600009BD807000004BE006FB19700FFB1970010
:10A610000C00BE0096D80700800F5400818F5C00AC
:10A62000140039006FB29700FFB29700600012006B
:10A63000E0801A000C0160000D806000800278004C
:10A64000020278000400BE00300598004105980021
:10A650000FB997009FB997000001510081815900FF
:10A6600082BF9F0093BF9F001A099000AA09900023
:10A67000120037007A0190008A099000E00F510023
:10A68000E08F59000B003A000B00780001F807003A
:10A690000001BE00E10F5000E08F58005000320072
:10A6A000E10F4000E08F48008900320070059800FB
:10A6B000010D9800120D9800230D9800E00F510035
:10A6C000E08F59002E003A00530037004A409000B6
:10A6D0000018A3000B0032001A007800EDF7070005
:10A6E0000001BE00E00F5000E08F580008003A0063
:10A6F0006FB29700FFB2970084BF9F0095BF9F0085
:10A70000260037001A007800A8F607000001BE00F6
:10A71000E10F4100E08F49006D003200E10F510070
:10A72000E08F59002E0036001A007800C008900013
:10A7300030089000800F5100818F590028003100AF
:10A74000120D9800230D98003A009000CA00900066
:10A750006FB29700FFB29700040040008580480068
:10A7600030059800410598000FB897009FB89700F2
:10A77000040050008580580080BF9F0091BF9F005B
:10A780000FBA97009FBA97006FB09700FFB097007D
:10A79000800F5200818F5A00CCFF3E003A0090009B
:10A7A000CA0090000FBA97009FBA970004004000BB
:10A7B0008580480030059800410598000FB8970043
:10A7C000F01FB200140032001A0078005FF6070094
:10A7D0000001BE00E00F5000E08F580005003A0075
:10A7E0004A4090000074A0004045980022002000DC
:10A7F000420037000FBA97009FBA9700472BDD0041
:10A800004920DE0000007300C928DE000206400077
:10A8100083864800010037006066B8003A00900067
:10A82000F01FB200210032003A099000CA099000DE
:10A83000820F5600838F5E001C0032004A40900059
:10A840000068A3000E003200010220008A80400050
:10A850001A0078001040900014C0B300DA1A070004
:10A86000CA4090000000E000030032000174A00024
:10A8700041459800190037000164A1004145980046
:10A88000010220008A8040001A00780010409000E9
:10A8900014C0B3000C01BE008F1A07000000E000D6
:10A8A0000B003A003C0D98004D0D98003A029000C4
:10A8B000CA0290005A009000EA0090000001EB00EC
:10A8C000800F5200818F5A000C00360005003700BF
:10A8D0004A4090000074A0004045980012002000FB
:10A8E0000600370054059800650598004A4090001E
:10A8F0000054A000404598000001EB0002007800E1
:10A900004F06BE004F05BE004F04BE000080FA0097
:10A9100000000600889FBE008A1F780000057800AE
:10A920008104780002047800E427070008417800D9
:10A93000894078000A407800EE2707000841780037
:10A94000894078000A407800F82707004F05780012
:10A950004F04BE0000000600E40F50001F0032004C
:10A9600009003E00E10F5000110032000041EB00F1
:10A970001B003900E20F500010003200E30F5000BE
:10A9800025003A0011003700E60F50001600320093
:10A9900002C2B3008040EB000A003900E70F50000C
:10A9A00015003200E80F50001B003A001600370077
:10A9B0000041EB0001C2B300110037000041EB0081
:10A9C00001C2B300014078000E0037000041EB00E7
:10A9D0008240780000C2B3000A00370002C2B30010
:10A9E00082407800F7FF370002C2B300824078004F
:10A9F0000040EB000300370002C2B3008040EB00D0
:10AA000002407800AD27370052C0B300F1C0B30058
:10AA100000C2B300A927070000000600881F7800C5
:10AA2000000478000001EB006000B800B9FF0700E7
:10AA30008043EB00074378008742780007427800A4
:10AA40008741780007417800874078000740780008
:10AA5000722707008040EB0000C1B300C326070047
:10AA60008040EB0010C1B300C02607008040EB001F
:10AA700040C1B300BD2607008040EB0050C1B300C9
:10AA8000BA2607008040EB0020C1B300B7260700BC
:10AA90008040EB0030C1B300B42607008040EB00DB
:10AAA00060C1B300B12607008040EB0070C1B30065
:10AAB000AE2607008040EB0001407800AB2607007F
:10AAC0008040EB0010C0B300A8260700E40F54003C
:10AAD0001400320006003E00E20F54000E00320067
:10AAE0000B003E00E10F540022003A000A0037003C
:10AAF000E60F54001B0032000C003900E70F540031
:10AB000018003200E80F54001A003A00170037000E
:10AB10000010200081180700400020007F18070067
:10AB20000D003700080078001100370040002000B9
:10AB30007A18070000012000781807008040EB0019
:10AB4000E0C1B300892607007832EF00C1AC2100D4
:10AB5000F0DF2F00910860005A32EF005C32EF0006
:10AB6000040037005A32EF005C32EF004000200052
:10AB70006A1807004F04780000000600001020004B
:10AB80005A18070000202000581807000001200074
:10AB9000561807004000200054180700100020003D
:10ABA000521807000001200050183700881F780055
:10ABB0000004780068FF0700E40F54002200320010
:10ABC00006003E00E20F54002A00320015003E004D
:10ABD000E10F540029003A0008003700E60F540046
:10ABE000240032001A003900E70F54001F00320021
:10ABF000E80F540021003A001E0037008043EB00AC
:10AC00000743780005C2B30005427800854178000B
:10AC1000074178008740780007407800FF2607004A
:10AC200014003700001020003018070040002000FA
:10AC30002E1807000041EB0082407800F0C0B300FE
:10AC40001E2707000D003700080078000A003700B3
:10AC500040002000251807000001200023180700ED
:10AC6000A00F2000C093880004003700F62FEF00EB
:10AC7000F42FEF00400020001C1807004F0478005C
:10AC80000000060000417800FF4F500002003E0027
:10AC90008000FB00070037008000EB00F0C3B3002A
:10ACA000804F510003003E000040E8000240500089
:10ACB0008000FB000100780000000600C27F8000D9
:10ACC000010040000100370069005000E80F50000B
:10ACD000FDFF3C0001003700690040000000E0007B
:10ACE000FDFF3500E40F5000F5FF3200E80F500083
:10ACF000F3FF32000000E00002003A000200E00032
:10AD0000EFFF320000000600EC874700889FBE007E
:10AD10008A9FBE008C9FBE008E1F7800F14FEC0012
:10AD200080407800F1EFB70040C6B30080CF5000FC
:10AD30001C0036000040E800F1EFB700B1CFBF00C3
:10AD40000400320010C0B300110020009E5EE2003B
:10AD5000010032008000EB009EFEB7000104E0001D
:10AD600010003200D07F80002CFF0700917F800010
:10AD70000100E00012003200D07F8000808F500080
:10AD800004003A000000EB0088FF0700FA2FEF00F4
:10AD9000040037000100780084FF0700917F8000E5
:10ADA000D17F880042380700D17F80008001780081
:10ADB0000000E000060032000100780017FF0700E5
:10ADC00000402000D51707006CFF07002C05370056
:10ADD000E38F5000B001320004003E00E18F5000CC
:10ADE00044003200E5003E0007003700E68F5000C7
:10ADF000B9033200E78F500067043200E58F50003E
:10AE00001F053A00B7023700AFCFBF000400320081
:10AE100010C0B300110020009D5EE200010032006E
:10AE20008000EB009DFEB7000104E000040032004A
:10AE3000907F80008080EB00A0FF0700907F88005B
:10AE4000B0CFBF000400320010C0B30011002000DA
:10AE50009C5EE200010032008000EB009CFEB70027
:10AE60000104E00004003200907F80008080EB004D
:10AE700092FF0700907F8800B2CFBF00040032002D
:10AE800010C0B300110020009B5EE2000100320000
:10AE90008000EB009BFEB7000104E00004003200DC
:10AEA000907F80001100200084FF0700907F8800C1
:10AEB000B3CFBF000400320010C0B3001100200067
:10AEC0009A5EE200010032008000EB009AFEB700BB
:10AED0000104E00004003200907F80001100200097
:10AEE00076FF0700907F8800907F80009AFE070021
:10AEF000E30437000892800001007800222421003A
:10AF000092007800888F500002003400010478001D
:10AF1000800178000000E8000281E800E50F5000A1
:10AF2000F7FF3A0005F8800062801100240020003D
:10AF300000017800110009008402D8000001FD0022
:10AF40000280B90000057800C0DA20008000EB0024
:10AF5000800F540004003400080050001100090064
:10AF60000400D8008000FD0000FA2000800F54008B
:10AF7000020034008500EA000D00370070BB20009D
:10AF8000800F540007003C0080C12F0000004400E7
:10AF900072002000110009000200D800C112200038
:10AFA00080805000F07C2000800F540002003400AC
:10AFB000858F500001003400850078008504EA0088
:10AFC000898F50000100350081047800301F200077
:10AFD000800F540003003C005A32EF005C32EF0057
:10AFE0000400370009004500E09288000A80540000
:10AFF000D0928800F04FEC008000FB00F0EFB7002B
:10B000000004E000090034000001EB000000EB0048
:10B0100040FE070080C2B300F04FE3000B00340095
:10B0200000C8B300F0EFB700080037008100EA0065
:10B0300042002000110009008200D8008000FD00BD
:10B040000001EB000000EB0032FE0700B2CFBF00B2
:10B050000400320010C0B30011002000995EE2002D
:10B06000010032008000EB0099FEB7000104E0000F
:10B070000700320000F880002003B00000F88800CC
:10B08000411F2000810F50000100340001F88800AA
:10B09000AFCFBF000400320010C0B3001100200089
:10B0A000985EE200010032008000EB0098FEB700DD
:10B0B0000104E00007003200E0FC2F00001FB40094
:10B0C00000F8880041ED2F00810F500001003D0085
:10B0D00001F888008040EB00401F2000800F5400E2
:10B0E0000400340011C0B30010002000975EE2009D
:10B0F000010032000000EB008000FD0097FEB70069
:10B100008000FD000004E00002003200600020002A
:10B110007A3007000A00E0000C003A000900E00065
:10B1200053043A00EF4FE20051043A00401F200060
:10B13000800F54004E04340010C0B300EFEFB7008E
:10B14000700020006D300700C8003700EF6FEF007F
:10B15000C6003700C0928000810F5000C700340045
:10B160008040EB0080C0B300002507008040EB006A
:10B17000B0C0B300FD2407004104370078815700B8
:10B1800084752A0007000900345978008200B10054
:10B19000ED4FEC0080407800EDEFB7004240A90091
:10B1A0000800340003417800C425070080C2B300C2
:10B1B000ED4FE3000B00340000CCB300EDEFB7001F
:10B1C000080037000000FB000000EA002200200019
:10B1D000110009000200D800034178008040780087
:10B1E000B6250700EECFEC0080417800EEEFB70007
:10B1F0000080FB004500DE0002C2B300F8005000F2
:10B2000082F07F008000E900E7806000FFC16100FC
:10B2100003415100F880500082F07F000000E800F8
:10B22000670060007800500003F07F00FFEB97009C
:10B230002FE997009FE897006FEB9700DFEA9700F0
:10B240004FEA9700BFE997000FE8970073250700C2
:10B25000B2CFBF000400320010C0B30011002000C4
:10B26000965EE200010032008000EB0096FEB7001F
:10B270000104E00007003200F0F780002003B00076
:10B28000F0F78800411F2000810F500001003400BA
:10B29000F1F78800AFCFBF000400320010C0B30048
:10B2A00011002000955EE200010032008000EB00FA
:10B2B00095FEB7000104E00007003200E0FC2F001B
:10B2C000FE1EB400F0F7880041ED2F00810F500002
:10B2D00001003D00F1F78800FEF780000E00E0005D
:10B2E0005100350008928000149280006145B90039
:10B2F00004004200CF80DE000A0540008B85480034
:10B30000209280006300B900CF80DE000A05400073
:10B310008B8548003292800002004100CF80DE0021
:10B320000A0540008B854800469280006130B900D4
:10B330000A0540008B854800C0FF2F0000C4B900FB
:10B34000CFC4DE00D0FF2F0000A2B900CFA2DE00E4
:10B350000804420089844A006311B900CF91DE00DD
:10B3600008044100898449004233DD00CFB3DE0088
:10B370000804430089844B000A0044008B804C0081
:10B380006176B9000C01BE002BD50700027D2000BC
:10B39000811F7800110009004208D800CF00780012
:10B3A0000000570080BF9F00D0928800080555001C
:10B3B00089855D000C01BE000A00BE001ED5070095
:10B3C000047D2000811F7800110009004408D80086
:10B3D000CF00780000005700E092880081DA2F004B
:10B3E0000FB89700810F500001003D00D1928800F6
:10B3F000E0928000810F500001003D00E192880042
:10B4000081252000D0928000810F5000010034007F
:10B41000D1928800E0928000810F50001300340028
:10B42000E192880011003700609280000E80B90020
:10B4300042ED2F00811F7800110009004208D8005A
:10B44000CF00780000004700D09288005092800022
:10B450000E80B900811F7800110009004208D80051
:10B46000CF00780000004700E0928800110820001B
:10B47000B0928000810F500036FF3C005A32EF003E
:10B480005C32EF0001C2B30080C0B3003724070074
:10B4900001C2B30036FF3700E0F7800080004000B3
:10B4A00080804000509380000000E00001003D00DB
:10B4B0000000EA0080804000609380000000E0000F
:10B4C00001003D000000EA00808040007093800091
:10B4D0000000E00001003D000000EA0000804000A4
:10B4E0004200DE00E0F7880083007800ED0F500096
:10B4F00001003E00110020008104780083407800A4
:10B50000EE0F50000400360011C0B30013002000FD
:10B51000945EE200010032008001EB00010078003F
:10B5200094FEB7000304E000040032000041EB0089
:10B5300082407800F0C0B300E0240700E0F780000C
:10B54000ED0F50000F003E00EA0FEC00507F880026
:10B55000E50F500007003400EA0F500001003A00E8
:10B56000EA2FEF000041EB008240780000C2B300F8
:10B57000190037000041EB0082407800024078005B
:10B5800015003700EC4FEC008001FB00ECEFB7003A
:10B590000004E0000A0034000001EB008000EB0032
:10B5A00003007800DBFC070080C2B300EC4FE3002F
:10B5B0000A00340000CCB300ECEFB70007003700FE
:10B5C0000300EA0022002000110009000200D80058
:10B5D0000041EB0082407800B82407008012E200AE
:10B5E000030032008032EF0050002000432F07009C
:10B5F00017928000813E2000818F53001700340095
:10B6000020928000810F500014003400309280009E
:10B61000810F50001100340050928000810F5000C3
:10B6200003003C0060928000810F50000B0034004A
:10B6300021082000B0928000810F500007003400E4
:10B64000C0928000810F5000040034005A32EF0095
:10B650005C32EF001900200058003700089280008B
:10B66000823E2000820F54000B003C00828F53006A
:10B6700009003C0020928000820F500006003C0030
:10B6800030928000820F500003003C004092800006
:10B69000820F5000380034005400200011000900CF
:10B6A0000404D800000378004200200011000900C3
:10B6B0008203D8000003430020928000110009009B
:10B6C0000200D800000343003092800045928000C1
:10B6D000801F7800110009000200D80000017800E6
:10B6E0004F007800801F7800110009008402D80004
:10B6F000800078004F007800010141000203430000
:10B7000062002000801F7800110009000204D800A8
:10B71000800078004F00780080017800811F780059
:10B72000110009008403D8008001FD00CF007800DB
:10B7300083804000811F7800110009000400D800B8
:10B74000CF007800809FBE00110009008202D8005F
:10B75000800278004F00BE0005004000808050004D
:10B76000010043000000EA00D0928800868050006B
:10B77000E19288001100370051928000828F5000C2
:10B7800003003C0060928000820F500009003400EA
:10B7900042002000110009008200D800D0928800E9
:10B7A00060928000110009000200D800E092880039
:10B7B000020037005A32EF005C32EF00110820001F
:10B7C000B0928000810F500003003400C0928000CE
:10B7D000810F50000A003C005A32EF005C32EF004B
:10B7E0000041EB008240780000C2B3004124070012
:10B7F0000041EB008240780000C2B3000700370030
:10B800000041EB00824078000240780039240700B4
:10B810000041EB008240780002407800432407009A
:10B8200081DA2F00D0928000810F500001003D008E
:10B83000D1928800E0928000810F500001003D000D
:10B84000E192880081252000D0928000810F500075
:10B8500001003400D1928800E0928000810F5000F6
:10B8600001003400E19288008040EB000900E00014
:10B870000400320011C0B30010002000935EE2000B
:10B88000010032000000EB008000FD0093FEB700D5
:10B890008000FD000004E0000200320040002000B3
:10B8A000982E07008040EB000900E00004003A00F9
:10B8B00011C0B30010002000925EE20001003200CF
:10B8C0000000EB008000FD0092FEB7008000FD004C
:10B8D0000004E0006A0232000080EB00872E0700BF
:10B8E00067023700CD3AAB0041003200C1AC210005
:10B8F000F0DF2F009108600077FE2000974378006A
:10B900000704E0000C003A0007007800E8EFB700F9
:10B9100010C0B300E7EFB700074378008742780014
:10B920000742780087417800074178008740780017
:10B930007F40400014003700E1CF530014003A006C
:10B9400081FE200091407800E2CF500028003400B2
:10B95000FDCF500026003C0020C0B300E7EFB70049
:10B960000140E800E3EFB700FFC343000043EB00F2
:10B9700086427800064278008641780006417800C9
:10B980008740780007407800A4230700180037009C
:10B99000E2CF530016003A0081FE2000914078006B
:10B9A00001407800E34FE30011003D0070C2B30096
:10B9B00080CF50000E003C0030C0B300E7EFB7006E
:10B9C000FEC34300074378008042EB000542780045
:10B9D000854178000741780087407800074078006B
:10B9E0008E23070070002000442E0700E96FEF004F
:10B9F00081FE20009140780030C6B30080CF500017
:10BA000002003C000140E800E8EFB70020C3B300AB
:10BA1000E84FE3000A003400E76FEF008043EB00DB
:10BA20000743780087427800074278008741780012
:10BA300007417800874078000740780077230700A7
:10BA400081FE200091407800E5CF500019003A00B7
:10BA5000E4CFBF00E14F50000A003A0070FE200022
:10BA600011C0B30090CF100032003A0020C0B300E4
:10BA7000E4EFB70000052000D092880000FB2F0003
:10BA80000A003700E24F50002A003A0070FE200002
:10BA900012C0B300904F110026003A000240780017
:10BAA000E4EFB70000052000D0928800E092880003
:10BAB00020003700FECF50000F003A0070FE20003B
:10BAC000E44FE20005003A0024C0B300904F12009A
:10BAD00018003A0010C0B300F1FF370021C0B300D6
:10BAE00090CF100013003A00E46FEF005A32EF00DD
:10BAF0005C32EF000F00370080C2B30080CF5000EF
:10BB00000C003A0070FE200032C0B300904F1100CC
:10BB100008003A0011C0B30001007800E4EFB7005C
:10BB200000052000D09288005C32EF000100780010
:10BB3000E6EFB70011082000B0928000810F50009E
:10BB400003003400C0928000810F50000A003C00C6
:10BB50005A32EF005C32EF000041EB008240780087
:10BB600000C2B300632307000041EB00824078006D
:10BB700000C2B300070037000041EB0082407800AC
:10BB8000024078005B2307000041EB008240780010
:10BB90000240780065230700E64FE20036003200DD
:10BBA000E54FEC00E5EFB70001C6B300814F500050
:10BBB00001003400E56FEF00E5CFBF0004C2B30021
:10BBC0008444400081CF54000100360081C45400F9
:10BBD00002C4B30002444000814F5400010036000B
:10BBE0000144540027FC0700004578000940780014
:10BBF00024FC0700804478000840780021FC0700FE
:10BC00000044780000417800894078000A407800BC
:10BC10002A230700094178008A407800084078000C
:10BC2000422307000A4178008840780009407800E4
:10BC300030230700E94FEC0080407800E9EFB700BF
:10BC4000F0C7B30080CF50008D013A00E66FEF00DF
:10BC5000E96FEF000041EB0082407800024078007D
:10BC6000322307000041EB00824078000240780058
:10BC70002023070082013700E94FEC0000417800E3
:10BC8000E9EFB7004240A900090034008040EB0012
:10BC9000014078000923070080C2B300E94FE300A8
:10BCA0007701340000C8B300E9EFB7007401370032
:10BCB0000001FB000201EA0043002000110009001E
:10BCC0000301D800000178008040EB0001407800BB
:10BCD000FA2207006A013700E24FEC0000417800C9
:10BCE000E2EFB7004240A90009003400804078002C
:10BCF00003407800F122070080C2B300E24FE30066
:10BD00000C00340000CCB300E2EFB70009003700AC
:10BD10008000FB008100EA002200200011000900E1
:10BD20008200D8008000FD000141780003407800C7
:10BD3000E2220700AF4FE20009003200B24FE200FA
:10BD400007003200C09280005612B400220020008A
:10BD5000110009000200D8006009B000D0F7880087
:10BD6000B04FE2000F003200B34FE2000D0032008E
:10BD7000C09280005612B400220020001100090079
:10BD80000200D800C0F7880051092000810F500040
:10BD900002003E00800C2000C0F78800A0F62F00B3
:10BDA000F83EB400B0928000D2F78000820F5000BD
:10BDB00001003100E06FEF00C1F78000810F5000FB
:10BDC0000200360010C0B300E0EFB700C092800060
:10BDD000820F500001003100E16FEF00810F500031
:10BDE0000200360010C0B300E1EFB70001FE2000F2
:10BDF000914078000104E00002003200E1CF5000E1
:10BE000005003A00E14FE20003003A00010078002B
:10BE1000DFEFB7001300370010FE200012C0B300A0
:10BE2000904F110004003A000104E00002003A00C3
:10BE3000DFEFEF000B003700DFCFBF004240A9006B
:10BE40000200340020C0B300050037000004E00009
:10BE500002003D00E0CFB30001003700A0C0B300F6
:10BE6000DFEFB700F7FD2000974378000704E000FC
:10BE70000B003A00C0122000D0928800E0928800A7
:10BE8000074378008742780004C2B30087417800F6
:10BE9000074178008740780004407800360037007A
:10BEA000E1CF53000B003A00C0122000D09288006E
:10BEB0005C32EF008043EB00074378008742780054
:10BEC0000742780003C2B30007417800834078003E
:10BED00028003700E1CF43000A003A005A32EF0051
:10BEE000C0122000E092880007C2B3000043EB00BC
:10BEF0008742780006427800864178000641780043
:10BF00001B003700E2CF43000D003A0040ED2F0048
:10BF1000D0928800C0122000E09288008043EB009D
:10BF200006C2B30087427800074278008741780054
:10BF30000741780087407800074078000E003700FE
:10BF4000E2CF53000E003A00C0122000D0928800C9
:10BF500040ED2F00E09288008043EB00074378001B
:10BF600087427800074278008741780002C2B30018
:10BF7000864078000640780028220700C00037007D
:10BF8000EACF5300BE003A00C0122000D0928800D1
:10BF900040ED2F00B4003700DE4FEC000041780088
:10BFA000DEEFB7004240A90008003400834078006B
:10BFB0004222070080C2B300DE4FE3000B003400D2
:10BFC00000CCB300DEEFB700080037000000FB0034
:10BFD0000000EA0022002000110009000200D80041
:10BFE00000417800834078003422070005FB2000E0
:10BFF00095427800054078000504E0000400320016
:10C0000010C0B30011002000915EE2000100320078
:10C010008000EB0091FEB7000104E0000200320056
:10C0200080F32F00A07F880034FB200014427800AA
:10C03000044078000404E0000400320010C0B300A3
:10C0400011002000905EE200010032008000EB0051
:10C0500090FEB7000104E00002003200800C2000D6
:10C06000A07F8800F3FA2000934178000340780015
:10C070000304E0000400320010C0B30011002000EF
:10C080008F5EE200010032008000EB008FFEB700FF
:10C090000104E00006003200F40FE200020032006A
:10C0A000F42FEF000200370080F32F00F62FB400CA
:10C0B00021FB200091407800014078000104E0005D
:10C0C0000400320010C0B300120020008E5EE200B7
:10C0D000010032000001EB008EFEB7000204E00018
:10C0E00006003200F40FE20002003200F42FEF00ED
:10C0F00002003700800C2000F62FB4000304E0009B
:10C1000003003200100020000104E00001003A00AA
:10C110000000EB00804078000004E00003003200E3
:10C12000100020008D5EE200010032000000EB00F4
:10C130008000FD008DFEB7008000FD000004E000DF
:10C1400001003200F62FEF000404E000030032008B
:10C15000100020000504E00001003A000000EB00A0
:10C16000804078000004E00003003200100020004E
:10C170008C5EE200010032000000EB008000FD0058
:10C180008CFEB7008000FD000004E00001003200DA
:10C19000F42FEF00A09380000000E0001B003200AD
:10C1A000E40F50000D00320003003C00E20F50008D
:10C1B00015003A0005003700E60F5000100032006D
:10C1C000E80F500010003A0006003700800C2000F5
:10C1D000F40FE200080032000500370080F32F0062
:10C1E0000800370080F32F00F40FE2000200320055
:10C1F000F42FEF0004003700F62FB40002003700E0
:10C20000800C2000A07F88007432EF00822520007F
:10C21000B07F8000820F500001003400B27F8800A0
:10C2200081DA2F00B07F8000810F500001003D00B7
:10C23000B17F8800A07F8000820F50000100340091
:10C24000A27F8800A07F8000810F500001003D0088
:10C25000A17F8800B07F8000A27F80008200400024
:10C26000D192880002005000E0928800040037005C
:10C27000301F2000800F5400B4FB34007BFC3700DB
:10C280004F0778004F06BE004F05BE004F04BE00AA
:10C29000CF00B10000000600C07F88000000EB0066
:10C2A00042FA0700F80FE20002003200F22FEF001E
:10C2B0000300370010002000907F8800A6F90700D7
:10C2C000B04620008912370000402000911207007C
:10C2D0008080EB000000E00001003200D17F800090
:10C2E0000100780000000600E80F50000200340052
:10C2F0000000400071005000000006008000EB00CC
:10C30000E80F500001003400110020000100780007
:10C31000000006000200FA00F0BF9F00E30F50008B
:10C320001700320006003C00E10F50000E00320002
:10C3300010003C000000E00008003200160037004A
:10C34000E90F50000B003200EA0F50000F003200DE
:10C35000E40F500010003A000C0037009460A90070
:10C360008460A9001100370094E0A90084E0A900CE
:10C370000E0037009500A9008500A9000B003700CA
:10C380009760A9008760A900080037009780A9007E
:10C390008780A900050037008F81E9004210200046
:10C3A000913F2000A06B2A00AE3407000080FA0005
:10C3B000000006000400FA00E0BF9F00F1BF9F00EC
:10C3C000E18F5000040036008F81E90062102000E8
:10C3D000912220003E0037006FB89700E30F500015
:10C3E0002800320006003C00E10F5000140032002B
:10C3F0001B003C000000E000080032003100370064
:10C40000E90F50000D003200EA0F50001C0032000E
:10C41000E40F50002B003A0022003700E1C060001A
:10C4200081C0400004C1BF000014A10001407000A1
:10C4300004E1B70005A1A9002700370013A1A90056
:10C44000E1C0600081C0400010C1BF000014A10025
:10C450000140700010E1B70011A1A9001E003700D3
:10C46000E1C0600081C0400012C1BF000014A10003
:10C470000140700012E1B70013A1A90016003700B7
:10C4800021A1A900E1C0600081C040001EC1BF0021
:10C490000014A100014070001EE1B7001FA1A90017
:10C4A0000D003700E1C0600081C0400020C1BF0026
:10C4B0000014A1000140700020E1B70021A1A900F3
:10C4C00005003700E48157004210200011262000AB
:10C4D000A06B2A00633407000080FA000000060009
:10C4E0000200FA00F0BF9F00E30F5000230032006B
:10C4F00006003C00E10F50001200320018003C0022
:10C500000000E000080032002A003700E90F500068
:10C510000C003200EA0F500018003200E40F500007
:10C5200024003A001C003700E1C06000C608DD00AE
:10C5300004C1BF000064A1000140700004E1B70025
:10C5400021003700E1C06000C608DD0010C1BF0057
:10C550000064A1000140700010E1B7001A0037002C
:10C56000E1C06000C608DD0012C1BF000064A10088
:10C570000140700012E1B70013003700E1C0600015
:10C58000C608DD001EC1BF000064A10001407000AC
:10C590001EE1B7000C003700E1C06000C608DD00F6
:10C5A00020C1BF000064A1000140700020E1B7007D
:10C5B000050037008F81E90042102000412920004A
:10C5C000A06B2A00273407000080FA000000060054
:10C5D0000200FA00F0BF9F0001417800EA0F50000E
:10C5E0001A003E0010002000FFB897008100DD0017
:10C5F000010078006020B20006003A00804120006F
:10C60000008060000A003A000108A30014003A000C
:10C610000E003700E1406100C308DD0010C1BF001B
:10C620000034A1000140700010E1B7000C00370099
:10C63000E1406100C308DD001EC1BF000034A1005D
:10C64000014070001EE1B700050037008F81E9004E
:10C6500042102000A1462000A06B2A0001340700F0
:10C660000080FA00000006000200FA00F0BF9F0000
:10C67000E30F50002C00320006003C00E10F500098
:10C68000150032001E003C000000E00008003200EF
:10C6900039003700E90F50000F003200EA0F500058
:10C6A00021003200E40F500033003A002800370028
:10C6B00063C060004400DD0041102000914078001C
:10C6C000F2CCB30082C0600080C07000010078002E
:10C6D00004E1B7002D00370063C060004400DD00B6
:10C6E0000111200091407800F2CCB30082C06000BC
:10C6F00080C070000100780010E1B700230037000F
:10C7000063C060004400DD002111200091407800EA
:10C71000F2CCB30082C0600080C0700001007800DD
:10C7200012E1B7001900370063C060004400DD006B
:10C73000E111200091407800F2CCB30082C060008B
:10C7400080C07000010078001EE1B7000F003700C4
:10C7500063C060004400DD000112200091407800B9
:10C76000F2CCB30082C0600080C07000010078008D
:10C7700020E1B700050037008F81E900421020005A
:10C78000214A2000A06B2A00B63307000080FA007F
:10C79000000006000200FA00F0BF9F00E30F500007
:10C7A0001600320006003C00E10F50000E0032007F
:10C7B0000F003C000000E0000800320013003700CA
:10C7C000E90F500007003200EA0F50000A00320063
:10C7D000E40F50000D003A000A00370002088800FC
:10C7E0000F00370043088800320888000C0037002B
:10C7F000520888000A003700B3088800A2088800A1
:10C8000007003700C2088800050037008F81E90063
:10C8100042102000D11E2000A06B2A009133070097
:10C820000080FA00000006000200FA00F0BF9F003E
:10C83000E30F50001800320006003C00E10F5000EA
:10C840000D00320012003C000000E0000800320041
:10C850001E003700E90F50000A003200EA0F5000B6
:10C860000F003200E40F500018003A0015003700A6
:10C87000000880000100370030088000010020001F
:10C88000170037003208800040088000060037009B
:10C8900050088000F9FF3700A0088000F7FF37003C
:10C8A000A2088000B00880000300200001002000E2
:10C8B000C000DD00000020000000710081807100D8
:10C8C00007003700C0088000ECFF37008F81E900C7
:10C8D0004210200051212000A06B2A006133070084
:10C8E0000080FA00000006000200FA00F0BF9F007E
:10C8F000E30F50001F00320006003C00E10F500023
:10C900001100320016003C000000E0000800320078
:10C9100024003700E90F500011003200EA0F5000E8
:10C920001A003200E40F50001E003A0017003700D2
:10C9300094C0BF004300DE00610060009460A80066
:10C940008460A8001C00370094C0BF000080FB007A
:10C950004700DE0094E0A80084E0A800160037003D
:10C9600095C0BF00610060009500A8008500A80088
:10C970001100370097C0BF004300DE006100600077
:10C980009760A8008760A8000B00370097C0BF0021
:10C990004400DE00610060009780A8008780A80046
:10C9A000050037008F81E90042102000F13320009C
:10C9B000A06B2A002B3307000080FA00000006005D
:10C9C0000200FA00F0BF9F00E30F50001600320093
:10C9D00006003C00E10F50000D00320010003C004A
:10C9E0000000E0000800320016003700E90F500098
:10C9F0000B003200EA0F50000E003200E40F50002E
:10CA000010003A000B00370084C0BF000700370059
:10CA100084C0BF000080FB004700DE000E0037002E
:10CA200085C0BF000500370087C0BF004300DE009F
:10CA30000200370087C0BF004400DE0061006000D4
:10CA4000050037008F81E9004210200011372000D7
:10CA5000A06B2A00033307000080FA0000000600E4
:10CA60000200FA00F0BF9F00E30F500027003200E1
:10CA700006003C00E10F5000130032001B003C0098
:10CA80000000E0000800320032003700E90F5000DB
:10CA900016003200EA0F500024003200E40F50006C
:10CAA0002C003A002100370084C0BF004300DE00A4
:10CAB00061016000E1C06000C308DD0084C0BF0008
:10CAC0000034A1000600370084C0BF000080FB00D6
:10CAD0004701DE00C708DD0084C0BF000074A1006C
:10CAE0000140700084E0B7001F00370085C0BF0020
:10CAF00061016000E1C0600085C0BF000004A100CA
:10CB00000140700085E0B7001700370087C0BF0004
:10CB10004300DE0061016000E1C06000C308DD0089
:10CB200087C0BF000034A1000700370087C0BF00E6
:10CB30004400DE0061016000E1C06000C408DD0067
:10CB400087C0BF000044A1000140700087E0B7002B
:10CB5000050037008F81E90042102000613B200072
:10CB6000A06B2A00BF320700020078000080FA00A4
:10CB7000000006000200FA00F0BF9F00E30F500023
:10CB80001400320006003C00E10F50000D0032009E
:10CB90000E003C000000E0000800320011003700E9
:10CBA000E90F500007003200EA0F50000900320080
:10CBB000E40F50000B003A000800370004C1BF002A
:10CBC0000D00370010C1BF000B00370012C1BF00BD
:10CBD000090037001EC1BF000700370020C1BF0099
:10CBE000050037008F81E9004210200091422000AB
:10CBF000A06B2A009B3207004400DE006300600047
:10CC0000E10F50000900320006003900E20F500029
:10CC100008003200E30F500007003A000010200027
:10CC200005003700100020000300370080002000BE
:10CC300001003700000420000080FA000000060018
:10CC4000EF02B000889FBE008A9FBE008C9FBE008E
:10CC50008E1F780080B79F0092B79F00A3B79F00F8
:10CC6000B1B79F006000B8006011B800C0A79F0076
:10CC7000D1A79F00E2A79F00F3A79F0061FC2F00B0
:10CC80008F8040006A804000226D2A000700090062
:10CC9000321878000001B1008FB69700EC8F560073
:10CCA00004003600FA8140004210200021102000CC
:10CCB0000F003700E88F560002003C000D0078009E
:10CCC000020037000D804600710050004200DD0078
:10CCD00061E22100608078000018A30006003A009D
:10CCE00000FE2F008F014000321020006110200054
:10CCF000A06B2A005B3207003FB697000C00E000F3
:10CD000012003200E30F560010003200E60F56000A
:10CD10000E003200E90F56000C003200E10F460011
:10CD20000A003200E20F460008003200E30F46001E
:10CD300006003200E40F460004003200FA8157007A
:10CD400052102000B1102000E9FF37000C00E00075
:10CD5000150035001FB49700AFB497006055B800B8
:10CD60000007EB0009003700A400200005002000A8
:10CD70006033B8000800BE000A01BE00DBCE070029
:10CD80000205BE000004BE000E07E80069001600A0
:10CD9000800F5700F4FF3500C8A79F00D9A79F0058
:10CDA000EAA79F00FBA79F00E88F560083003C0086
:10CDB0008040EB000D00780005FE07003FB09700B3
:10CDC0000000E000510035004FA49700DFA4970059
:10CDD0006FA59700FFA59700BF3107006011B8004D
:10CDE0000040E10001C8E10002D0E10003D8E10009
:10CDF000130039004FA49700DFA497006FA5970098
:10CE0000FFA59700B43107006011B80004F02F00AF
:10CE1000F50F20006033B800B4CE07000040E100F9
:10CE200001C8E10002D0E10003D8E10004003E00A7
:10CE30000006EB0001FD2F008F8640000600370042
:10CE400082FC2F008F01410012102000D111200020
:10CE5000A7FF37000C06E8004FA49700DFA4970057
:10CE60006FA59700FFA597009B3107003D01BE000D
:10CE7000C2B79F00D3B79F008001EB00E3B79F00CC
:10CE8000F3B79F000001EB004FB29700DFB29700AD
:10CE90006FB39700FFB3970094CE0700F4FF2F0005
:10CEA000050020006033B80090CE07000040E1008C
:10CEB00001C8E10002D0E10003D8E100E5FF3E0037
:10CEC0004FA49700DFA497006FA59700FFA59700D8
:10CED000813107006011B8004FB29700DFB29700B0
:10CEE0006FB39700FFB3970080CE07000203BE0028
:10CEF0000002BE000800BE000A01BE0023CF0700EA
:10CF00000205BE000004BE000B0037000086EA00E8
:10CF10001FB09700AFB09700E10F4000E08F5800BE
:10CF200004003600FE81570012102000711220000C
:10CF30006FFF37000004BE000FB097008C00780030
:10CF4000C9FD07000FB09700B0A79F00E20F500087
:10CF50000F00320005003C000000E0000800320035
:10CF6000E10F500010003A0007003700E30F5000B7
:10CF700009003200E40F50000B003A0008003700AF
:10CF800018088800790037006808880077003700A3
:10CF90007808880075003700D808880073003700CB
:10CFA000E80888007100370063FC2F008F81410082
:10CFB00042102000014D20004DFF370011C0B3008A
:10CFC0000D00780082FD07003FB097000000E000F0
:10CFD0004D0035004FA49700DFA497006FA5970080
:10CFE000FFA597003C3107006011B8000040E10048
:10CFF00001C8E10002D0E10003D8E10015003900CA
:10D000004FA49700DFA497006FA59700FFA5970096
:10D01000313107006011B80004F02F00F5FF2F0038
:10D02000F60F20000700200030CE07000040E1008E
:10D0300001C8E10002D0E10003D8E10005003E0094
:10D040000007EB0000FD2F000F00400080BF9F0095
:10D050000600370081FC2F008F8140001210200055
:10D06000A113200022FF37000E07E8004FA497000D
:10D07000DFA497006FA59700FFA597001631070062
:10D080000FB997003206BE0082BF9F000C01BE00A0
:10D09000E9CD07000002BE006033B8000800BE0002
:10D0A0000A01BE00B9CE0700F4FF2F00F5FF2F00E4
:10D0B0006033B8000400E1000588E1000690E1005B
:10D0C0000798E100E8FF3E004FA49700DFA4970017
:10D0D0006FA59700FFA59700FF3007000002BE0074
:10D0E0006033B8000800BE000A01BE00A7CE0700EA
:10D0F0000C02BE006033B800A4CE07000205BE00DB
:10D100000004BE00030037000087EA001FB4970048
:10D11000AFB497000FB097008E00780052FD070063
:10D120000800BE000FB19700B2A79F00E90F5100A1
:10D1300003003200EA0F510007003A0003003700F5
:10D14000680888007108880008003700D80888003F
:10D15000E10888000500370063FC2F008F81410043
:10D1600042102000A14F2000E1FE37000FB09700D1
:10D170006011B80087FD07004F0778004F06BE001A
:10D180004F05BE004F04BE00EF02B10000000600D4
:10D19000E80F500002003400000040007100500011
:10D1A000C200DD0060E221006100780061006000E3
:10D1B000000006000200FA00F0BF9F000001BE0060
:10D1C000EC0F5000040036008F81E900421020006F
:10D1D000E11920000C003700E80F50000200340075
:10D1E00000004000710050004200DD0061E22100BB
:10D1F000608078000018A30005003A008F81E900E4
:10D2000032102000211A2000A06B2A0015310700DF
:10D21000E30F51002000320006003C00E10F5100F6
:10D220001100320016003C000200E000080032004D
:10D2300025003700E90F51000B003200EA0F5100C2
:10D2400015003200E40F51001F003A0018003700AB
:10D25000C718DD0005C1BF000074A10001407000C7
:10D2600005E1B7001C003700C718DD0011C1BF0081
:10D270000074A1000140700011E1B70016003700F2
:10D28000C718DD0013C1BF000074A1000140700089
:10D2900013E1B70010003700C718DD001FC1BF0041
:10D2A0000074A100014070001FE1B7000A003700C0
:10D2B000C718DD0021C1BF000074A100014070004B
:10D2C00021E1B700040037008F81E90042102000FF
:10D2D000511C2000CCFF37000080FA00000006003F
:10D2E0008000EB00B3FF370011002000B1FF3700D2
:10D2F0000400FA00E0BF9F0001027800F2BF9F0027
:10D3000000017800EC0F500004003600E481570063
:10D3100042102000812A200007003700FFB9970043
:10D320000300E900E60F5000050036008F81E90098
:10D3300022002000912A2000A06B2A00C93007009B
:10D34000E80F510002003C000200780002003700A4
:10D350000200410071005000C200DD0040E22100E7
:10D3600084307800E30F51003100320006003C00A9
:10D37000E10F51001700320022003C000200E000E3
:10D380000800320041003700E90F51001D00320053
:10D39000EA0F510032003200E40F51003B003A0026
:10D3A0002F00370067C061004400DD00510A2000F3
:10D3B00091407800F2C8B30082C0600080C0700065
:10D3C00001007800A5E0B7008460A9009460A8007F
:10D3D0003200370067C061004400DD00710A2000A0
:10D3E00091407800F2C8B30082C0600080C0700035
:10D3F00001007800A7E0B70084E0A90094E0A8004D
:10D400002600370067C06100810A20009140780043
:10D4100082CFB30082C0600080C07000010078003D
:10D42000A8E0B7008500A9009500A8001B00370000
:10D4300067C061004400DD00110B200091407800BE
:10D44000F2C8B30082C0600080C0700001007800A4
:10D45000B1E0B7008760A9009760A8000F0037000F
:10D4600067C06100210B20009140780082CFB3009B
:10D4700082C0600080C0700001007800B2E0B70098
:10D480008780A9009780A80004003700E481570036
:10D4900042102000D12E2000A7FF37000080FA00A4
:10D4A000000006000200FA00889FBE008A1F780074
:10D4B000C0BF9F000204BE00010578000001780093
:10D4C000EC0F500004003600E881570042102000A5
:10D4D000210C20000C003700E80F5000020034003F
:10D4E00000004000710050004200DD0061E22100B8
:10D4F000608078000008A30005003A00E88157002A
:10D5000022102000610C2000A06B2A00553007007B
:10D51000E80F510002003C000200780002003700D2
:10D520000200410071005000C201DD000380E800EC
:10D5300044E22100840040001110A0001100A1006D
:10D54000E80F5100050034006680410004004000EF
:10D550001000A1001120A000010037001120A1003F
:10D56000020078006BFB07008A0078000801BE000B
:10D570004FB89700B2FD07008000EB004FB897004E
:10D580008CFB07008000EB004FB89700D4FB07002E
:10D590004F0578004F04BE000080FA00000006002E
:10D5A0000200FA00F0BF9F0080007800EC0F5000EE
:10D5B000050036008F81E90042102000E1152000AF
:10D5C000A06B2A0027300700E80F5000020034004B
:10D5D00000004000710050004201DD000280E800C0
:10D5E00043E22100030040001010A1001000A00041
:10D5F000E88F500003003400660041000300400043
:10D600001000A0000080FA000000060090089000C2
:10D61000E001900001814000628179008100E90011
:10D620001108980002007800000006000200FA00CD
:10D63000889FBE0080047800010478000000E000AC
:10D6400005003A00000028000100E00062003500FB
:10D650000900780060003700010378000100E00055
:10D6600001003D000103EA00090078000900E00024
:10D6700001003D000900EA00010024000800E0006C
:10D6800050003200CF80DE0066815700811F780095
:10D69000110009004688D80001097800CF00780001
:10D6A000DFB89700610AB800C021DD000200200049
:10D6B000809FBE00110009004699D8000001780043
:10D6C0004F00BE00020278008002780040A8DE0011
:10D6D000CF80DE008080CF000100E0000300320038
:10D6E0000002200001015000040037000281CF0039
:10D6F0000200E0000100320070011100EC01510055
:10D700000A003B00C2282000030020000400BE00E5
:10D7100049CC0700440BDD004C00DE000000730024
:10D72000CC88DE0080007800220037001000200046
:10D7300001002000020378000603E9000300330023
:10D740000000400081804800FBFF370000005200CD
:10D7500081805A00680151000201E9000300330092
:10D760008180D1000080D300FBFF37007F03600081
:10D770004319DD004580DE00000141000201410047
:10D78000C1A42900628278000302200006805100B3
:10D7900000A2B9000281E800628078000680B9002A
:10D7A000040240008582480011000900432AD80085
:10D7B000800078000800E00002003D000000280022
:10D7C000810050000900E0000200340001007800F0
:10D7D000010037000100EA004F04BE000080FA009B
:10D7E00000000600800078000000E0000C003D0012
:10D7F00002002C00820F500003003D0000002800B2
:10D80000008040000400370010002800828F500084
:10D81000200034000100EA00170020000800370053
:10D8200000002400808F500002003C0001007800BE
:10D830000200370000002800010050008003EB00C8
:10D840004781DE0000027800F407B20002014100C7
:10D85000A69429000008200004005000E2017B008B
:10D860000380B9000281E80062017B0002A2B900D6
:10D870000000420081804A004909DD004700DE00C7
:10D8800000007100C788DE000700E00001003200E0
:10D890000000EA0000000600010024000100400032
:10D8A000D0FF37000100240001003700C288DE00ED
:10D8B000808F5000FDFF3C00800178000000EB00ED
:10D8C00007003700010140000080D100828F510025
:10D8D000020035008281510001004000C288DE0054
:10D8E0000100E000F7FF3A0000000600889FBE003C
:10D8F0008A1F780080047800010478000102780013
:10D900008003EB005A002000190037006420B800A3
:10D91000809FBE00110009004A88D80000027800EC
:10D920004F00BE008900780004004200808144005E
:10D93000840278008003EB000B00370011037800AD
:10D9400013017800020053004240A9000300340094
:10D950008208780086097800170020008502E80018
:10D960008180E8008381E800888F5200F3FF39004E
:10D97000E10F5200E5FF3E000700E000E9FF3A003A
:10D980004F0578004F04BE0000000600889FBE00CF
:10D990008A1F7800000578001CFF070080047800CB
:10D9A0000A00780019FF0700000478000A007800D8
:10D9B00016FF070000027800098144008800440037
:10D9C0008001EB00050037004A00900061317800CB
:10D9D0008301E8000281E8008180E800848F510023
:10D9E000F9FF39004F0578004F04BE000000060023
:10D9F000889FBE008A1F78000005780003FF07009B
:10DA0000800478000A00780000FF07000004780016
:10DA10000A007800FDFE0700800178000804440039
:10DA2000898044000001EB00040037004A009000A8
:10DA3000E83078000201E8008180E800830F51009F
:10DA4000FAFF39004F0578004F04BE0000000600C1
:10DA5000889FBE008A9FBE0080057800EBFE07000D
:10DA6000800478000B007800E8FE070000047800CE
:10DA70000B007800E5FE0700000578000B00780039
:10DA8000E2FE0700800278004B0090008A0045000B
:10DA90006102780089844400080144008001EB00A1
:10DAA00007003700CB009000628078000000420041
:10DAB00080B478008301E8008984E8000281E800EE
:10DAC000858F5100F7FF39004F05BE004F04BE009F
:10DAD00000000600889FBE008A9FBE008005780077
:10DAE000CAFE0700000578000B007800C7FE07009B
:10DAF000800478000B007800C4FE07000004780062
:10DB00000B007800C1FE0700000278000A054500FE
:10DB100089844400080444008001EB0009003700B8
:10DB20004B009000E9007800680178008280400096
:10DB3000013578008301E8000A85E8008984E8005F
:10DB40000884E800848F5100F5FF39004F05BE00BE
:10DB50004F04BE0000000600889FBE008A9FBE00E2
:10DB600080057800A9FE0700000578000B0078000A
:10DB7000A6FE0700800478000B007800A3FE0700D3
:10DB8000000478000B007800A0FE07000002780077
:10DB90000A05450089844400080444008001EB0024
:10DBA000090037004B009000E90078006801780018
:10DBB00082805000013578008301E8000A85E80082
:10DBC0008984E8000884E800848F5100F5FF39005B
:10DBD0004F05BE004F04BE0000000600889FBE0037
:10DBE0008A9FBE008C1F78008005780087FE0700A2
:10DBF000000578000B00780084FE070080047800A0
:10DC00000B00780081FE0700000478000B0078000C
:10DC10007EFE0700000678000A0345008982440062
:10DC2000080244008003EB00090037004B0090001D
:10DC300065017800E40078000191B90002337800B2
:10DC40008703E8000683E8008582E8000482E80094
:10DC50008C8F5300F5FF39004F0678004F05BE004A
:10DC60004F04BE0000000600889FBE008A9FBE00D1
:10DC70008C9FBE008E1F78008005780063FE070031
:10DC8000000578000B00780060FE07008004780033
:10DC90000B0078005DFE0700000478000B007800A0
:10DCA0005AFE0700000778000A064500098544006F
:10DCB000880444008006EB00160037004B049000F7
:10DCC0006A007C006102B90069007C006101B90052
:10DCD0000A85E8008984E8000000E00006003200C0
:10DCE0000400BE00F2CA070000367C008D06E80082
:10DCF0000C86E8000700370023002000F305980099
:10DD000070814500710029000B007800F51F0700A5
:10DD1000020037008E8F5600E8FF39004F07780069
:10DD20004F06BE004F05BE004F04BE0000000600B7
:10DD3000889FBE008A9FBE008005780033FE0700E2
:10DD4000000578000B00780030FE070080047800A2
:10DD50000B0078002DFE0700000478000B0078000F
:10DD60002AFE070009834400880244000A02450095
:10DD70008003EB000B0037004B019000E6017900B7
:10DD8000E5007900838F50000100340083007800A3
:10DD9000013279008703E8000683E8008582E80005
:10DDA0000482E800808F5300F3FF39004F05BE0066
:10DDB0004F04BE0000000600889FBE008A9FBE0080
:10DDC0008005780011FE0700000578000B00780040
:10DDD0000EFE0700800478000B0078000BFE0700A1
:10DDE000000478000B00780008FE07000983440057
:10DDF000880244000A0245008003EB000B00370054
:10DE00004B019000E6017900E5007900838F500016
:10DE100001003D0083007800013279008703E800AB
:10DE20000683E8008582E8000482E800808F5300C2
:10DE3000F3FF39004F05BE004F04BE00000006008E
:10DE4000889FBE008A9FBE008C9FBE008004780021
:10DE5000EEFD07000005780009007800EBFD0700E3
:10DE60000006780009007800E8FD070080057800CA
:10DE70004904900009007800E4FD0700000040001C
:10DE800060047C0009007800E0FD0700800678004F
:10DE900000022000800F540005003C000B83450069
:10DEA0008C0146006022B8008003EB000D003700B3
:10DEB000C90090000A004500010040000008EB0086
:10DEC0001200370063807800668178000280B90014
:10DED00004024000858248008703E8000683E800CA
:10DEE0008381E800C90090008D8F5300F5FF390051
:10DEF0000A0045000804E900030033008582D100D0
:10DF00000482D300FBFF370004B078004F06BE0048
:10DF10004F05BE004F04BE0000000600889FBE00F3
:10DF20008A9FBE008C1F780000047800B7FD0700B0
:10DF30008004780008007800B4FD070080057800B0
:10DF400008007800B1FD070000057800080078009F
:10DF5000AEFD07000006780008007800ABFD070062
:10DF6000000378000000E00024003200C8009000A8
:10DF700009804400608078006102B9008B8545000B
:10DF800080B578000A05450000B578000900E80072
:10DF90008001400017002000010178000F003700C9
:10DFA000E30079000B004100908F500001003D001C
:10DFB000010878004800900000004500908F500054
:10DFC00001003400010878006108B9000402400033
:10DFD000858248008703E8008381E800868F53002C
:10DFE000EFFF39000C044600020444006131B80020
:10DFF0000400BE002ECA0700000C78004F0678000F
:10E000004F05BE004F04BE0000000600889FBE0002
:10E010008A9FBE00800478007CFD070080057800A0
:10E020000900780079FD07000005780009007800F4
:10E0300076FD0700000478000900780073FD0700F2
:10E04000000278000000E00016003200880344005F
:10E050008A0245000B814500F8FF270006002800D2
:10E060008001EB000D00370049009000E2007800CD
:10E07000888F500002003D00833278000104780050
:10E08000868F5000030034004900900083337800ED
:10E09000010378008301E8000281E800848F5100C9
:10E0A000F1FF39004F05BE004F04BE00000006001E
:10E0B000889FBE000004780054FD070080047800AB
:10E0C0000800780051FD07008000780009814400B5
:10E0D000480090000000410004FE07004F04BE000D
:10E0E00000000600E8874700889FBE008A9FBE00A8
:10E0F0008C9FBE008E1F78000006780043FD07004D
:10E10000800578000C00780040FD070000057800CD
:10E110000C0078003DFD0700800478000C007800BA
:10E120003AFD0700000478000C00780037FD070076
:10E1300080BF9F008B854500EBB79F000A07450015
:10E1400089864400880444000000EB00F0B79F007B
:10E150001F0037004C0490006E007C006102B90083
:10E160006D007C006101B90069007C006105B900A7
:10E170000E87E8008D86E8008984E8000000E00052
:10E180000C0032000400BE00ABC907000A01BE004B
:10E19000C7C907006FB1970000317C007FB09700BE
:10E1A0000000E800F0B79F000281E800E2B79F009E
:10E1B0000700370023002000730698007001460016
:10E1C000710029000C007800C61E0700040037000B
:10E1D000FFB097000FB99700828F5000DDFF390024
:10E1E0004F0778004F06BE004F05BE004F04BE002B
:10E1F0008F00B10000000600889FBE008A9FBE000D
:10E200008C9FBE008E1F780000067800FFFC070080
:10E21000000578000C007800FCFC07008004780002
:10E220000C007800F9FC0700000478000C0078006E
:10E23000F6FC070000077800898544008804440044
:10E240000A0545008006EB00090037004C049000E9
:10E25000E9007C006B007C00F4FC070000357C00CA
:10E260008D06E8008B85E8008984E8000A85E800CF
:10E270008E8F5600F5FF39004F0778004F06BE001D
:10E280004F05BE004F04BE0000000600889FBE0080
:10E290008A9FBE008C9FBE0080057800DBFC0700D3
:10E2A000800478000B007800D8FC07000004780098
:10E2B0000B007800D5FC07008006780008054400B4
:10E2C000898444000006EB00070037004B049000EF
:10E2D0006A007C0043FD070080347C000C06E800E7
:10E2E0000A85E8008984E8008D0F5600F7FF3900A1
:10E2F0004F06BE004F05BE004F04BE0000000600E2
:10E30000889FBE008A9FBE008C9FBE00800578005B
:10E31000BEFC0700800478000B007800BBFC0700FF
:10E32000000478000B007800B8FC07008006780035
:10E3300008054400898444000006EB00070037000C
:10E340004B0490006A007C0053FD070080347C0081
:10E350000C06E8000A85E8008984E8008D0F560065
:10E36000F7FF39004F06BE004F05BE004F04BE0048
:10E37000000006000C00FA00889FBE008A9FBE00C5
:10E380008C9FBE0000047800A0FC07008005780088
:10E39000080078009DFC07008004780008007800E1
:10E3A0009AFC070048059000898444000000400062
:10E3B00060047D000800780037FD07006101B900A6
:10E3C00082BF9F0093BF9F0069007D006101B9007B
:10E3D000E2B79F00F3B79F000800780001FD070037
:10E3E0006101B900C2B79F00D3B79F000900450083
:10E3F000100090006106B9008B8545006FB1970051
:10E40000FFB197000FB897009FB897000AC907009F
:10E410000004BE000C01BE004FB09700DFB09700B3
:10E4200005C907000004540081845C00C149DD0077
:10E430004F44DE0008847100CFCCDE0088357D00BB
:10E440000B0545000C01BE000FB897009FB8970060
:10E45000F9C807000004BE006FB19700FFB1970034
:10E460004FB09700DFB09700F3C8070008044000E2
:10E47000898448004148DD004F44DE0008047000F4
:10E48000CFCCDE00180598004F06BE004F05BE0039
:10E490004F04BE000080FA0000000600889FBE0006
:10E4A0008A9FBE008C9FBE008005780057FC070045
:10E4B000800478000B00780054FC0700000478000A
:10E4C0000B00780051FC0700800678000805440026
:10E4D000898444000006EB00070037004B049000DD
:10E4E0006A007C00EFFC070080347C000C06E8002A
:10E4F0000A85E8008984E8008D0F5600F7FF39008F
:10E500004F06BE004F05BE004F04BE0000000600CF
:10E51000889FBE008A9FBE008C9FBE0000047800CA
:10E520003AFC0700000578000800780037FC070077
:10E53000800578000800780034FC0700800478002B
:10E540000800780031FC070000027800C802900043
:10E5500009804400E0847A000B804500008042007E
:10E560008000EB00040037008100E8000080E80034
:10E57000848F500048003E001000E000FAFF3A008F
:10E580000180450000004000008042000080E8005B
:10E59000810378008703E800848F53000900360068
:10E5A0000100E000400032000100E9000A014500DE
:10E5B000890F5000400039000000D10000B17A00FE
:10E5C000430037003000E000F2FF32000003EB00B0
:10E5D00006047800860678002C002000868143001F
:10E5E00006017800040037000201E8008301E8001A
:10E5F000840F510008003100110009008481D80007
:10E600008000FD000B0040000000400005004000BD
:10E610001000E000F4FF3A0086005100888F50009F
:10E620000700340006004100811F78001100090036
:10E630000C00D80080067800CF0078000104780034
:10E64000840F510010003100828143000400370024
:10E650000201E8008301E800840F51000A00310044
:10E66000110009008481D8008000FD000B004000EB
:10E6700000004000050040001000E000F4FF320000
:10E6800002037800D5FF37000A014500890F5400C6
:10E690000B003D00080037000A004500050040005F
:10E6A0000008EB000A0037000A00450005004000A2
:10E6B0000088EB000600370005004100FCFF370032
:10E6C0000D804300110009000480D80001B17A00D8
:10E6D0004F06BE004F05BE004F04BE0000000600FE
:10E6E00050FA88000000060052FA800050252600EB
:10E6F0000091B900906123000200400050FA8800A8
:10E7000000000600889FBE0080047800BFFB070061
:10E710000004780009007800BCFB070000027800C4
:10E7200050FA8000080444008001EB0056252600C2
:10E7300095612300060037000680B9000080420082
:10E7400049019000003479008301E8000884E80062
:10E75000848F5100F8FF390050FA88004F04BE0042
:10E76000000006000080FB00C300DE00B27F240032
:10E7700002814000C308DD000100500011002000AC
:10E780008008DD0012C9700000000600A0F98000BA
:10E79000B1F9800061014000E0814800A2F98800E1
:10E7A000B3F9880000302A0021002000800F5100BA
:10E7B000818F590007003A00343FEF00363FEF00E9
:10E7C000A17F240011407800E14F40000100320099
:10E7D0008048E800000006000001EB001102210063
:10E7E00000012000B62A070061012000807E24007D
:10E7F000C42A0700E52A0700F03F8A00000006004F
:10E8000020C0B300D7FF3700C1F980008100E800C5
:10E81000C1F9880000A62E00808F500027003A0022
:10E82000383FEF00403F8200E10F4000020032001D
:10E830000000E800403F8A00A3F607000000E00067
:10E8400006003D00917F240011407800E14F400018
:10E85000090032008048E80007003700E800400067
:10E86000807E24000080400010417800E14F41008C
:10E87000010032000248E80084C4BF000038A30051
:10E880000E0032008A2907000000E0000600320076
:10E89000503F8200E10F4000080032000000E80015
:10E8A000503F8A0000000600603F8200E10F4000F8
:10E8B000020032000000E800603F8A00000006000D
:10E8C0008000780060042000808F50000B00390029
:10E8D0000000E800808F5000040036006E00400009
:10E8E000808F500005003A000200370070C0B3006E
:10E8F0009CFF370000C1B3009AFF0700000006002C
:10E900008000780000052000808F50000E003E003F
:10E910000080E900808F50001A003100A002200022
:10E92000808F50001F00390064004000808F50002D
:10E930001000360070FC2F0000804000EC0F5000EB
:10E9400018003E000D00370030052000808F500079
:10E9500004003E000000E900808F50000D003100EF
:10E960000A00370040052000808F50000D003A005B
:10E970000A003700F0C0B3000700370080C0B300C2
:10E9800005003700E0C0B3000300370090C0B300BB
:10E990000100370010C1B30072FF370000C1B3009F
:10E9A00070FF070000000600889FBE008A1F7800E5
:10E9B0000005EB001800200029002000D1D48000C1
:10E9C000C0D48000910F1000310036009500370050
:10E9D000E9007800E0FF2F00010050000100200056
:10E9E000EF0F5000E08F580021003E000060010052
:10E9F0000F0037000E0037000D0037000C00370005
:10EA00000B0037000A0037000B0037000C003700FE
:10EA10000B0037000C0037001500370010003700DE
:10EA20000B0037000C0037000F0037000E003700D6
:10EA3000F0C0B3000D00370080C0B3000B003700FA
:10EA4000E0C0B3000900370000C1B3000700370081
:10EA500010C1B3000500370070C0B30003003700D9
:10EA600040C1B3000100370050C1B3003DFF0700B3
:10EA7000090078009A1AB400100090008A0F500024
:10EA800001003600000578000884E800E4844400B2
:10EA9000D0D48000900F5400CDFF39005E003700C5
:10EAA000D4D480008801440063017A004C10DE0059
:10EAB00001002000ED0F5000E08F580055003E008F
:10EAC000006001000D003700520037001D003700C4
:10EAD0000D00370010003700130037001600370014
:10EAE0004C0037004B003700180037001500370086
:10EAF0001A003700240037001D0037008A0F540029
:10EB00004800310043003700F0FF200000006100A2
:10EB10007BFF07003F003700F0FF2000000061008E
:10EB200067FF07003B003700F0FF20000000610096
:10EB300073FF070003003700F0FF200000006100B2
:10EB40005FFF07000884E800330037004410DD0051
:10EB50004480DE000000440007003700030042004C
:10EB60001000900066FF0700630444002A0037008D
:10EB7000F0FF2000000061008A0F500025003600E1
:10EB80000005780023003700F0FF2000000061003E
:10EB9000010020007B005000E0805800ED0F500085
:10EBA000E08F58001B003E00006001000D003700A0
:10EBB0000C0037000B0037000C0037000D00370049
:10EBC0000C0037000B003700060037000B00370041
:10EBD0000C0037000B0037000C0037000B0037002B
:10EBE0000A003700A0C0B30009003700D0C0B3004E
:10EBF00007003700C0C0B3000500370020C1B300D4
:10EC000003003700B0C0B3000100370030C1B300CB
:10EC1000D4FE07000804E800C0D48000800F540030
:10EC20009FFF39004F0578004F04BE00000006002A
:10EC3000F17E240011407800E14F400001003200D5
:10EC40008048E80058FF3700889FBE008A9FBE00BA
:10EC50000004BE0000402000010020000805400024
:10EC6000898548000B0037000800BE0059170700CF
:10EC7000F2FF2F00F30F2000820F5000838F580007
:10EC80000200320010002000060037006204440039
:10EC9000E0844C008A0F54008B8F5C00F2FF390037
:10ECA0000000EB004F05BE004F04BE000000060050
:10ECB0004A00FA00881F78008A9FBE008C9FBE0021
:10ECC00055FC2F000F8242000006BE0092BF9F003D
:10ECD000A3BF9F00E00F5100E08F590005003A00EC
:10ECE000D20220008000EB000400780074C8070006
:10ECF000DC00370084017800D20220001FB89700A2
:10ED0000AFB89700491707004FE897000040E800A8
:10ED1000C0EF9F001FB89700AFB897007E05400076
:10ED2000E0854800C600370001FB2F000F8440003B
:10ED300088017800520120000A00BE003B1707003E
:10ED40001FE89700EF7097000140700090EF9F0060
:10ED50002FE89700FF70970001407000A0EF9F0020
:10ED60003FE897008F78970001407000B0EF9F0058
:10ED7000FFE097008180FB000FE897004800DD006E
:10ED800001007000BFC097008180FB0001004000BF
:10ED9000F0E79F004800DE0080EF9F00DFE0970073
:10EDA0008180FB006FE097004800DD0001007000EB
:10EDB000AFC097008180FB0001004000D0E79F00BA
:10EDC0004800DE00E0E79F00BFE097008180FB0085
:10EDD0004FE097004800DD00010070009FC09700E1
:10EDE0008180FB0001004000B0E79F004800DE008A
:10EDF000C0E79F009FE097008180FB002FE0970015
:10EE00004800DD00010070008FC097008180FB008A
:10EE10000100400090E79F004800DE00A0E79F004F
:10EE2000FFD897008180FB000FE097004800DD00CD
:10EE300001007000FF7897008180FB000100400016
:10EE4000F0DF9F004800DE0080E79F00DFD89700DA
:10EE50008180FB006FD897004800DD000100700042
:10EE6000EF7897008180FB0001004000D0DF9F0019
:10EE70004800DE00E0DF9F00BFD897008180FB00E4
:10EE80004FD897004800DD0001007000DF78970040
:10EE90008180FB0001004000B0DF9F004800DE00E1
:10EEA000C0DF9F009FD897008180FB002FD897007C
:10EEB0004800DD0001007000CF7897008180FB00E2
:10EEC0000100400090DF9F004800DE00A0DF9F00AF
:10EED000FFD097008180FB000FD897004800DD002D
:10EEE00001007000BF7897008180FB0001004000A6
:10EEF000F0D79F004800DE0080DF9F00DFD0970042
:10EF00008180FB006FD097004800DD000100700099
:10EF1000AF7897008180FB0001004000D0D79F00B0
:10EF20004800DE00E0D79F009FD097008180FB0063
:10EF30002FD097004800DD0001017000BFD097007E
:10EF40008180FB004FD097004800DD0081017000F8
:10EF50002800900000004100E080490090D79F0009
:10EF60004801DE00A2D79F00B1D79F004808DE000D
:10EF7000C0D79F00DFC897008180FB006FC8970053
:10EF80004800DD0001017000FFC897008180FB0090
:10EF90000FD097004800DD00810170001F98970096
:10EFA00000004100E0804900D0CF9F004801DE0012
:10EFB000E2CF9F00F1CF9F004808DE0080D79F007E
:10EFC0009FC897008180FB002FC897004800DD0094
:10EFD00001017000BFC897008180FB004FC89700F7
:10EFE0004800DD0081017000180078000000410039
:10EFF000E080490090CF9F004801DE00A2CF9F0033
:10F00000B1CF9F004808DE00C0CF9F00FFC097002F
:10F010008180FB000FC897004800DD0001007000F0
:10F020009F7897008180FB0001004000F0C79F009F
:10F030004800DE0080CF9F006E054500E0854D0052
:10F0400000402000010020001FB99700AFB99700D1
:10F050000200400083804800800F5500818F5D00D2
:10F0600031FF390053FC2F000F8441008042EB0038
:10F0700062CC7200E5C79F000C00BE00F2FE0700E4
:10F080000000E000100032000C00BE00BA160700BD
:10F090000D003700C1FA2F008F8040000800780073
:10F0A000B0587800B0587800904878006F91970079
:10F0B000FF9197000C00BE00C616070062064600CE
:10F0C000E0864E00630444006E805700800F5400B9
:10F0D000F0FF3A004F06BE004F05BE004F04780017
:10F0E0000080FA00000006002E00FA0023FD2F0029
:10F0F0008F814100D20220004C1607009FA8970084
:10F100000110A2000100EA00010070004F00DE00C3
:10F11000610010000080FA00000006001600FA00EE
:10F12000889FBE008A9FBE000005BE007E0440008E
:10F13000E084480009003700FE815700520120009A
:10F140000800BE00391607000FE897000008A3006A
:10F150000A003A006E044400E0844C0000402000A5
:10F16000010020000A0040008B804800800F5400FE
:10F17000818F5C00F0FF39006044B8000800BE00D9
:10F180004F05BE004F04BE000080FA0000000600DC
:10F19000817E2400F20F2000114861009140900010
:10F1A00011409800A37E2400930061002140980044
:10F1B0009341900033409800C17E2400110161000A
:10F1C000424098009140900051409800B17F240047
:10F1D0009140780061409800C17F24009140780000
:10F1E00071409800D17F2400914078000148980038
:10F1F000E17E24009140780011489800F17E2400BF
:10F200009140780021489800017F240091407800C7
:10F2100031489800117F24009140780041489800BF
:10F22000217F24009140780051489800317F2400CC
:10F230009140780061489800617F240091407800F7
:10F2400071489800717F2400914078000150980027
:10F25000517F24009140780011509800917F240044
:10F260009140780021509800A17F240091407800BF
:10F2700031509800000006001A00FA00881F78003C
:10F280008A9FBE000001EB00110221000001200056
:10F290000B28070061012000807E24001928070048
:10F2A0003A280700E17F2400910F5000040032004B
:10F2B000820120008000EB00807E240000C7070050
:10F2C00040C7BF000018A3000300320010C0B30005
:10F2D00024FD07004027A900A07F24001004E000BF
:10F2E00004003A00817E2400005A2000910F100093
:10F2F000650036005E32EF000004EB005E12E200B3
:10F3000006003A0010002000952807000804E800D5
:10F3100000712200800F5400F8FF3A00F192800043
:10F32000F0282000808F50005700340000C02300D8
:10F33000110020006CFF07000000E00007003A0009
:10F34000000024001100200067FF07006011B800D2
:10F350000000E0001E0032001400370000C023004F
:10F36000110020006DFF07000005BE00E00F5000F7
:10F37000E08F58001B003A0000002400110020001C
:10F3800059FF07000000E00008003A0002C0230017
:10F3900013002000000024001100200044FE07009C
:10F3A000EA0124001B0020000E00370000002400AA
:10F3B0001100200059FF07000005BE00E00F5000BB
:10F3C000E08F580007003A000200240013002000DC
:10F3D00000C023001100200035FE0700EAC1230011
:10F3E0001B0020007C8457000800780068FF07009D
:10F3F0000D00370001FE2F008F80400008007800CC
:10F40000B0587800B0587800904878000FB1970055
:10F410009FB197000A00BE00EE1507006205450087
:10F42000E0854D006304440067805700800F54005E
:10F43000F0FF3A000200240013002000820F550064
:10F44000838F5D0004003A0002C0230013002000F7
:10F450000A00BE0007003700004024001100200011
:10F46000800F5500818F5D0003003A0000C023002B
:10F47000110020000EFE0700820120008000EB003A
:10F48000807E24008EC60700E17E240011407800B3
:10F49000E14F4000010032008048E8004F05BE0007
:10F4A0004F0478000080FA00000006001C00FA00FB
:10F4B000889FBE008A1F78000005780050019000E8
:10F4C000E001900014EC070008C0230019002000A0
:10F4D0000800BE003F15070080B79F0091B79F004E
:10F4E000E3FD2F008F814100320020008380E8007F
:10F4F0000A0078008EEA07007FA89700E30F50000B
:10F5000024003A0062044400E0844C0000402400DF
:10F5100011002000800F5400818F5C00ECFF3A0046
:10F520007C8457000800780019FF0700E3FD2F00D6
:10F530008F81410052012000880078000A00780085
:10F540007BEA0700820120008000EB00807E24001F
:10F550005BC6070000C0230011002000BAFD0700B1
:10F560000000E0000300320000C023001100200072
:10F57000811507000000240011002000B2FD0700E3
:10F580000000E00003003200000024001100200011
:10F59000791507004F0578004F04BE000080FA007F
:10F5A000000006008000EB00010898007100980040
:10F5B0002118980020019000010978003001900086
:10F5C00002014100400090003DC63700200190003C
:10F5D00012037800150020002300200009003700E6
:10F5E0006482410062807900810F500003003A007C
:10F5F0000300410010009000000006008582E80032
:10F6000084017800868F5200F5FF39000000050064
:10F610000400FA0080089000E1BF9F00F000900015
:10F62000F1BF9F004300200064815700A100290022
:10F63000AC1907000080FA0000000600889FBE0099
:10F6400000047800E1FF0700800478000000E0007B
:10F6500012003200780090000008A300050032007C
:10F660007001440023002000810029000800780078
:10F670009C190700090C98000080EB00100C980002
:10F68000780090000000A000700498000018A3000B
:10F690000200320008007800DDFF07000900780052
:10F6A0004F04BE0000000600889FBE008004780062
:10F6B000020478006119B800F10F5100E08F590081
:10F6C0005B003E00026001001100370012003700AD
:10F6D00013003700140037001500370017003700FB
:10F6E0002A0037002D0037002E0037002F0037008A
:10F6F000300037003300370036003700390037005C
:10F700003C0037003F00370042003700440037001C
:10F710000809DD00490037000889DE00470037008E
:10F720000881400045003700088150004300370041
:10F730000888B90000017800400037000800E000A8
:10F740000E003A00004027000000E00003003200F5
:10F75000880078000900780029FC070023002000B9
:10F76000F3049800708144007100290009007800BA
:10F770005C1907000801780030003700110009000B
:10F780008800D800000178002C0037001100090023
:10F790008800D80001017800280037000881700037
:10F7A00026003700088168002400370008816000C7
:10F7B000220037000001EB00888F50001F003A0044
:10F7C0001D0037000001EB00888F50001B00320045
:10F7D000190037000001EB00888F5000170034003B
:10F7E000150037000001EB00888F50001300350032
:10F7F000110037000001EB00888F50000F003D0022
:10F800000D0037000001EB00888F50000B003C001A
:10F81000090037000100E00007003A00020037004D
:10F820000100E000020032000800E00002003A009F
:10F830000001EB00010037001200200002007800F8
:10F840004F04BE00000006000600FA00889FBE00BC
:10F850000004780020029000800A90000581420098
:10F86000E2047A004C48DE0001002000EE0F500058
:10F87000E08F5800F6003E00006001000E003700E7
:10F880001100370019003700270037003200370019
:10F890003D0037004F003700730037008A00370003
:10F8A000990037009C003700C2003700CF003700B6
:10F8B000D5003700DF003700780090000000A1007D
:10F8C00070049800E200370068019000180890006A
:10F8D0000000E800100C980000004000C448DD0063
:10F8E000C488DE0001307900C4003700E8019000D0
:10F8F000980890008100E800110C98008180400079
:10F90000080890002801900000004000020040001C
:10F910001000900080B07900080890000080E80096
:10F92000000C9800CA003700E80190009808900089
:10F930008100E800110C980081804000F0FF200059
:10F9400000806400480190000000400060017900E0
:10F9500082B07900A900370018099000F0FF20005C
:10F96000008064004802900000004000E801900020
:10F9700082004100E181790003307A000201E90050
:10F98000120C98009D003700F0FF20008081640079
:10F990000200420010029000180890000000400091
:10F9A000E80090000101400012007800840F500030
:10F9B00003003900B5BF9F00C4BF9F00130037008C
:10F9C00003004000C80090000000400060897800FB
:10F9D000D1FF3700F0FF2000808164000200420068
:10F9E00010019000E800900018089000000040000E
:10F9F0008080400071BA970011007800820F50009B
:10FA000011003900B5BF9F00C2BF9F00D0BF9F004B
:10FA10002000200070049800630020006A815700D5
:10FA20006100290008007800AE1807000040270098
:10FA30000000E000860032008000EB000800780043
:10FA40006FFB07008200370003004000C8009000F1
:10FA50000000400004B07800180890000080E90021
:10FA6000100C9800ACFF3700180890000000400010
:10FA7000E80090008101400013017800090078003F
:10FA8000F00FB200E10F500007003200040039000F
:10FA90008000EB00E20F500009003A000700370039
:10FAA0008200EA0006003700820078000200E000D1
:10FAB00003003D008200EA00010037008280EA0076
:10FAC000810978004D003700E80090001808900088
:10FAD000000040006081780080804000F1B897000D
:10FAE0008981FB0008007800EFFE0700980890006D
:10FAF0008100E900110C98006801900081804000AD
:10FB0000803079003D0037004448DD004480DE004D
:10FB10000080420082FF3700E80090001808900043
:10FB2000000040006081780080804000F1B89700BC
:10FB30008981FB0008007800DBFE070000027800E6
:10FB4000180890000080E900100C98000400E00004
:10FB5000040032000988A3000A0032000998A300BB
:10FB60000800320028019000080890008000400042
:10FB700001004100900190000400E00002003A0002
:10FB80000700370023002000080890000000400014
:10FB9000A8009000010040001090A0000200370073
:10FBA000010041001090A100080890000080410071
:10FBB0005BFF370002004200A0019000100190009E
:10FBC000020141004800900000014100F1FF2000C7
:10FBD000818064008381410008007800411807009B
:10FBE00008089000630040004DFF3700F1FF20003F
:10FBF0008180640008007800DE0D0700080890008E
:10FC00000000E80046FF37006801900018089000E7
:10FC10000000E800100C98000000400088089000E8
:10FC20008100E80001307900F0FF200000806400CE
:10FC30003BFF3700180890006801900080004000EA
:10FC400061017900020C98000000E900100C980096
:10FC50004F04BE000080FA00000006000000FA0019
:10FC6000889FBE008A9FBE008C9FBE0080057800E2
:10FC7000010578008F0678000100780097C407001E
:10FC80000004780063064000650040000000A10009
:10FC9000808747008D047800004027000000E000C6
:10FCA000030032008A0078000B007800D4FA0700C5
:10FCB00020002000F00598000B089000800C7800D0
:10FCC000A844980063804400080178008A00780006
:10FCD00088C407008C017800090178009100290090
:10FCE0000B007800FF1707008D0778004F06BE0055
:10FCF0004F05BE004F04BE000080FA000000060061
:10FD000080007800201A9000F40140000001EB0010
:10FD10000800370001089000B30F100004003A00FB
:10FD2000710090000010A000F00098001000050085
:10FD30000201E800840F5100F6FF390000000500C1
:10FD4000889FBE008A1F78000004780001057800B3
:10FD5000700090000020A000700498008004EB0068
:10FD60000100E00004003A000D00370008007800B0
:10FD7000B5FE07008904E800780090000008A300A1
:10FD80000C0032000028A3000A0032008A8F5400C1
:10FD9000F6FF3A000700370008007800AAFE0700C7
:10FDA000780090000008A300020032000028A300A1
:10FDB000F9FF3A00780090000020A100700498003C
:10FDC0004F0578004F04BE0000000600889FBE006B
:10FDD0008A1F780000047800010578007000900008
:10FDE0000020A000700498008004EB000100E000F7
:10FDF00008003A001B00370008007800C0FF070029
:10FE00008904E8000000E0000A003A0008007800D9
:10FE10008DFE0700780090000008A3001600320055
:10FE20000028A300140032008A8F5400F2FF3A0029
:10FE300011003700780090000010A00070049800B6
:10FE400008007800F2FD07000E0037000800780077
:10FE5000ABFF07000000E000F6FF3A000800780062
:10FE600079FE0700780090000008A300020032002D
:10FE70000028A300F5FF3A00780090000020A100C0
:10FE8000700498004F0578004F04BE000000060083
:10FE900000017800700090000008A3000B00320001
:10FEA0000018A30009003A00221890000000E000AA
:10FEB0000300320002007800C4FF07000200370090
:10FEC000020078009EFF07001000050000000500FA
:10FED00080017800201990000000EB00EF0F510026
:10FEE00006003E00020041007400400001B07900AD
:10FEF0000200E800A0199800100020000000060091
:10FF00000001780001037800A019900074024000FD
:10FF10000000EB008302E900140037008000E800D5
:10FF2000B40F130010003A0025199800818040009A
:10FF3000F480400080017800050278000000400055
:10FF4000740040000101410001005000030037002F
:10FF5000123079008301E8000281E800848F5100AB
:10FF6000FBFF39001000050001007800830F5000EE
:10FF7000EAFF3900000005008000EB00211898001E
:10FF80000000060000027800920078000100E00006
:10FF9000060035008DFD07008001EB000000E00049
:10FFA0000F003A00130020000D003700130020005E
:10FFB000F0FF2900808F50000900360012019000E8
:10FFC0008001EB000000E800808F50000400320048
:10FFD000940069000100EA0001007000CF01DE001A
:10FFE00003007800000006000400FA00881F780073
:10FFF000000478008102780000002A00808F500001
:020000040001F9
:1000000003003A00080078006A17070077003700FD
:1000100012007800980F500074003A000282E80045
:10002000F0FF2500F1FF2F0005004000E0804800B0
:10003000EE0F5000E08F58006C003E0000600100A1
:100040000E0037001A003700210037002B00370060
:1000500030003700350037002B00370035003700FF
:1000600040003700430037004500370049003700A3
:1000700056003700580037005A0037008381E900E6
:100080001400780000014000840078000002EB00BA
:100090000400370028009000113178000402E800C5
:1000A0000281E8008180E800830F5200F9FF3900E7
:1000B00020002000700498008080EB000800780089
:1000C0005EFD07000000E00048003A000E00370027
:1000D000780090000010A1007004980008007800DB
:1000E0004BFD0700806127000000E0003F00320068
:1000F00008007800CEFA07003C0037007800900036
:100100000010A000700498000800780040FD07006F
:1001100036003700780090000008A300330032005A
:1001200008007800C8FD0700F7FF37002000200016
:10013000F4FF370094007800D1BF9F0008007800DA
:1001400063FF07000080FB00E0BF9F00430020002A
:1001500066815700B100290008007800E116070009
:1001600022003700940078000800780064FF070040
:100170001E0037000000EB00201C98001B00370019
:10018000220190009400780008007800EB16070028
:10019000160037008381E900140078000001400058
:1001A000840078000002EB00040037004800900053
:1001B000113178000402E8000281E8008180E80043
:1001C000830F5200F9FF390008003700080078005B
:1001D000700C07000500370008007800210C0700AC
:1001E00002003700080078005D0C07004F0478001B
:1001F0000080FA0000000600889FBE008A1F780079
:10020000AE7EAB001F003200AD5EE2000D0032009A
:10021000ACDEEC00ACFEB700FF4F50000200340033
:1002200000CEB300ACFEB700ACDEBF000000FB00A8
:1002300001003B000000EA0080407800E0C0B3000D
:10024000CA1007008040EB00AD5EE20004003A00F7
:1002500011C0B30010002000D05EE20001003200A7
:100260000000EB008000FD00D0FEB7008000FD0024
:100270000004E000030032008040EB00E0C0B30067
:10028000BA100700AEBEAB00D800320084C4BF0075
:10029000684460003B003200AA5EE2000B003A00B6
:1002A0008040EB0050C0B300B01007008040EB006E
:1002B00060C0B300AD1007008040EB0070C0B30019
:1002C000AA10070010C0B300AAFEB700B1EA2100CF
:1002D00091407800100020000104E000040032008A
:1002E0000100FB0072C0B300EA0F500007003C00A1
:1002F00022002000811F7800110009000200D800B0
:1003000000017800CF0078000241E80082C0400080
:1003100001007800ABFEB70040C6B30080CF5000AC
:1003200012003400A95EEC0080407800A9FEB700FE
:1003300010C0B300ABFEB700E3CF500001003A009D
:10034000A97EEF0098EA2100184478000804E00034
:1003500006003A008840780070C0B30083100700A0
:100360008840780060C0B30080100700B1EA210027
:1003700091407800A9DEBF00654040007B10070077
:100380009A003700009380005E12B400823E200085
:100390000280B900A2F82000809FBE001100090071
:1003A0004288D800800478004F00BE00AA5EE200B8
:1003B0002100320008007800AAFEB7005018200083
:1003C000808F54000800360001C2B30050C0B30053
:1003D0006610070001C2B30060C0B30063100700DD
:1003E00001C2B3001200370080162000808F540035
:1003F0000500360001C2B30050C0B3005B10070017
:1004000001C2B3000700370040152000808F540060
:100410000900360001C2B30050C0B30053100700FA
:100420008840780060C0B300501007008840780012
:1004300070C0B3004D1007008040EB005018200042
:10044000808F54000400360011C0B300100020005B
:10045000CF5EE200010032000000EB008000FD00F2
:10046000CFFEB7008000FD000004E000090032006C
:1004700001C2B30050C0B3003C10070001C2B3007A
:1004800060C0B3003910070001C2B30070C0B300F0
:10049000361007008040EB0070E92F000080440018
:1004A000F70F500004003E0011C0B3001000200000
:1004B000CE5EE200010032000000EB008000FD0093
:1004C000CEFEB7008000FD000004E000090032000D
:1004D00001C2B30050C0B3002410070001C2B30032
:1004E00060C0B300211007008040EB0070C0B30073
:1004F0001E1007008040EB00B0EA2F00008044008F
:10050000EE0F500004003E0011C0B30010002000A8
:10051000CD5EE200010032000000EB008000FD0033
:10052000CDFEB7008000FD000004E00009003200AD
:1005300001C2B30050C0B3000C1007008040EB00B4
:1005400060C0B300091007008040EB0070C0B3002A
:10055000061007008040EB0040152000808F5400FB
:1005600004003E0011C0B30010002000CC5EE20089
:10057000010032000000EB008000FD00CCFEB7005F
:100580008000FD000004E000060032008040EB0027
:1005900060C0B300F50F07008040EB0070C0B300EF
:1005A000F20F070040152000808F54000F003E001E
:1005B000AB5EEC00ABFEB700E34F500003003A0027
:1005C00001C2B30050C0B300E80F0700B0EA210039
:1005D00051C0B30090CF1000040034008040EB0005
:1005E00050C0B300E10F0700AB7EEF00AE3EAB00A2
:1005F0008A003200F3FA200041EA210044FB200087
:100600001304E0000800320011417800634041000B
:100610008048780002C2B300824F500003003600C9
:1006200082487800010037008048EB008301E80031
:100630008100E800848F5100F1FF3A00A65EE200DD
:100640000A0032000802200061EA2100914078008F
:1006500008407800C50F07000804E80040022000A9
:10066000800F540019003200F7FF370041EA2100E3
:10067000914078000104E0000200320010C2B30093
:10068000BA0F070051EA2100914078000104E00010
:100690000200320020C2B300B40F070071EA21004B
:1006A000914078000104E0000200320000C2B30073
:1006B000AE0F070081EA2100914078000104E000BC
:1006C0000200320030C2B300A80F0700A45EE200AF
:1006D00003003A0010002000A65EE2000100320094
:1006E0000000EB00804078000004E00003003200CE
:1006F00010002000CB5EE200010032000000EB00A1
:100700008000FD00CBFEB7008000FD000004E0008B
:10071000030032008040EB0010C2B300930F0700CB
:10072000A55EE20003003A0010002000A65EE20091
:10073000010032000000EB00804078000004E0007F
:100740000300320010002000CA5EE2000100320007
:100750000000EB008000FD00CAFEB7008000FD0035
:100760000004E000030032008040EB0020C2B30030
:100770007E0F0700A75EE20003003A001000200091
:10078000A65EE200010032000000EB00804078002D
:100790000004E0000300320010002000C95EE20007
:1007A000010032000000EB008000FD00C9FEB70030
:1007B0008000FD000004E000030032008040EB00F8
:1007C00000C2B300690F0700A85EE20003003A0010
:1007D00010002000A65EE200010032000000EB00E5
:1007E000804078000004E000030032001000200088
:1007F000C85EE200010032000000EB008000FD0056
:10080000C8FEB7008000FD000004E00003003200D5
:100810008040EB0030C2B300540F0700AE1EAB00A7
:100820003C003200AFCFBF000400320010C0B30064
:1008300011002000C75EE200010032008000EB00E2
:10084000C7FEB7000104E0000200320020002000D3
:10085000AA1A0700B0CFBF000400320010C0B300D6
:1008600011002000C65EE200010032008000EB00B3
:10087000C6FEB7000104E0000200320020002000A4
:100880009E1A0700B1CFBF000400320010C0B300B1
:1008900011002000C55EE200010032008000EB0084
:1008A000C5FEB7000104E000020032003000200065
:1008B000921A0700B2CFBF000400320010C0B3008C
:1008C00011002000C45EE200010032008000EB0055
:1008D000C4FEB7000104E000020032002000200046
:1008E000861A0700B3CFBF000400320010C0B30067
:1008F00011002000C35EE200010032008000EB0026
:10090000C3FEB7000104E000020032002000200016
:100910007A1A0700AE5EAB005300320021E12100DD
:100920000324210002E0210004E2210013007800EA
:10093000910F100001003D00800878000000E000E9
:1009400003003200920F100001003400000978000B
:100950008180E8008381E8000281E800848F5000F4
:10096000F2FF3A006225210043E2210012007800E4
:10097000910F100001003D00800878008180E800A0
:100980000281E800838F5000F8FF3A008004EB00FA
:100990000905780000E02100EA0078000024210029
:1009A0006A0078000101500020E121006A0078000F
:1009B000810150000200E00001003D000001EB0059
:1009C000000220000090B900809FBE0011000900C5
:1009D0004308D800000478004F00BE0060DF21000B
:1009E0006940780088407800E00E0700E28F5400EC
:1009F00003003A00F85DEC0088407800DB0E070049
:100A00008904E8000A85E800E78F5400E1FF3A0016
:100A10006825210009E22100DADF210019017800B0
:100A2000180078000000E00001003D000000EB002D
:100A3000010220000180B900811F78001100090027
:100A40004208D800CF007800804078003A40780013
:100A5000C60E07000884E8008984E800A02521006C
:100A6000800F5400EDFF3A00AEDEAB0016003200FE
:100A70008040EB00B45EE20004003A0011C0B30015
:100A800010002000C25EE200010032000000EB0016
:100A90008000FD00C2FEB7008000FD000004E00001
:100AA000030032008040EB00D0C1B300AF0E07005E
:100AB000B45EE20004003200B47EEF0001C2B30075
:100AC000D0C1B300A90E0700AF1EAB004B0032002F
:100AD00070938000F40F500042003C00619380004E
:100AE00050938000D1F2070022002000110009007D
:100AF0000200D8008000FD00067D20000680400036
:100B0000F3F92000C9012000830F500020003600B7
:100B10000577210005804000B9012000830F5000B7
:100B20001B0036000471220004804000A90120004F
:100B3000830F500016003600006B23000081400038
:100B400099012000830F5100110036008901200017
:100B5000F0D52600800F51000D003E0006805000A9
:100B6000EC844400830F50000900360005805000DB
:100B70008904E800830F500005003600048050000F
:100B8000F9012000830F5000010036008084EB0043
:100B9000709380000000E00001003D000000EA00CA
:100BA00080004000800220000104500001003B0052
:100BB0000004EB000900E0000800350010F580009B
:100BC0000000E000020035008040EB00670E0700E7
:100BD0008840780009407800640E070019F5880005
:100BE0000600370010F580000000E000020035002C
:100BF0008040EB005D0E0700A2BEEF00AF3EAB00F1
:100C000024003200A15EEC00A1FEB700EA4F5000C4
:100C100020003A00A17EEF0081938000500920005F
:100C2000808F500005003C008040EB0060C2B300A4
:100C30004E0E070001C2B3001400370080112000DF
:100C4000808F50000500340001C2B3006E404000A8
:100C5000460E07008040EB000C003700A8F62F007E
:100C6000088440004544DD002208200011000900EE
:100C70000204D800000478008840780060C2B30005
:100C80003A0E070001C2B30088C0500070C2B30022
:100C9000360E0700AF5EAB00010032001AE8070015
:100CA000AF7EAB00010032008F0407004F057800D3
:100CB0004F04BE0000000600881F78000104780081
:100CC00080F5880031002000420120000300200050
:100CD000F4F1070080F5800008017800C10F2800BA
:100CE00083F107004F04780000000600881F780099
:100CF00000047800AE1EE20002003A0080F5800099
:100D000079F1070008007800AE3EB7004F04780084
:100D100000000600AE1EB600000006000080EA00DB
:100D2000AE1EB60070F5880002003A0080F5800023
:100D30006BF107000000060002EA21001241780072
:100D40000080FB00C301DE00AE9EAB001700320046
:100D5000C19380000100E0000C003200810F5000C0
:100D60000500340082CF51000300360003007800F4
:100D7000A0FEB700070037000204E00005003200C3
:100D80000240E900A0FEB700020037000100780031
:100D9000A0FEB70001EA210091407800814F510088
:100DA00002003200E0C1B300F00D070000000600B1
:100DB000D1EA2100914078000000E00003003D00EE
:100DC00063406000014070000200370000C0EA008C
:100DD00001406000ADFEB700000006000080FB008F
:100DE0004013880060C2BF000008A300FDFF32006E
:100DF000401380000080FB0000000600401F200020
:100E000020F9880000C0EB00F4FF070000C0EB00F1
:100E1000F2FF0700E14F400002003200241FE20011
:100E2000FAFF3A000080FB0000000600CDC2A800D7
:100E300000C0EB00E9FF3700CDC2A900EFFF0700BB
:100E400011002000E14F400002003200F7FF0700D0
:100E50008000EB000100780000000600889FBE00C3
:100E60000004BE004006200030F9880000C0EB00FE
:100E7000DAFF0700E14F400003003A00261FE200BE
:100E800025003200F9FF3700E24F400022003A000F
:100E9000F10F20004113880060C2BF000008A300CA
:100EA000FDFF320040138000004C780041138800A1
:100EB00060C2BF000008A300FDFF320040138000A5
:100EC000104498004113880060C2BF000008A300CE
:100ED000FDFF320040138000204498004113880039
:100EE00060C2BF000008A300FDFF32004013800075
:100EF0003044980064044400E4845400E5FF3A0060
:100F000000C0EB00B5FF070000C0EB00B3FF070017
:100F100010002000010037000000EB004F04BE006D
:100F200000000600889FBE0000047800814478001D
:100F3000B2FF0700E14F400015003A000940780079
:100F4000A6FF0700E3CF4400130032000920200071
:100F500018407800A1FF0700184090000884E800BE
:100F60009EFF07008984E900F9FF3A0000C0EB000A
:100F70009AFF070000C0EB0098FF070000C0EB00DD
:100F800096FF07007F006000E50F5000020032006E
:100F90000000EB0001003700100020004F04BE00ED
:100FA00000000600889FBE008A1F78000045780078
:100FB0000204BE000004E00006003D000A74A10027
:100FC0006011B80070C3B300F6FF0700E14F500096
:100FD00028003E0095FF070097FF0700F10F200053
:100FE0000000E000240032000A4078000064A00005
:100FF0007AFF07004848DE000100200077FF070065
:101000004048DE000100200074FF07004849DD0071
:101010004840DE0000007100C848DE006FFF070096
:10102000084078006DFF070050C9B3000A04E000D3
:10103000040032006E405000E84F550001003200BD
:1010400010C0B30065FF0700A8C0B300EC4F550007
:1010500002003A0000C0EB0060FF070000C0EB0098
:101060005EFF07000004E00002003D000844E900C4
:10107000FAFF3A008080FB00010078004F057800FD
:101080004F04BE00000006000400FA00889FBE0066
:101090008A1F7800110020000004E00082003A005E
:1010A000CBC2BF000068A3007D003200CDC2A80003
:1010B000C9C2A900B0132000101388006422EF00F9
:1010C00061E2A80061E2A90062C2BF0031CEB300B4
:1010D000014060004041B30062E2B70062C2BF005D
:1010E000C1CFB300014060000004A00062E2B7007D
:1010F00061E2A800A8C0B30000C0EB0037FF070002
:101100000844E900FCFF3A006011B800084078008C
:10111000A4FF070080447800E14F50004A003A00E5
:10112000803E200030F98800A21A20000300200031
:1011300080C0B3009BFF0700E14F50002A003A0037
:10114000EA84570000C0EB0024FF0700805C7800B1
:1011500066805700808F5400FAFF3A000FF897001E
:10116000E14F500038003A009FF89700A0CAB30042
:1011700080CF500034003A00261FE2000600320003
:10118000020020000300240090CAB30085FF07007E
:101190000004E000F8FF3A00261FE2002A003200B7
:1011A0006011B800A0C3B3007EFF07000004E00098
:1011B00025003A006A84570000C0EB0007FF0700D3
:1011C000005C7800890F5400FBFF3A00EFF09700B5
:1011D0000180FB00C8C0B3000068A3001B003A00F8
:1011E00048C0B300190037006011B80090CAB300BE
:1011F0006CFF070028C0B3009ACAB300E14F50004B
:10120000020036000944780009457800261FE200F4
:10121000050032006011B8000A40780061FF070045
:101220000004E000F9FF3A00261FE2000600320049
:10123000022020000300200000C1B30059FF070076
:101240000004E000010032000044EB000880FB00D5
:1012500010F98800F5FE07000804E0000B003200DA
:10126000481FA90061E2A90062C2BF0031CEB300ED
:10127000014060008041B30062E2B70030C0B300BB
:101280006262B70061E2A80005003700EAFE0700CD
:10129000E6FE0700C9C2A80061E2A900481FA80035
:1012A00048DFBF008080FB00010078004F05780018
:1012B0004F04BE000080FA0000000600110020006C
:1012C0000004E00002003A0048DFBF008080FB001D
:1012D0000100780000000600889FBE008A1F780089
:1012E00001057800844478000004E00032003A00F0
:1012F0000404E0003000320048DFBF0061046000F9
:10130000300020002D003A00227FAB0004003A009C
:101310004918DD00C711DE00830170004911DD00AE
:10132000E1CF54000B003A0010C1B3001DFF0700CD
:101330000004E00019003A00012020000A007800B3
:10134000C6FE07000000E000140032008844780068
:101350001300370020C1B30012FF07000004E000B3
:101360000F003A0009447800012020000A007800AC
:10137000BAFE07000000E000030032000A20B000BF
:101380000844E900F8FF3A00884478006011B8008A
:10139000C0C0B30003FF07000100370019C0B3004D
:1013A000A2FE07000000EB000904E0000300320089
:1013B0001000200001003700400020004F05780099
:1013C0004F04BE0000000600889FBE008A9FBE003A
:1013D0008C1F7800810578000204BE000445780067
:1013E0000004E00040003A000404E0003E00320047
:1013F00048DFBF00310020000008A3003B003A0096
:1014000048DFBF00640660002100200037003A007A
:1014100010F980000038A30004003A00C918DD006C
:10142000C714DE00898470004914DD00E14F5500C7
:101430000C003A000801BE0080C1B300D9FE0700CD
:101440000004E00021003A00E1CFB3000B00780077
:10145000B4FE07000000E0001C0032000C457800DC
:101460001B00370066006000040032000A81FB00A8
:101470000300200070C9B300CAFE07000801BE00C7
:1014800090C1B300C7FE07000004E00010003A005E
:101490000A447800C1CFB3000B007800A1FE07001A
:1014A0000000E000030032000B20B0000844E90017
:1014B000F8FF3A0008457800D1CFB3000000EB00F8
:1014C00098FE07000000E00001003A001AC0B300D7
:1014D00056FE07008000EB000A04E0000300320023
:1014E00011002000010037004100200001007800B9
:1014F0004F0678004F05BE004F04BE0000000600F6
:101500001000FA00889FBE008A1F7800020578004C
:10151000480020000004E000D1003A0048DFBF008E
:10152000E104600038002000CD003A00EACF50000E
:10153000A400320008003E00E1CF50001600320047
:1015400010003900E2CF50004F003200E3CF5000CE
:101550000A003A004F003700ECCF50009C003200E8
:101560006011B80090C0B3009B003900EDCF50006F
:101570009E003200EECF5000A9003200480020004B
:10158000B60037002CFE07000000E000B00032007B
:1015900026FE07001B0037006011B80090C0B300A2
:1015A00080FE07000004E000A9003A0001012000CD
:1015B0007680570029FE07000000E000A4003200FA
:1015C000AFE897000180FB004600DE003FF2970085
:1015D000AFF09700E14F50000C003A000480FB0090
:1015E0004809DD00020040000000E8000100200082
:1015F0004A09DD00C600DE00810071004A00DD00FE
:10160000008DBE0009047800940037000181FB00C2
:101610004611DE001FF097000080FB004200DD0055
:10162000000141000FF09700630060004A00DD00F8
:10163000000141000201E80003002000FFE89700DC
:10164000EFC060004FF097000008B2004780DE0056
:1016500080C04000630062000000400080C0400085
:1016600081C0E8008180FB00E98050008100E90032
:10167000030033000201410083814900FBFF370072
:10168000028DBE00DFFF3700002020000009780037
:10169000DCFF370010F98000640460001D00320098
:1016A0006011B800D0C8B3003EFE07000004E0009F
:1016B00067003A0000C0EB00C8FD070001012000F0
:1016C00076805700E5FD07000000E0006000320072
:1016D00008C3B30000C0EB00C0FD07000844E900E8
:1016E000FCFF3A004FF197000281FB004411DE003D
:1016F00000012000010020000201E9000300330086
:101700000000400081804800FBFF3700008DBE00D4
:10171000510037006011B80090C0B30021FE0700EF
:101720000004E0004A003A000101200076805700E2
:10173000CAFD07000000E000450032005FF197009D
:10174000CFF0970010F98000620260000F003200B5
:1017500001007800F003B200000040000208B2006F
:101760004711DE00020040000000E8007FF1970012
:101770000281FB004611DE000201E9000200DD00EB
:1017800001002000008DBE00340037000280FB0005
:1017900001017800C207B2004291DE000201E800B8
:1017A000E3006000C308DD004500DE0080804000EB
:1017B0008100E8000191B900028DBE0004047800A8
:1017C0002600370022DFBF00004978008DFF370078
:1017D0006011B800A0C0B300F2FD070001012000B5
:1017E0000004E00016003200190037006011B80054
:1017F000A0C3B300EBFD07000004E00014003A00B2
:101800000904780000C0EB0074FD070000757C003F
:101810000804E800E40F54000F003200F9FF37001D
:101820006011B800D0C8B300DEFD07000004E0007E
:1018300007003A0000C0EB0068FD0700010420002B
:101840000A00780085FD07000000E00002003A0071
:1018500018002000010037000004EB0073FD0700B2
:10186000080078004F0578004F04BE000080FA00A1
:101870000000060030F980000000E00002003200A5
:101880000000E90030F9880020F980000000E00045
:10189000020032000000E90020F988000000060084
:1018A000889FBE00800478000004EB00030037002E
:1018B000803E20002A1F07000804E800890F54001A
:1018C000FBFF39004F04BE00000006008040EB0023
:1018D00050C0B300250B070001C2B30000C1B30024
:1018E000220B0700E0152000EDFF07008040EB0011
:1018F00000C1B3001D0B070001C2B30010C1B3004B
:101900001A0B0700E0152000E5FF07008040EB0000
:1019100010C1B300150B070001C2B30040C1B300F2
:10192000120B0700E0152000DDFF07008040EB00F0
:1019300040C1B3000D0B070001C2B30050C1B3009A
:101940000A0B0700E0152000D5FF07008040EB00E0
:1019500050C1B300050B070001C2B30020C1B300A2
:10196000020B0700E0152000CDFF07008040EB00D0
:1019700020C1B300FD0A070001C2B30030C1B300AB
:10198000FA0A0700E0152000C5FF07008040EB00C1
:1019900030C1B300F50A070001C2B300D0C1B300E3
:1019A000F20A0700E0152000BDFF07008040EB00B1
:1019B000D0C1B300ED0A070001C2B300E0C1B3001B
:1019C000EA0A0700E0152000B5FF07008040EB00A1
:1019D000E0C1B300E50A070001C2B30050C0B30084
:1019E000E20A0700E0152000ADFF07008040EB0091
:1019F00050C0B300DD0A070001C2B30060C0B300ED
:101A0000DA0A0700E0152000A5FF07008040EB0080
:101A100060C0B300D50A070001C2B30070C0B300B4
:101A2000D20A0700E01520009DFF07008040EB0070
:101A300070C0B300CD0A070001C2B300C0C1B3003B
:101A4000CA0A0700E015200095FF07008040EB0060
:101A5000C0C1B300C50A070001C2B30040C2B30051
:101A6000C20A0700E01520008DFF07008040EB0050
:101A700040C2B300BD0A070001C2B30050C2B300A8
:101A8000BA0A0700E015200085FF07008040EB0040
:101A900050C2B300B50A070001C2B300F0C1B300E1
:101AA000B20A0700E01520007DFF07008040EB0030
:101AB000F0C1B300AD0A070001C2B30080C1B3009A
:101AC000AA0A0700E015200075FF07008040EB0020
:101AD00080C1B300A50A070001C2B30090C1B300E2
:101AE000A20A0700E01520006DFF07008040EB0010
:101AF00090C1B3009D0A070001C2B300A0C1B300AA
:101B00009A0A0700E015200065FF07008040EB00FF
:101B1000A0C1B300950A070001C2B300B0C1B30071
:101B2000920A0700E01520005DFF07008040EB00EF
:101B3000B0C1B3008D0A070001C2B30020C2B300D8
:101B40008A0A0700E015200055FF07008040EB00DF
:101B500020C2B300850A070001C2B300014078002B
:101B6000820A0700E01520004DFF07008040EB00CF
:101B700000C2B3007D0A070001C2B30030C2B30047
:101B80007A0A0700E015200045FF07008040EB00BF
:101B900030C2B300750A070001C2B30010C2B3001F
:101BA000720A0700E01520003DFF07008040EB00AF
:101BB00010C2B3006D0A070001C2B30060C2B300D7
:101BC0006A0A0700E015200035FF07008040EB009F
:101BD00060C2B300650A070001C2B30070C2B3005F
:101BE000620A0700E01520002DFF07008040EB008F
:101BF00070C2B3005D0A070001C2B3000040EB00F1
:101C00005A0A0700E015200025FF07008040EB007E
:101C100001407800550A070001C2B300E0C0B300DC
:101C2000520A0700E01520001DFF07008040EB006E
:101C3000E0C0B3004D0A070001C2B30010C0B300FA
:101C40004A0A0700E015200015FF07008040EB005E
:101C500010C0B300450A070001C2B30060C1B30061
:101C6000420A0700E01520000DFF07008040EB004E
:101C700060C1B3003D0A070001C2B30070C1B300E8
:101C80003A0A0700E015200005FF07008040EB003E
:101C900070C1B300350A070001C2B30080C0B300B1
:101CA000320A0700E0152000FDFE07008040EB002F
:101CB00080C0B3002D0A070001C2B30090C0B3007A
:101CC0002A0A0700E0152000F5FE07008040EB001F
:101CD00090C0B300250A070001C2B300A0C0B30042
:101CE000220A0700E0152000EDFE07008040EB000F
:101CF000A0C0B3001D0A070001C2B300B0C0B3000A
:101D00001A0A0700E0152000E5FE07008040EB00FE
:101D1000B0C0B300150A070001C2B300C0C0B300D1
:101D2000120A0700E0152000DDFE07008040EB00EE
:101D3000C0C0B3000D0A070001C2B300D0C0B30099
:101D40000A0A0700E0152000D5FE07008040EB00DE
:101D5000D0C0B300050A070001C2B30020C0B30021
:101D6000020A0700E0152000CDFE07008040EB00CE
:101D700020C0B300FD09070001C2B30030C0B300AA
:101D8000FA090700E0152000C5FE07008040EB00BF
:101D900030C0B300F509070001C2B30040C0B30072
:101DA000F2090700E0152000BDFE07008040EB00AF
:101DB00040C0B300ED09070001C2B30020C0B3006A
:101DC000EA09070001C2B30000C1B300E709070038
:101DD00001C2B30010C1B300E409070001C2B3009F
:101DE00040C1B300E109070001C2B30020C1B30044
:101DF000DE09070001C2B30030C1B300DB090700F0
:101E000001C2B3000040EB00D809070001C2B300D3
:101E100010C0B300D509070001C2B300E0C1B30090
:101E2000D209070001C2B30070C2B300CF09070096
:101E300001C2B30080C1B300CC09070001C2B300E6
:101E400090C1B300C909070001C2B300A0C1B3002B
:101E5000C609070001C2B300B0C1B300C30907003F
:101E600001C2B300C0C1B300C009070001C2B30082
:101E700040C2B300BD09070001C2B30050C2B300A5
:101E8000BA09070001C2B300F0C1B300B7090700E7
:101E900001C2B300D0C1B300B409070001C2B3004E
:101EA00060C1B300B109070001C2B30070C1B30043
:101EB000AE09070001C2B30080C0B300AB09070040
:101EC00001C2B300D0C0B300A809070001C2B3002B
:101ED000E0C0B300A50907000080200083FB0700D5
:101EE000100020002D193700889FBE0070F32F00CE
:101EF0007012B400A1122000810F500004003E00B7
:101F0000301FA8008040EB0070C2B30097090700A3
:101F100001938000F092800080804000803E20008D
:101F20000088B900A2F82000801F78001100090085
:101F30004288D800800078004F007800C118B100B6
:101F400010022000808F500004003E008040EB0013
:101F5000D0C0B30085090700303FA800B9C72F00E3
:101F6000090078004012B400A8C12000880F50007A
:101F700004003E008040EB0000C1B3007B09070075
:101F8000305FA800090078004212B400880F5000AA
:101F900004003E008040EB0010C1B300730907004D
:101FA000307FA800090078004412B400880F500068
:101FB00004003E008040EB0040C1B3006B09070005
:101FC000309FA800090078004612B400880F500026
:101FD00004003E008040EB0020C1B300630907000D
:101FE00030BFA800090078004812B400880F5000E4
:101FF00004003E008040EB0030C1B3005B090700E5
:1020000030DFA800090078004A12B400880F5000A1
:1020100004003E008040EB000140780053090700B7
:1020200030FFA800090078004C12B400880F50005F
:1020300004003E008040EB0010C0B3004B090700D5
:10204000311FA800B9F92F00090078005612B4001A
:10205000E8312000880F500004003E008040EB0073
:1020600060C1B30041090700313FA80009007800B2
:102070005812B400880F500004003E008040EB006E
:1020800070C1B30039090700315FA8007412E20083
:1020900002003A007212E200040032008040EB00BD
:1020A000D0C1B30031090700317FA800B19380008F
:1020B00080022000808F50000B003400D1938000FC
:1020C000800C2000808F500007003400B0122000E8
:1020D000808F500004003C00319FA8008040EB003E
:1020E000E0C1B3002109070031BFA8008040EB0028
:1020F000C0C1B3001D09070031DFA8008040EB001C
:1021000050C2B300190907002612E2000D00320088
:102110008040EB0090C1B300140907008040EB0041
:10212000B0C1B300110907008040EB0040C2B3000A
:102130000E0907008040EB00F0C1B3000B09070057
:1021400031FFA8002812E200040032008040EB00BA
:1021500080C1B30005090700321FA8002A12E2005F
:10216000040032008040EB00A0C1B300FF0807006C
:10217000323FA800461B07000000E00004003200C8
:102180008040EB00E0C0B300F8080700325FA80011
:102190006A12EC00E20F50000A003E006C12EC00E4
:1021A000E20F500007003E0070938000F40F5000D3
:1021B000040034008040EB0080C0B300EB0807004F
:1021C000327FA80082F9800093F98000F0FF2F0091
:1021D000F1002000800F5100818F590006003A0065
:1021E0008040EB0020C0B300E008070001C2B3004C
:1021F00030C0B300DD08070071F980008101E800FC
:1022000073F98800700C2000808F510002003E009E
:102210000000E800D092880084F32F000480400082
:10222000620C2000820F500001003E00D492880012
:1022300000E72F0000804000820F500003003E00A6
:102240005A32EF00800C2000E092880080DA2F00E4
:1022500000804000820F500001003E00E4928800A0
:1022600000CE2F0000804000E1182000810F5000B8
:1022700001003E005C32EF00004B2000808F5100D7
:1022800001003A002E3FEF004F04BE0000000600A0
:1022900090089000E0019000018140006281790087
:1022A0008100E90011089800020078000000060093
:1022B000889FBE008A1F780000047800C004900048
:1022C000F3FF07000000400060857C00C804900018
:1022D00008007800EEFF070000004000E0807C006E
:1022E000EF0F5500070032000A00E000050035003E
:1022F00070022000800F550002003C000A40780068
:102300009A0807004F0578004F04BE000000060041
:10231000800178000003EB000271220054002000CD
:10232000A5002000811F7800110009008281D800DB
:1023300081017800CF0078000000E00004003A003E
:102340000600E00002003A00E10F510003003A00ED
:1023500006C3B3008658400016002000811F780095
:10236000110009000581D80000017800CF00780035
:102370000402E900EBFF3A00E0C2B30080487800B5
:1023800070C7B3009040980076405000A04098007D
:1023900075404000B0409800C4409800000006001E
:1023A0000E00FA00881F7800F080570092442A003F
:1023B0000C000900B2587800D100B1004004900030
:1023C000B3FF07000000400060047C001000200004
:1023D00052FA07003B1307000000EB00E10F440036
:1023E00004003200EF80570008007800C8FF0700A3
:1023F000708057005B1307004F0478000080FA00DC
:10240000000006000E00FA00881F7800F0805700D8
:1024100062452A000C000900B2587800D100B100D2
:10242000400490009AFF07000000400060047C0018
:10243000E10F440002003A00850C07000700370056
:102440001000200035FA0700EF80570008007800E0
:10245000AFFF070070805700550C07004F0478004D
:102460000080FA00000006000E00FA00881F7800C5
:10247000F080570032462A000C000900B25878005C
:10248000D100B1004004900081FF0700000040002F
:1024900060047C001000200020FA070009130700E8
:1024A0000000EB00E10F440004003200EF80570011
:1024B0000800780096FF0700708057002913070076
:1024C0004F0478000080FA00000006000E00FA00B9
:1024D000881F7800F080570002472A000C0009008E
:1024E000B2587800D100B1004004900068FF0700A6
:1024F0000000400060047C001000200007FA070084
:10250000F0120700080078007C1307000000E000CC
:1025100005003200EF805700080078007CFF0700BC
:10252000708057000F1307004F0478000080FA00F6
:1025300000000600E6874700889FBE008A9FBE0015
:102540008C9FBE008E1F780000047800C0049000AD
:102550004FFF070000004000E0847C0089BF9F001F
:10256000C80490000800780049FF07000000400000
:10257000E0847C00F9B79F00C80490000800780050
:1025800043FF07000000400060877C00C804900003
:10259000080078003EFF070000004000E0867C0055
:1025A000C80490000800780039FF070000004000D0
:1025B00060867C00C80490000800780034FF0700A3
:1025C00000004000E0857C00C8049000080078000E
:1025D0002FFF07000000400060857C00C8049000C9
:1025E000080078002AFF07000000400060847C009B
:1025F00000102000C9F90700884378000A437800DA
:102600008B4278000C4278008D4178000E417800B2
:10261000EFE897000FF09700800807004F07780059
:102620004F06BE004F05BE004F04BE006F00B10054
:1026300000000600889FBE008A9FBE00000478004C
:10264000C004900012FF070000004000E0857C00FD
:10265000C8049000080078000DFF0700000040004B
:1026600060857C00C80490000800780008FF07001F
:102670000000400060817C008A4078000B407800B8
:102680008E0807004F05BE004F04BE000000060084
:10269000889FBE008A9FBE0000047800C00490009E
:1026A000FBFE070000004000E0857C00C8049000AD
:1026B00008007800F6FE07000000400060857C00FE
:1026C000C804900008007800F1FE070000004000F8
:1026D00060817C008A4078000B4078008508070004
:1026E0004F05BE004F04BE0000000600889FBE00DC
:1026F0008A9FBE0000047800C0049000E4FE07003A
:1027000000004000E0857C00C804900008007800CC
:10271000DFFE07000000400060857C00C8049000D8
:1027200008007800DAFE07000000400060817C00AD
:102730008A4078000B4078007C0807004F05BE00F7
:102740004F04BE0000000600889FBE008A9FBE00A6
:102750008C1F780000047800C0049000CCFE0700B5
:102760000000400060867C00C804900008007800EB
:10277000C7FE070000004000E0857C00C804900010
:1027800008007800C2FE07000000400060857C0061
:10279000C804900008007800BDFE0700000040005B
:1027A00060847C00200020005CF907008C407800E9
:1027B00000C2B3006D0707008B40780030C2B30041
:1027C0006A0707008A40780010C2B3006707070055
:1027D0008840780020C2B300640707004F067800E5
:1027E0004F05BE004F04BE0000000600E68747000C
:1027F000889FBE008A9FBE008C9FBE008E1F7800FF
:1028000000047800C0049000A1FE07000000400012
:10281000E0847C0089BF9F00C80490000800780015
:102820009BFE070000004000E0847C00F9B79F0099
:10283000C80490000800780095FE070000004000E2
:1028400060877C00C80490000800780090FE0700B4
:1028500000004000E0867C00C8049000080078007A
:102860008BFE07000000400060867C00C8049000DA
:102870000800780086FE070000004000E0857C002C
:10288000C80490000800780081FE070000004000A6
:1028900060857C00C8049000080078007CFE07007A
:1028A0000000400060847C00400020001BF907000D
:1028B0008FF0970000C1B3002C070700EFE89700E6
:1028C00010C1B300290707008E40780040C1B30053
:1028D000260707008D40780050C1B300230707008A
:1028E0008C40780020C1B300200707008B4078009F
:1028F00030C1B3001D0707008A4078000040EB009C
:102900001A0707008840780010C0B30017070700B7
:102910004F0778004F06BE004F05BE004F04BE00B3
:102920006F00B10000000600889FBE008A1F78007B
:1029300000047800C004900055FE0700000040002D
:1029400060857C00C80490000800780050FE0700F5
:102950000000400060847C0040002000EFF8070089
:102960008A40780060C1B300000707008840780003
:1029700070C1B300FD0607004F0578004F04BE008C
:1029800000000600881F78004004900040FE070009
:102990000000400060047C0000042000DFF8070015
:1029A00088407800D0C1B300F00607004F047800DB
:1029B00000000600881F78004004900034FE0700E5
:1029C0000000400060047C0000012000D3F80700F4
:1029D00088407800E0C1B300E40607004F047800A7
:1029E00000000600889FBE008A1F7800000478005F
:1029F000C004900026FE07000000400060857C00B7
:102A0000C80490000800780021FE07000000400084
:102A100060847C0000202000C0F807008A40780015
:102A200060C2B300D10607008840780070C2B300CE
:102A3000CE0607004F0578004F04BE0000000600D8
:102A4000889FBE008A1F780000047800C0049000B0
:102A50000FFE07000000400060857C00C804900065
:102A6000080078000AFE07000000400060847C0037
:102A700010002000A9F807009211070088007800D4
:102A80000A0078002C1207004F0578004F04BE00A2
:102A900000000600889FBE0080047800400490007B
:102AA000FBFD070000004000800144000001EB0036
:102AB000630079000008B000F10F2000810F500082
:102AC00004003600D1472A000900780063F40700AB
:102AD000060037000281E800C0112000800F51007D
:102AE000F3FF3A0003007800DF1807004F04BE0030
:102AF00000000600501F00005210000000000000FF
:102B0000961A000016010000020000000000FE00FE
:102B100005901F005A02CE0011200000501F000037
:102B200000000000000000000000000000000000A5
:102B30000000000000000000000000000000000095
:102B40000000000000000000000000000000000085
:102B50000000000000004E001B3E1B002E1B260044
:102B60001B3A9900FA98B600985098000498B00063
:102B7000975E97001097B20096509600E0959A00E5
:102B800095289500EC949200944694000294BA0023
:102B9000937E930032938A00929E0F00920F8600DC
:102BA0000F7A0F006E0F46000F320F000A0F1E0043
:102BB0000F820E00F20ECA000EBA0E00AE0EA20078
:102BC0000E920E00760E0A001F000000F29D090012
:102BD0009E000000000027009E3E9E0001004E0067
:102BE0009E010000569E0000000000005C9E7200E6
:102BF0009E0100004E9E010000569E000000000055
:102C000000819E00909E0000000000004C99500042
:102C100099809900A89AC6006CF86C00286D6A002B
:102C20006DAC6D00EE6D34006E986E00DC6E2000B1
:102C30006F8E6F000670580070727000FC70460056
:102C400071807100BA714E007288720082735800F0
:102C500091029200D0913400926692009A921A00EA
:102C6000937693004893200095A49300F6939400E4
:102C700094C29400DA94F200944A95005CB5000086
:102C8000C6110000BC04000000000000AC1B0000E6
:102C9000B400000000000000FC0F00000400000071
:102CA00000000000A22F0000DC0000000000000077
:102CB000AE0F00003000000000000000421F0000C6
:102CC0000200000000000000021F000008000000D9
:102CD00002000000601C0300800F0F000F000000C6
:102CE000601C0000A0000000000000000A1F00009F
:102CF00008000000020000003AA74400A7000000FE
:102D000000000000E01E00000C00000000000000B9
:102D1000AA3000000C00000000000000441F00006A
:102D20000200000000000000961D000030000000BE
:102D3000000000003A1F0000040000000000000036
:102D4000EC1E00000C00000000000000121F00003C
:102D500008000000000000001A1F0000080000002A
:102D600000000000B21E0000100000000000000083
:102D7000461F0000020000000000000000080000E4
:102D80007606000000000000D21E00000E000000C9
:102D900000000000821600000C020000000000008D
:102DA0003E1F00000400000000000000481F00005B
:102DB000020000000200000001000000221F0000CD
:102DC00006000000000000004A1F00000200000092
:102DD000000000008E180000080200000000000043
:102DE000781E00001400000000000000241E0000F7
:102DF00024000000020000000000010000000000AC
:102E000001000000000100000000010000000000BF
:102E100001000000000100000000010000000000AF
:102E200001000000000100004C1F00000200000033
:102E300002000000E8030000281F00000600000058
:102E4000000000004E1F0000020000000200000011
:102E50002ECB0000481E00001800000000000000FB
:102E6000C0110000060000000200000076117A0088
:102E700011901100BE1100000200000002000000CD
:102E800032110000901100002E000000020000002E
:102E90002E0354000068000079006D0000690000F6
:102EA0006F002D00004900004900200000200000B4
:102EB0002000200000200000200020000020000052
:102EC0002000200000200000200020000000000062
:102ED0007A110000160000000200000016034D00E9
:102EE000006F0000620073000079000061002E0096
:102EF000006F000072006700000000007611000003
:102F000004000000020000000403090004000000A7
:102F100032110000440000000200000009024300DA
:102F2000000201000080FA00090400000001020014
:102F30000201000005240000100104002402020028
:102F4000052406000001050024010000010705001A
:102F5000810308000002090004010000020A0000C9
:102F60000000070005020200400000000705820083
:102F700002400000000000002011000012000000CC
:102F80000200000012010000020200000008170009
:102F9000060A000000000100020001001E110000EE
:102FA00002000000000000001611000008000000F0
:102FB00000000000C61D00003000000000000000FE
:102FC000601E00001800000000000000001D00004E
:102FD0009600000000000000A01E0000120000008B
:102FE00000000000C21E00001000000000000000F1
:102FF000F61D00002E000000020000001011140059
:1030000012130000011617000084030084038400DB
:103010000384030084038400038403000000000091
:1030200000A00F00A00FA0000FA00F00A00FA00095
:103030000FA00F0084038400030000008C1E00001A
:103040001400000000000000DE0F00001E00000061
:1030500000000000F81E00000A000000020000004E
:10306000900104000120000096002C0001000000E7
:103070002E1F00000600000000000000760E000079
:103080003801000002000000A2A1AD00A18E0000E6
:10309000D8A1000000000000DDA1E800A1010000AF
:1030A000F7A1010000FAA1000000000000FDA1004E
:1030B0000EA20100001AA20001001E00A2000000E2
:1030C00000002300A22EA20001003C00A20000008C
:1030D00000004000A248A20001003C00A200000045
:1030E00000005300A25FA20001007B00A2010000CB
:1030F00081A200000000000087A29300A20100004E
:103100007BA201000081A2000100B100A201000029
:10311000B7A2010000BDA2000100C300A20100008F
:10312000C9A2010000CFA2000000000000D5A2004B
:10313000E2A20100007BA20001008100A2010000C8
:10314000B1A2010000B7A2000000000000F3A2003D
:1031500004A30100001AA20001001B00A30100004B
:103160001EA200000000000021A33300A301000004
:103170001AA20100001BA30001001E00A200000013
:1031800000004B00A354A30001001A00A20100009C
:103190001BA30100001EA200000000000064A300A9
:1031A00070A30100007BA20001008100A2010000C9
:1031B000B1A2010000B7A2000100BD00A201000001
:1031C000C3A2010000C9A2000100CF00A2000000BC
:1031D00000008700A394A3000100B500A300000035
:1031E0000000B700A3C4A3000100B500A3000000C5
:1031F0000000DD00A3E8A3000100B500A30000006B
:1032000000000100A40EA4000100B500A30000000E
:1032100000002800A432A40001003C00A20100002C
:103220003EA40000000000007E3000002C000000E2
:1032300000000000341F0000060000000000000035
:103240000000000090089000E00190000181400023
:10325000628179008100E90011089800020078007D
:1032600000000600FC0D070000003700660D070097
:103270000000E000FDFF3A0000003700F4100700F6
:103280000000E000FDFF3A009EC0A90000480400D5
:1032900001000000000006000000FE000000060023
:1032A000889FBE008004780040049000E5FF07007E
:1032B0000000400060047C0009007800E1FF070086
:1032C0008000780090052000800F54000400360034
:1032D000810D2A000900780060F20700060037001F
:1032E000C90190000181400088004400C0BA21005B
:1032F0006100780000B179004F04BE0000000600B4
:10330000889FBE008004780040049000CDFF070035
:103310000000400060047C0009007800C9FF07003D
:103320008000780090052000800F540004003600D3
:10333000810D2A000900780048F2070006003700D6
:10334000880144004901900081804000C0BA2100FA
:1033500061017900823178004F04BE000000060050
:10336000010F2A003DF2370040092A000000060044
:10337000000006008180400062B52100E100790074
:103380000140010080D5290000000600E0AC2100CA
:1033900000000600F0874700889FBE008A9FBE009D
:1033A0008C9FBE008E1F780080BF9F00588E8000CB
:1033B000698E800020009000D0B79F0050C0B300FD
:1033C000E8EC07000085EB008085EB006066B80044
:1033D0003E0020000800BE007E0507008A0F500056
:1033E0008B8F5800020031000005BE000806BE00A9
:1033F000008020000100200008044000898448006B
:103400000E07E900F3FF3A0091102A00E10F450092
:10341000E08F4D004600320061054500E0854D001B
:10342000EAB79F00FBB79F000C04BE002A002000F3
:103430000800BE00D00507000A05E9000040200092
:103440000100200008044000898448000A00E000D0
:10345000F7FF3A000C00BE00FA0507006FB09700B6
:10346000FFB09700250607008FB897002100900055
:10347000C1BF200049060700780607000C00BE0007
:10348000540507006FB19700FFB19700800F5100FE
:10349000818F59000200320041122A0024003700B7
:1034A00062054600E0854E00E93F20007A8457001F
:1034B00088017800320020000A00BE005B0507008A
:1034C00032002000DFB097000800780062B60700E5
:1034D0000000E00013003A00DFB19700E3814100F3
:1034E000D3B79F0062054500E0854D008904E900DF
:1034F000EEFF3A00FC815700220020000A00BE00C7
:103500004A05070022002000DFB097007C805700AA
:1035100051B6070001172A000000E00004003A003D
:1035200002003700A1142A000100370061192A00A7
:103530000FB89700C9F107004F0778004F06BE008B
:103540004F05BE004F04BE000F01B1000000060091
:10355000889FBE008A9FBE008C9FBE003A8E80006E
:103560004B8E80000A04BE000006EB002DDE290011
:103570000800BE00200507009D0F500007003A001C
:103580000C06E8000808B0000980B0008D86E8004D
:10359000E80F560005003200F5FF37000C00E00090
:1035A00002003200E80F560003003A000A00BE0095
:1035B000710507000006EB004760DD00CF80DE00EC
:1035C0000A0040008B8048009E050700ACDBBF006E
:1035D0008080FB00000020008C01460022DE2900D4
:1035E00063017900030020000200700083807000F6
:1035F000C2050700310B2000D0BA2100E705070003
:10360000160607004F06BE004F05BE004F04BE0061
:1036100000000600889FBE008A9FBE008C9FBE00EF
:103620003C8E80004D8E80000C04BE000005EB0037
:103630002BDE29000800BE00EF0407009B0F50009E
:1036400007003A000A05E8000808B0000980B00049
:103650008B85E800E80F550004003200F5FF3700C5
:103660000080EB000A00E0000F0032000A04E900CD
:103670004744DD00CFC4DE000C0444008D844C00C0
:103680000800BE00E2040700ACFBB700620444007F
:10369000E0844C00D3BA2100320B20000800BE00A9
:1036A000E20407000000EB004F06BE004F05BE001D
:1036B0004F04BE00000006000000FE00FEFF3700C1
:1036C0000400FA00889FBE008A9FBE008C1F78000D
:1036D00010002000B0D488000280220000002000EA
:1036E0008000780002007800508E8800618E88008B
:1036F0000040240011002000308E8800418E880098
:10370000B3202000C2B822008300780070D92200C4
:10371000230C070094C4BF000008A300020032007D
:103720009EC0A80001003700D8150700CFC0BF0019
:1037300081CFB300014060005040B300CFE0B7003C
:1037400060A9210097EF0700B0D48000708E880038
:1037500080002000B0908800588E8000698E800024
:103760006055B8009ABF9F00ABBF9F003C0020008F
:103770000800BE00970407008A0F50008B8F580086
:10378000030039000005BE0098BF9F00A9BF9F003D
:1037900000802000010020000804400089844800C7
:1037A0000C06E900F2FF3A00E00F5500E08F5D00E3
:1037B00002003A000C047800080037001FB9970097
:1037C000AFB9970062004100E0804900D3D4800087
:1037D000C2BF20009504070018002000C0B52900D2
:1037E000A2170700080078004F0678004F05BE00BA
:1037F0004F04BE000080FA0000000600CC3AEF0043
:103800008080EB0060A921008CEF0700B60C070058
:10381000813E200060A921009DF1070060A92100E0
:10382000EC0907007D0C07002CD580000C00D100AE
:10383000E105600002003A000C08A300F3FF3A0023
:10384000C9AC210020042000010C200010C8700029
:103850001904CF0005003900D60B07000000E00076
:1038600002003200A4CA0200000000002004200070
:10387000F101200010C86000080578000800E00091
:10388000E2FF32000B00E000020032000C08A3004F
:10389000DEFF3A000A00E900110020008008DD0088
:1038A0008180EA00998C6000B1D48000818E88000C
:1038B000E1FF2F0080805000D2FF37009EC0A9009A
:1038C0008EA4EF008AA4EF00AA24EF00AC24EF003E
:1038D000AE24EF002000200030258800A824EF004F
:1038E0008644A900F0092000802488006024880014
:1038F0008804A800010021004808DE00C0248800D8
:103900000000EB008018EB008018EB000000E800DE
:10391000EC0F5000FBFF3A009424A8009624EF001F
:1039200094A4A9009424A900810020000700370076
:10393000512488005C70EF006270EF0063D0BF001C
:103940006370EF0064D0BF006470EF008AC4BF00F2
:103950000038A300F6FF3A0010002000C083880062
:10396000D08388007C30EF007E30EF008430EF00A1
:103970000000EB0004052100A20421008000780073
:10398000E506210023072100001AEB000019EB00D7
:1039900001F07A0001F079000000E800E30F500028
:1039A000F9FF3A008000210080828800D0002000CA
:1039B00050258800000321001080880080C0B300DB
:1039C00000F0B70040C8B30001F0B7004270EF004C
:1039D0004030EF00000006007810E20022003A00BC
:1039E00014002000C4838800D18380000100E0001F
:1039F0001D003A00D483880058D0BF00E24F500029
:103A000006003A00808280000148780081CCB30033
:103A100080828000114098000000060058D0BF004E
:103A2000E14F500010003A000184880083C0B300C9
:103A30003082800003487800318280000203210038
:103A40009200980040C8B300904098000484880019
:103A500040828000034878004182800092009800F4
:103A600000C8B3009040980000000600F08280007B
:103A700083C0B300E70F50000A003E00F0828000D0
:103A80008041780010C0B3005650E20004003200BC
:103A900056D0BF00E14F500002003A0020C0B300F2
:103AA00056F0B7000380FB005E30B50080828000D6
:103AB0000348780080032100408388005CD0BF0069
:103AC0000008A30002003200034178001200370012
:103AD000034178008041EB000600370040838000FE
:103AE000D18280003158780040838800D1828800DC
:103AF0000241E900834F5100F8FF3A000000060040
:103B000040838000D1828000315878004083880053
:103B1000D18288000241E9000204E000F8FF3A0087
:103B2000000006007C30EF007E30EF0058D0BF0070
:103B3000E24F500009003A0081C0B300408280008B
:103B400001487800418280008003210090009800A5
:103B500080CCB300904098000000060036D0BF0033
:103B60000080FB007103210091407800C808DD004F
:103B700080807000F0828000808F5000070031004C
:103B800061032100914078008180FB0037D0BF00A5
:103B90004800DD0001007000F0828800B3FF0700DC
:103BA00081032100808280001100980081CCB30045
:103BB0008082800011409800000006000080FB0019
:103BC000800140000180FB00008041004300DD00D7
:103BD0000200210002014000124090000074A10088
:103BE00010419800A00421000104E000010032000F
:103BF0000005210082317800124090000064A1008D
:103C000010419800E4004100114090000064A000C1
:103C10009040980000000600889FBE008A1F780030
:103C200000447800014578008184FB000938A30036
:103C3000020032008040EB00E0FF07000928A300EB
:103C40000300320011C0B30008407800DBFF07001A
:103C50000880FB0000004000A14A20000AF0780024
:103C60004F0578004F04BE000000060001417800B7
:103C70000004E0000C003A0081C0B30040828000E4
:103C800001487800418280000003210090009800E4
:103C9000C0C8B3009040980041C8B3008082800043
:103CA00011409800000006008080FB0081804000E9
:103CB0000280FB0080804000C308DD00020021007C
:103CC000028140001240900043C8B30003407000DE
:103CD0001041980040002100808040001140900079
:103CE00003407000904098000000060000437800F8
:103CF0000082FB00814378000104E00003003200F1
:103D000084004200000521000200370084004200C8
:103D1000A0042100E10278000500E00002003A0062
:103D200005007800000006000682FB009202980061
:103D3000834A7800154090000044B20090429800F9
:103D40001540900081C8B300014070009042980077
:103D50000704E000030032000400420001052100D6
:103D60000200370004004200A104210001004000CD
:103D70001024A200050078000000060080407800B2
:103D800094C4BF000058A300180032000181FB005A
:103D90000201410004052100E2017A001300BE0087
:103DA0000504200000806200010020008089BE0020
:103DB000E2017A000004200001002000931968004D
:103DC00093916800040141001224A200920078003F
:103DD000114090000044B20090409800920078009A
:103DE00011409000054068009040980000000600D7
:103DF0000000EB00A0248800602488000082880076
:103E000000000600018280000100E00011003A007D
:103E1000A12488006124880020002000302588002B
:103E2000412588008644A900F009200080248800EC
:103E3000602488009EC0A800010037009404A800F8
:103E400094C4BF000008A300FCFF32001000200053
:103E5000008288000000060021E3A90085A0A900D7
:103E6000004006000C00FA00F27F80002043A90009
:103E700000188000A0BF9F0010188000B0BF9F00F6
:103E800020188000C0BF9F0030188000D0BF9F0066
:103E900040188000E0BF9F0050188000F0BF9F00D6
:103EA000601880007018800040632800E0198800C6
:103EB000E20F51001400320005003C000200E00057
:103EC00008003200E10F51001A003A0009003700E3
:103ED000E30F510010003200E40F510015003A00CA
:103EE00011003700C802A900C822A8001000200055
:103EF00003003700C822A900C842A8002000200003
:103F0000F07F88000B003700C842A900C862A800F3
:103F100030002000FAFF3700C862A900C882A8005C
:103F200040002000F6FF3700C882A900C802A800A0
:103F3000FE2FEF0010002000F17F80000100DD0067
:103F400001C6270001007000801988009021EF0051
:103F5000C0C1B3009161B70021E3A80000000000D8
:103F60000000000000000000000000000000000051
:103F70002043A80000000000000000000000000036
:103F80000000000000000000000000003D63A800E9
:103F90000000000000000000000000000000000021
:103FA000000000000000000090C1BF0081CFB300FE
:103FB000014060000024A00090E1B7000000000074
:103FC00000000000000000000000000000000000F1
:103FD000000000003D23A900820078006C8057009B
:103FE000061407000080FA0000000600E07F800051
:103FF000BBE4070021E3A90095A0A9003DE3A900C7
:104000000000EB00800C8800900C8800C802A9001A
:10401000C822A900C842A900C862A900C882A90094
:104020007C15070083153700889FBE000004BE0082
:104030007B150700E87F880021A3A90021C3BF00EA
:10404000C1CFB3000140600021E3B70000CEB30050
:104050002063B7002043A90023C3BF007F40600056
:1040600023E3B7002343A80022C3BF0031CCB30031
:10407000014060008041B30022E3B7002223A80082
:104080002203A90025E3A800F0C1B3002563B7000F
:1040900000382E0060198800300020005019880078
:1040A00010C62700801988008001EB0043198800A2
:1040B00095A0A80067C164004411DD00AAC0BF003C
:1040C000F1C8B3000140600002407000AAE0B700F0
:1040D00040E32000E019880000E02700F019880084
:1040E0003DE3A800830C8800930C8800C0C1B30096
:1040F0009161B70010002000B00C8800B00C800067
:104100000005B000A00C88008080EB00F27F20004A
:104110000300200008007800E2E40700E07F800050
:104120000901780021F3290071E40700CC02A900FD
:10413000CC22A900CC42A900CC62A900CC82A90063
:10414000C802A900C822A900C842A900C862A900E3
:10415000C882A90020002000F07F880021E3A80089
:10416000000000000000000000000000000000004F
:10417000000000002043A800000000000000000034
:104180000000000000000000C802A8003D23A900B4
:1041900090C1BF0081CFB300014060000024A000A7
:1041A00090E1B700E07F80004FE407004F04BE00BD
:1041B0000000060074E7A90087E907000000FE0080
:1041C000000006002F02B00084C4BF004300DE00E0
:1041D000610060008086FB000004E0000300320004
:1041E000E0FF2F00B03B88000100370076A7EF000A
:1041F00070A7EF0072A7EF0074A7EF0078A7EF0099
:104200007AA7EF0000CEB3004260B70045C7BF00F9
:104210000044A1000046B30045E7B7000004EB00EE
:1042200008077800880478006055B8002C0020004A
:1042300040A7A8000040FE0040A7A90053E90700DE
:104240000800E000020032007607A9008804A800F8
:104250007007A9007647A90000E02700F019880040
:104260000029B000E019880025E3A80000382E00DE
:1042700060198800300020005019880021E3A80050
:1042800020002000401988008001EB00010220007E
:104290002023A800C842A8003C03A8004567A80046
:1042A00000000000000000003C03A9002023A9003A
:1042B000C842A9004567A90000188000808141001C
:1042C0008100E900F2FF3A000C00E0000A00320031
:1042D0000C06E90000FE2F000F0040008F00780060
:1042E00003187800810F5000FDFF3A000001200004
:1042F0000305B8000F0037000981440001FE2F00BC
:104300008280400061807F0000005500E0805D00F9
:1043100003054000E085480000FE2F000200400039
:1043200003B07F008904E800F08F540001003A00D8
:104330008C047800020120001100090042DDD80041
:1043400080007800D0152000808F500001003E00D2
:10435000E115200020EA2F0000804000808F5100EE
:10436000020039000007EB00040037000E07E800E8
:10437000E30F570001003A008EFF07007007A80006
:104380007647A8000800E000100032004567A8004A
:1043900084C4BF000028A30003003A0084C4BF0007
:1043A0000038A300FAFF32004567A90084C4BF00AB
:1043B0000038A300030032000D00E00003003A00C3
:1043C0007CFF07007607A8008006EB000800EA00E3
:1043D000080070004F00DE006104100094FF3700F9
:1043E0000600FA006680570041F021000400090031
:1043F000315878005000B10061DCBF0001C8B30043
:1044000001406000BFF8970001407000B0FF9F00BE
:1044100000C6210001D02100E681570004000900F8
:10442000335878005000B1005300B10065004000DF
:10443000810F5000F8FF3A000080FA0000000600EB
:10444000889FBE008A9FBE008C1F78008042780043
:1044500001427800834478008181FB000980FB00E1
:104460000080410001022000810F500002003C004A
:10447000094478000100370004C450008280FB002A
:10448000100020008105DD008880FB000585FB0011
:104490006519B900020045000CC621000C0040005F
:1044A0000B41780022100700894F540005003200AC
:1044B00088C054008180FB000C0045000B4178004F
:1044C0001B1007004F0678004F05BE004F04BE00CA
:1044D00000000600889FBE008A9FBE008C1F7800E7
:1044E0008042780001427800834478008181FB009B
:1044F0000980FB000080410001022000810F500074
:1045000002003C00094478000100370004C4500058
:104510008280FB00100020000100DD0080C5EA0061
:104520008880FB000585FB006519B9000200450085
:104530000CC621000C0040000B4178004110070020
:10454000894F54000500320088C054008180FB0070
:104550000C0045000B4178003A1007004F06780028
:104560004F05BE004F04BE0000000600889FBE003D
:104570008A9FBE00004178008144780070C2B30079
:10458000804F51004A003E000280FB00C305DE0060
:104590000B457800674461008880FB001000200014
:1045A0000102DD00044178008B81FB0040F0210016
:1045B0006340780080406200FFCF540039003E0025
:1045C0000904E00007003A0000C621000104E000F1
:1045D00002003200008041000F00370004C1EA00F1
:1045E000050037000104E0000E003A001D0037000E
:1045F00002C1EA0000C62100008041000102200043
:10460000101007002A0037000A80FB0001C62100B5
:10461000010040000441780001022000C40F07009F
:1046200023003700894178000841780088407800ED
:104630000B407800A7FF070089404400FFCF5000DF
:104640000200360000CEB30080C0400003C2B300B9
:1046500089C15100084178000B40780078FF0700BD
:1046600013003700894178000841780088407800BD
:104670000B40780072FF070089404400FFCF5000D4
:104680000200360000CEB30080C0400003C2B30079
:1046900089C15100084178000A4078008DFF070069
:1046A000030037000104E000D1FF3A00D6FF3700D5
:1046B0004F05BE004F04BE0000000600D5A2A900B1
:1046C000D7130700803E2000A51307004022EF000B
:1046D0004382A9004362A9004342A9004322A900E2
:1046E0004302A90042E2A90042C2A90042A2A800D6
:1046F00042C2BF0031CEB300014060008041B30030
:1047000042E2B70030C0B3004262B70010002000A0
:104710002012880041E2A80004DFBF000080FB00F7
:104720004012880005DFBF000080FB0040128800B7
:1047300006DFBF000080FB004012880007DFBF00DB
:104740000080FB004012880008DFBF000080FB00F3
:10475000401288008002200081130700D5A2A80023
:1047600045F021009542780054F021001442780071
:1047700063F021009341780072F02100124178002B
:1047800081F021009140780000C6210006D0210070
:104790000548780014409800234098003240980063
:1047A0004140980065004000860F5000F8FF3A0035
:1047B00000000600D5A2A9008002200068130700AF
:1047C00004DFBF000080FB004012880005DFBF004F
:1047D0000080FB004012880006DFBF000080FB0065
:1047E0004012880007DFBF000080FB0040128800F5
:1047F00008DFBF000080FB0040128800800220001C
:1048000057130700D5A2A80010002000541307007A
:10481000D5A2A90041E2A90086133700889FBE00F7
:104820008A9FBE008C9FBE008E1F780001447800D6
:104830008244780003457800844578000546780076
:1048400086467800074778008040780080C1B30032
:1048500046FF07008840780090C1B30043FF07007F
:1048600089407800A0C1B30040FF07008A4078006B
:10487000B0C1B3003DFF07008B407800C0C1B3005A
:104880003AFF07008C40780040C2B30037FF0700B2
:104890008D40780050C2B30034FF07008E4078008E
:1048A000F0C1B30031FF07004F0778004F06BE008C
:1048B0004F05BE004F04BE0000000600889FBE00EA
:1048C00001447800824478008040780020C0B30022
:1048D00026FF07008840780030C0B30023FF0700A0
:1048E0008940780040C0B30020FF07004F04BE009D
:1048F00000000600889FBE000144780082447800D2
:1049000080407800B0C0B30018FF070088407800EE
:10491000C0C0B30015FF070089407800D0C0B300C5
:1049200012FF07004F04BE0000000600889FBE0073
:1049300001447800824478008040780080C0B30051
:104940000AFF07008840780090C0B30007FF070007
:1049500089407800A0C0B30004FF07004F04BE00E8
:104960000000060021042000914078008180FB00B7
:10497000C508DE0092028000FF3FFC0000CEB300BD
:104980004260B700920288000500FC00500520003C
:10499000303B8800A00A2000303B880061E7A80077
:1049A000000000000000000061E7AF00FEFF3700DC
:1049B00092028000FF3FFC00C508DD0042C0BF003E
:1049C0007F4060000140700042E0B7009202880022
:1049D000000006000001BE009401800093018800E1
:1049E0001080BA001201BA0094018800800078009B
:1049F00002007800000006000002BE009201800064
:104A0000950188001000BA0092018800000006009D
:104A10000002BE0092018000950188001080BA005B
:104A2000920188000080FB0000000600E887470034
:104A3000889FBE008A9FBE008C9FBE008E1F78009C
:104A40000005BE00F2B79F0083BF9F00405EDE00FE
:104A50000D0020007FB097006104B800610046009F
:104A6000E0804E00C000DD00000020000A00500081
:104A70008B8058008100D1000080D30032002000DC
:104A8000030020006CAF0700800F5400818F5C0092
:104A9000010036000004BE00080778003200200044
:104AA000110009000284D800800378000103780017
:104AB00090018000E0B79F009C0188000A02BE00C0
:104AC0000FB997008001EB000A0037001400BA000C
:104AD000004978004800DE00104198009480BA0038
:104AE00021419800630141008301E8006202420015
:104AF000E0824A00878F5100F4FF39000600E00091
:104B0000060032001400BA0000597800E10F53008B
:104B1000020036004800DE00004978006FB09700C0
:104B20009001880032002000030020000800BE0031
:104B30004FAF070000004000818048000A05400098
:104B40008B8548000FB897000E00400080BF9F0083
:104B50007FB097000E005000F0B79F00BBFF3A00F7
:104B60004F0778004F06BE004F05BE004F04BE0041
:104B70008F00B100000006000400FA00881F7800D2
:104B8000D0BF9F00E1BF9F000001BE00F03FB20018
:104B900005003200E681570012E02000210A2000C3
:104BA00020722A00AF12070098018000930188004C
:104BB00020042400003B88006110B8000008BB00FE
